******************************************************************************
                  TMS470 Linker PC v4.9.5                      
******************************************************************************
>> Linked Fri May 27 13:45:57 2016

OUTPUT FILE NAME:   <modbus_cpld_20160527.out>
ENTRY POINT SYMBOL: "_c_int00"  address: 00208379


MEMORY CONFIGURATION

         name            origin    length      used     unused   attr    fill
----------------------  --------  ---------  --------  --------  ----  --------
  BOOTROM               00000000   00010000  00000000  00010000  R  X
  FLASH_BOOT            00200030   00000004  00000004  00000000  RW X
  FLASH                 00200034   0007ff9c  0000c6d3  000738c9  RW X
  C03SRAM               20000000   00008000  00002cf8  00005308  RW X
  S07SHRAM              20008000   00010000  00001956  0000e6aa  RW X
  CTOMMSGRAM            2007f000   00000800  00000000  00000800  R   
  MTOCMSGRAM            2007f800   00000800  00000000  00000800  RW  


SEGMENT ALLOCATION MAP

run origin  load origin   length   init length attrs members
----------  ----------- ---------- ----------- ----- -------
00200030    00200030    00000004   00000004    r-x
  00200030    00200030    00000004   00000004    r-x .ti_catalog_arm_cortexm3_concertoInit_begin
00200040    00200040    0000c199   0000c199    r-x
  00200040    00200040    000001ac   000001ac    r-- .resetVecs
  002001ec    002001ec    00009862   00009862    r-x .text
  00209a50    00209a50    00002789   00002789    r-- .const
0020c218    0020c218    00000500   00000500    r--
  0020c218    0020c218    000004f0   000004f0    r-- .cinit
  0020c708    0020c708    00000010   00000010    r-- .binit
20000000    20000000    000001ac   00000000    rw-
  20000000    20000000    000001ac   00000000    rw- .vecs
200001ac    0020c1dc    0000003c   0000003c    r-x
  200001ac    0020c1dc    0000003c   0000003c    r-x .flashfuncs
200001e8    200001e8    00002b10   00000000    rw-
  200001e8    200001e8    00002b10   00000000    rw- .bss
20008000    20008000    00001000   00000000    rw-
  20008000    20008000    00001000   00000000    rw- .stack
20009000    20009000    00000956   00000956    rw-
  20009000    20009000    00000956   00000956    rw- .data


SECTION ALLOCATION MAP

 output                                  attributes/
section   page    origin      length       input sections
--------  ----  ----------  ----------   ----------------
.bootVecs 
*          0    00000000    00000008     DSECT
                  00000000    00000008     boot.aem3 : boot.oem3 (.bootVecs)

xdc.meta   0    00000000    000000e8     COPY SECTION
                  00000000    000000e8     modbus_comm_pem3.oem3 (xdc.meta)

.ti_catalog_arm_cortexm3_concertoInit_begin 
*          0    00200030    00000004     
                  00200030    00000004     Boot.aem3 : Boot_asm.oem3 (.ti_catalog_arm_cortexm3_concertoInit_begin)

.resetVecs 
*          0    00200040    000001ac     
                  00200040    000001ac     modbus_comm_pem3.oem3 (.resetVecs)

.text      0    002001ec    00009862     
                  002001ec    00000970     driverlib.lib : sysctl.obj (.text)
                  00200b5c    00000450                   : gpio.obj (.text)
                  00200fac    000003d8     sysbios.lib : BIOS.obj (.text:ti_sysbios_family_arm_m3_Hwi_excDumpRegs__I)
                  00201384    0000036c     rtsv7M3_T_le_eabi.lib : lowlev.obj (.text)
                  002016f0    00000310     ti.targets.arm.rtsarm.aem3 : System.oem3 (.text:xdc_runtime_System_doPrint__I)
                  00201a00    000002ec     ti.sysbios.fatfs.aem3 : ff.oem3 (.text:chk_mounted)
                  00201cec    000002ec     rtsv7M3_T_le_eabi.lib : trgdrv.obj (.text)
                  00201fd8    000002a8     driverlib.lib : uart.obj (.text)
                  00202280    0000025c                   : interrupt.obj (.text)
                  002024dc    00000250     sysbios.lib : BIOS.obj (.text:ti_sysbios_heaps_HeapMem_free__E)
                  0020272c    00000250                 : BIOS.obj (.text:ti_sysbios_utils_Load_update__E)
                  0020297c    00000238                 : BIOS.obj (.text:ti_sysbios_heaps_HeapMem_alloc__E)
                  00202bb4    0000022c                 : BIOS.obj (.text:ti_sysbios_knl_Task_Instance_finalize__F)
                  00202de0    000001de     ti.sysbios.fatfs.aem3 : ff.oem3 (.text:f_write)
                  00202fbe    00000002     sysbios.lib : BIOS.obj (.text:nullFunc$0)
                  00202fc0    000001dc                 : BIOS.obj (.text:ti_sysbios_knl_Task_Instance_init__F)
                  0020319c    000001d8     Boot.aem3 : Boot.oem3 (.text:.bootCodeSection)
                  00203374    000001d4     sysbios.lib : BIOS.obj (.text:ti_sysbios_utils_Load_logLoads__I)
                  00203548    000001cc                 : BIOS.obj (.text:ti_sysbios_knl_Semaphore_pend__E)
                  00203714    000001ac     ti.uia.runtime.aem3 : LoggerStopMode.oem3 (.text:ti_uia_runtime_LoggerStopMode_write8__E)
                  002038c0    000001a4     ti.sysbios.fatfs.aem3 : ff.oem3 (.text:f_read)
                  00203a64    0000018c     gpio_mware.aem3 : GPIO.oem3 (.text:GPIO_write)
                  00203bf0    0000018c     sysbios.lib : BIOS.obj (.text:ti_sysbios_family_arm_m3_Hwi_excHandlerMax__I)
                  00203d7c    0000018a     ti.sysbios.fatfs.aem3 : ff.oem3 (.text:f_lseek)
                  00203f06    00000002     sysbios.lib : BIOS.obj (.text:ti_sysbios_family_arm_lm3_Timer_setNextTick__E)
                  00203f08    00000164     ti.uia.runtime.aem3 : LoggerStopMode.oem3 (.text:ti_uia_runtime_LoggerStopMode_writeMemoryRange__E)
                  0020406c    00000154     modbus_main.obj (.text:UartTask)
                  002041c0    00000152     ti.sysbios.fatfs.aem3 : ff.oem3 (.text:f_open)
                  00204312    00000002     sysbios.lib : BIOS.obj (.text:ti_sysbios_gates_GateHwi_Instance_init__F)
                  00204314    00000150     ti.targets.arm.rtsarm.aem3 : Core-mem.oem3 (.text:xdc_runtime_Core_createObject__I)
                  00204464    0000014c     ti.uia.runtime.aem3 : LoggerStopMode.oem3 (.text:ti_uia_runtime_LoggerStopMode_write4__E)
                  002045b0    0000013c     ti.targets.arm.rtsarm.aem3 : Error.oem3 (.text:xdc_runtime_Error_raiseX__F)
                  002046ec    00000128     sysbios.lib : BIOS.obj (.text:ti_sysbios_family_arm_m3_Hwi_dispatchC__I)
                  00204814    00000128                 : BIOS.obj (.text:ti_sysbios_knl_Clock_Instance_init__F)
                  0020493c    00000128                 : BIOS.obj (.text:ti_sysbios_knl_Clock_workFunc__E)
                  00204a64    00000128                 : BIOS.obj (.text:ti_sysbios_knl_Task_exit__E)
                  00204b8c    00000126     ti.sysbios.fatfs.aem3 : ff.oem3 (.text:f_rename)
                  00204cb2    00000002     --HOLE-- [fill = 0]
                  00204cb4    00000120     driverlib.lib : ssi.obj (.text)
                  00204dd4    00000120     sysbios.lib : BIOS.obj (.text:ti_sysbios_family_arm_m3_Hwi_Module_startup__F)
                  00204ef4    00000114                 : BIOS.obj (.text:ti_sysbios_knl_Swi_run__I)
                  00205008    00000113     ti.sysbios.fatfs.aem3 : ff.oem3 (.text:create_name)
                  0020511b    00000001     --HOLE-- [fill = 0]
                  0020511c    00000110     modbus_main.obj (.text:main)
                  0020522c    00000110     sysbios.lib : BIOS.obj (.text:ti_sysbios_knl_Task_schedule__I)
                  0020533c    00000104                 : m3_Hwi_asm.obj (.text:ti_sysbios_family_arm_m3_Hwi_dispatch__I)
                  00205440    00000104     modbus_main.obj (.text:uart1Isr)
                  00205544    000000fc     ti.targets.arm.rtsarm.aem3 : Startup.oem3 (.text:xdc_runtime_Startup_startMods__I)
                  00205640    000000f8     sysbios.lib : BIOS.obj (.text:ti_sysbios_knl_Task_postInit__I)
                  00205738    000000f4                 : BIOS.obj (.text:ti_sysbios_knl_Task_startup__E)
                  0020582c    000000f2     ti.sysbios.fatfs.aem3 : ff.oem3 (.text:dir_next)
                  0020591e    000000ee     modbus_comm_pem3.oem3 (.text:xdc_runtime_System_printfExtend__I)
                  00205a0c    000000ea     ti.sysbios.fatfs.aem3 : ff.oem3 (.text:put_fat)
                  00205af6    00000002     --HOLE-- [fill = 0]
                  00205af8    000000d4     sysbios.lib : BIOS.obj (.text:ti_sysbios_family_arm_lm3_Timer_enableTimers__I)
                  00205bcc    000000d0                 : BIOS.obj (.text:ti_sysbios_family_arm_m3_Hwi_excUsageFault__I)
                  00205c9c    000000ce     ti.sysbios.fatfs.aem3 : ff.oem3 (.text:get_fat)
                  00205d6a    00000002     --HOLE-- [fill = 0]
                  00205d6c    000000cc     rtsv7M3_T_le_eabi.lib : dtor_list.obj (.text)
                  00205e38    000000c0     ti.sysbios.fatfs.aem3 : ff.oem3 (.text:sync)
                  00205ef8    000000c0     sysbios.lib : BIOS.obj (.text:ti_sysbios_family_arm_lm3_Timer_startup__E)
                  00205fb8    000000c0                 : BIOS.obj (.text:ti_sysbios_heaps_HeapMem_Instance_init__F)
                  00206078    000000c0                 : BIOS.obj (.text:ti_sysbios_knl_Task_unblockI__E)
                  00206138    000000be     ti.sysbios.fatfs.aem3 : ff.oem3 (.text:f_sync)
                  002061f6    000000be                           : ff.oem3 (.text:f_unlink)
                  002062b4    000000bc     sysbios.lib : BIOS.obj (.text:ti_sysbios_knl_Semaphore_post__E)
                  00206370    000000b8                 : BIOS.obj (.text:ti_sysbios_family_arm_m3_Hwi_excBusFault__I)
                  00206428    000000b8                 : BIOS.obj (.text:ti_sysbios_utils_Load_idleFxn__E)
                  002064e0    000000b4                 : BIOS.obj (.text:ti_sysbios_family_arm_m3_Hwi_excHardFault__I)
                  00206594    000000b4                 : BIOS.obj (.text:ti_sysbios_gates_GateMutex_enter__E)
                  00206648    000000b0                 : BIOS.obj (.text:ti_sysbios_family_arm_m3_Hwi_excDebugMon__I)
                  002066f8    000000ac     driverlib.lib : watchdog.obj (.text)
                  002067a4    000000ac     ti.sysbios.fatfs.aem3 : ffcio.oem3 (.text:ffcio_open)
                  00206850    000000ac     sysbios.lib : BIOS.obj (.text:ti_sysbios_knl_Clock_Instance_finalize__F)
                  002068fc    000000ac                 : BIOS.obj (.text:ti_sysbios_knl_Swi_post__E)
                  002069a8    000000ac                 : BIOS.obj (.text:ti_sysbios_knl_Task_checkStacks__E)
                  00206a54    000000a8                 : BIOS.obj (.text:ti_sysbios_knl_Semaphore_Instance_init__F)
                  00206afc    000000a8                 : BIOS.obj (.text:ti_sysbios_knl_Swi_schedule__I)
                  00206ba4    000000a8                 : BIOS.obj (.text:ti_sysbios_utils_Load_addTask__E)
                  00206c4c    000000a4                 : BIOS.obj (.text:ti_sysbios_family_arm_m3_Hwi_excMemFault__I)
                  00206cf0    000000a0     auto_init.aem3 : auto_init.oem3 (.text)
                  00206d90    000000a0     sysbios.lib : BIOS.obj (.text:ti_sysbios_knl_Task_blockI__E)
                  00206e30    0000009c     rtsv7M3_T_le_eabi.lib : memcpy_t2.obj (.text)
                  00206ecc    00000096     ti.sysbios.fatfs.aem3 : ff.oem3 (.text:create_chain)
                  00206f62    00000002     --HOLE-- [fill = 0]
                  00206f64    00000092     ti.targets.arm.rtsarm.aem3 : Text.oem3 (.text:xdc_runtime_Text_putSite__F)
                  00206ff6    00000002     --HOLE-- [fill = 0]
                  00206ff8    00000090                                : Text.oem3 (.text:xdc_runtime_Text_putMod__F)
                  00207088    0000008c     sysbios.lib : BIOS.obj (.text:ti_sysbios_utils_Load_taskCreateHook__E)
                  00207114    00000084     TMDXDOCKH52C1.obj (.text:TMDXDOCKH52C1_initGeneral)
                  00207198    00000082     ti.sysbios.fatfs.aem3 : ff.oem3 (.text:dir_sdi)
                  0020721a    00000002     --HOLE-- [fill = 0]
                  0020721c    00000080     sysbios.lib : BIOS.obj (.text:ti_sysbios_family_arm_lm3_Timer_Module_startup__F)
                  0020729c    00000080                 : BIOS.obj (.text:ti_sysbios_knl_Task_Module_startup__F)
                  0020731c    00000080     ti.uia.runtime.aem3 : LoggerStopMode.oem3 (.text:ti_uia_runtime_LoggerStopMode_getContents__E)
                  0020739c    00000080                         : LoggerStopMode.oem3 (.text:ti_uia_runtime_LoggerStopMode_setFilterLevel__E)
                  0020741c    00000078     uart_mware.aem3 : UART.oem3 (.text:UART_init)
                  00207494    00000078     ti.sysbios.fatfs.aem3 : ff.oem3 (.text:follow_path)
                  0020750c    00000078     rtsv7M3_T_le_eabi.lib : memset_t2.obj (.text)
                  00207584    00000078     sysbios.lib : BIOS.obj (.text:ti_sysbios_utils_Load_taskDeleteHook__E)
                  002075fc    00000074     ti.uia.runtime.aem3 : LoggerStopMode.oem3 (.text:ti_uia_runtime_LoggerStopMode_getFilterLevel__E)
                  00207670    00000070     ti.sysbios.fatfs.aem3 : ff.oem3 (.text:check_fs)
                  002076e0    00000070     sysbios.lib : BIOS.obj (.text:rtsUnlock$0)
                  00207750    00000070                 : BIOS.obj (.text:ti_sysbios_knl_Clock_start__E)
                  002077c0    00000070                 : BIOS.obj (.text:ti_sysbios_utils_Load_removeTask__E)
                  00207830    00000070     ti.targets.arm.rtsarm.aem3 : Memory.oem3 (.text:xdc_runtime_Memory_alloc__F)
                  002078a0    0000006c     ti.sysbios.fatfs.aem3 : ff.oem3 (.text:move_window)
                  0020790c    0000006c     ti.uia.runtime.aem3 : LoggerStopMode.oem3 (.text:ti_uia_runtime_LoggerStopMode_writeBlockOfMemory__I)
                  00207978    0000006c     ti.targets.arm.rtsarm.aem3 : Error.oem3 (.text:xdc_runtime_Error_print__F)
                  002079e4    00000068     modbus_comm_pem3.oem3 (.text:ti_sysbios_knl_Task_Object__create__S)
                  00207a4c    00000066     ti.targets.arm.rtsarm.aem3 : Core-mem.oem3 (.text:xdc_runtime_Core_deleteObject__I)
                  00207ab2    00000064     ti.sysbios.fatfs.aem3 : ff.oem3 (.text:remove_chain)
                  00207b16    00000062                           : ff.oem3 (.text:dir_register)
                  00207b78    00000060     gpio_mware.aem3 : GPIO.oem3 (.text:GPIO_init)
                  00207bd8    00000060     rtsv7M3_T_le_eabi.lib : trgmsg.obj (.text)
                  00207c38    00000060     sysbios.lib : BIOS.obj (.text:ti_sysbios_knl_Clock_logTick__E)
                  00207c98    00000060                 : BIOS.obj (.text:ti_sysbios_knl_Clock_startI__E)
                  00207cf8    00000060     modbus_comm_pem3.oem3 (.text:ti_uia_runtime_LoggerStopMode_Object__create__S)
                  00207d58    0000005e     rtsv7M3_T_le_eabi.lib : copy_decompress_rle.obj (.text)
                  00207db6    0000005e     ti.uia.runtime.aem3 : LoggerStopMode.oem3 (.text:ti_uia_runtime_LoggerStopMode_readBlockOfMemory__I)
                  00207e14    00000057     ti.targets.arm.rtsarm.aem3 : Text.oem3 (.text:xdc_runtime_Text_putLab__F)
                  00207e6b    00000001     --HOLE-- [fill = 0]
                  00207e6c    00000054     sysbios.lib : BIOS.obj (.text:ti_sysbios_knl_Swi_restoreHwi__E)
                  00207ec0    00000050     TMDXDOCKH52C1.obj (.text:TMDXDOCKH52C1_initUART)
                  00207f10    00000050     sysbios.lib : BIOS.obj (.text:ti_sysbios_utils_Load_taskSwitchHook__E)
                  00207f60    00000050     ti.targets.arm.rtsarm.aem3 : Startup.oem3 (.text:xdc_runtime_Startup_exec__F)
                  00207fb0    00000050                                : System.oem3 (.text:xdc_runtime_System_formatNum__I)
                  00208000    0000004c     sysbios.lib : m3_TaskSupport_asm.obj (.text:_ti_sysbios_family_arm_m3_TaskSupport_buildTaskStack)
                  0020804c    0000004c     modbus_comm_pem3.oem3 (.text:ti_sysbios_fatfs_startup)
                  00208098    0000004c     sysbios.lib : BIOS.obj (.text:ti_sysbios_knl_Clock_getTicks__E)
                  002080e4    0000004c     ti.uia.runtime.aem3 : LoggerStopMode.oem3 (.text:ti_uia_runtime_LoggerStopMode_filterOutEvent__I)
                  00208130    0000004c                         : QueueDescriptor.oem3 (.text:ti_uia_runtime_QueueDescriptor_removeFromList__E)
                  0020817c    0000004c     ti.targets.arm.rtsarm.aem3 : Text.oem3 (.text:xdc_runtime_Text_visitRope2__I)
                  002081c8    00000048     rtsv7M3_T_le_eabi.lib : cpy_tbl.obj (.text)
                  00208210    00000048     sysbios.lib : BIOS.obj (.text:ti_sysbios_family_arm_m3_Hwi_excReserved__I)
                  00208258    00000048                 : BIOS.obj (.text:ti_sysbios_heaps_HeapMem_getStats__E)
                  002082a0    00000048     ti.targets.arm.rtsarm.aem3 : Assert.oem3 (.text:xdc_runtime_Assert_raise__I)
                  002082e8    00000048                                : Core-params.oem3 (.text:xdc_runtime_Core_assignParams__I)
                  00208330    00000046     ti.uia.runtime.aem3 : LoggerStopMode.oem3 (.text:ti_uia_runtime_LoggerStopMode_Instance_init__F)
                  00208376    00000002     --HOLE-- [fill = 0]
                  00208378    00000044     boot.aem3 : boot.oem3 (.text)
                  002083bc    00000044     ti.sysbios.fatfs.aem3 : ff.oem3 (.text:dir_find)
                  00208400    00000044     rtsv7M3_T_le_eabi.lib : exit.obj (.text)
                  00208444    00000044     sysbios.lib : BIOS.obj (.text:ti_sysbios_BIOS_errorRaiseHook__I)
                  00208488    00000044     ti.uia.runtime.aem3 : LoggerStopMode.oem3 (.text:ti_uia_runtime_LoggerStopMode_reset__F)
                  002084cc    00000044                         : QueueDescriptor.oem3 (.text:ti_uia_runtime_QueueDescriptor_addToList__E)
                  00208510    00000044     ti.targets.arm.rtsarm.aem3 : SysMin.oem3 (.text:xdc_runtime_SysMin_flush__F)
                  00208554    00000040     sysbios.lib : m3_Hwi_asm_switch.obj (.text:_ti_sysbios_family_xxx_Hwi_switchToIsrStack)
                  00208594    00000040     ti.sysbios.fatfs.aem3 : ff.oem3 (.text:dir_read)
                  002085d4    00000040     sysbios.lib : BIOS.obj (.text:ti_sysbios_knl_Idle_loop__E)
                  00208614    00000040                 : BIOS.obj (.text:ti_sysbios_knl_Swi_startup__E)
                  00208654    00000040     ti.targets.arm.rtsarm.aem3 : System.oem3 (.text:xdc_runtime_System_atexit__F)
                  00208694    0000003c     modbus_comm_pem3.oem3 (.text:ti_sysbios_family_arm_m3_Hwi_disableInterrupt__E)
                  002086d0    0000003c     modbus_comm_pem3.oem3 (.text:ti_sysbios_family_arm_m3_Hwi_enableInterrupt__E)
                  0020870c    0000003c     sysbios.lib : BIOS.obj (.text:ti_sysbios_family_arm_m3_Hwi_excSvCall__I)
                  00208748    0000003c                 : BIOS.obj (.text:ti_sysbios_heaps_HeapMem_init__I)
                  00208784    0000003c     modbus_comm_pem3.oem3 (.text:ti_sysbios_knl_Clock_Object__create__S)
                  002087c0    00000038     sysbios.lib : BIOS.obj (.text:ti_sysbios_family_arm_m3_Hwi_excNoIsr__I)
                  002087f8    00000038                 : BIOS.obj (.text:ti_sysbios_family_arm_m3_Hwi_initVTOR__I)
                  00208830    00000038                 : BIOS.obj (.text:ti_sysbios_family_arm_m3_TaskSupport_start__E)
                  00208868    00000038     modbus_comm_pem3.oem3 (.text:ti_sysbios_knl_Semaphore_Object__create__S)
                  002088a0    00000038     sysbios.lib : BIOS.obj (.text:ti_sysbios_knl_Semaphore_pendTimeout__I)
                  002088d8    00000038     ti.targets.arm.rtsarm.aem3 : SysMin.oem3 (.text:xdc_runtime_SysMin_putch__F)
                  00208910    00000036     driverlib.lib : cpu.obj (.text)
                  00208946    00000002     --HOLE-- [fill = 0]
                  00208948    00000034     TMDXDOCKH52C1.obj (.text:TMDXDOCKH52C1_initGPIO)
                  0020897c    00000034     ti.sysbios.fatfs.aem3 : ffcio.oem3 (.text:ffcio_lseek)
                  002089b0    00000034     sysbios.lib : BIOS.obj (.text:ti_sysbios_family_arm_m3_Hwi_excNmi__I)
                  002089e4    00000034     modbus_comm_pem3.oem3 (.text:ti_sysbios_gates_GateHwi_Object__create__S)
                  00208a18    00000034     modbus_comm_pem3.oem3 (.text:ti_sysbios_gates_GateMutex_Object__create__S)
                  00208a4c    00000034     modbus_comm_pem3.oem3 (.text:ti_sysbios_heaps_HeapMem_Object__create__S)
                  00208a80    00000034     modbus_comm_pem3.oem3 (.text:ti_sysbios_knl_Queue_Object__create__S)
                  00208ab4    00000034     sysbios.lib : BIOS.obj (.text:ti_sysbios_knl_Task_restore__E)
                  00208ae8    00000032     ti.sysbios.fatfs.aem3 : ff.oem3 (.text:validate)
                  00208b1a    00000002     --HOLE-- [fill = 0]
                  00208b1c    00000031     ti.targets.arm.rtsarm.aem3 : Text.oem3 (.text:xdc_runtime_Text_printVisFxn__I)
                  00208b4d    00000001     --HOLE-- [fill = 0]
                  00208b4e    00000030     rtsv7M3_T_le_eabi.lib : strncpy.obj (.text)
                  00208b7e    00000002     --HOLE-- [fill = 0]
                  00208b80    00000030     modbus_comm_pem3.oem3 (.text:ti_sysbios_BIOS_exitFunc__I)
                  00208bb0    00000030     sysbios.lib : BIOS.obj (.text:ti_sysbios_family_arm_lm3_Timer_getExpiredCounts__E)
                  00208be0    00000030                 : BIOS.obj (.text:ti_sysbios_hal_Hwi_checkStack:ti_sysbios_hal_Hwi_checkStack)
                  00208c10    00000030                 : BIOS.obj (.text:ti_sysbios_knl_Clock_Module_startup__F)
                  00208c40    00000030     ti.targets.arm.rtsarm.aem3 : Core-label.oem3 (.text:xdc_runtime_Core_assignLabel__I)
                  00208c70    00000030                                : SysMin.oem3 (.text:xdc_runtime_SysMin_abort__F)
                  00208ca0    00000030                                : Text.oem3 (.text:xdc_runtime_Text_xprintf__I)
                  00208cd0    0000002e     modbus_comm_pem3.oem3 (.text:malloc)
                  00208cfe    00000002     --HOLE-- [fill = 0]
                  00208d00    0000002c     TMDXDOCKH52C1.obj (.text:TMDXDOCKH52C1_setMaxSPIbitrate)
                  00208d2c    0000002c     sysbios.lib : BIOS.obj (.text:ti_sysbios_hal_Hwi_initStack:ti_sysbios_hal_Hwi_initStack)
                  00208d58    0000002c     modbus_comm_pem3.oem3 (.text:ti_sysbios_knl_Clock_doTick__I)
                  00208d84    0000002c     sysbios.lib : BIOS.obj (.text:ti_sysbios_knl_Task_allBlockedFunction__I)
                  00208db0    0000002c     ti.uia.runtime.aem3 : LoggerStopMode.oem3 (.text:ti_uia_runtime_LoggerStopMode_Module_startup__F)
                  00208ddc    0000002c                         : LoggerStopMode.oem3 (.text:ti_uia_runtime_LoggerStopMode_disable__E)
                  00208e08    0000002c                         : LoggerStopMode.oem3 (.text:ti_uia_runtime_LoggerStopMode_enable__E)
                  00208e34    0000002c     ti.targets.arm.rtsarm.aem3 : System.oem3 (.text:xdc_runtime_System_rtsExit__I)
                  00208e60    0000002c                                : Text.oem3 (.text:xdc_runtime_Text_cordText__F)
                  00208e8c    00000028     modbus_comm_pem3.oem3 (.text:ti_sysbios_BIOS_startFunc__I)
                  00208eb4    00000028     sysbios.lib : BIOS.obj (.text:ti_sysbios_family_arm_f28m35x_TimestampProvider_get64__E)
                  00208edc    00000028                 : BIOS.obj (.text:ti_sysbios_gates_GateMutex_Instance_init__F)
                  00208f04    00000028     modbus_main.obj (.text:ti_sysbios_knl_Task_create)
                  00208f2c    00000028     ti.uia.runtime.aem3 : LogSync.oem3 (.text:ti_uia_runtime_LogSync_Module_startup__F)
                  00208f54    00000028                         : QueueDescriptor.oem3 (.text:ti_uia_runtime_QueueDescriptor_initHeader__E)
                  00208f7c    00000024     ti.sysbios.fatfs.aem3 : ff.oem3 (.text:dir_remove)
                  00208fa0    00000024                           : ffcio.oem3 (.text:ffcio_close)
                  00208fc4    00000024                           : ff.oem3 (.text:mem_cmp)
                  00208fe8    00000024     sysbios.lib : BIOS.obj (.text:ti_sysbios_BIOS_registerRTSLock__I)
                  0020900c    00000024                 : BIOS.obj (.text:ti_sysbios_family_arm_lm3_Timer_isrStub__E)
                  00209030    00000024                 : BIOS.obj (.text:ti_sysbios_family_arm_m3_Hwi_doTaskRestore__I)
                  00209054    00000024     modbus_comm_pem3.oem3 (.text:ti_sysbios_gates_GateMutex_Object__delete__S)
                  00209078    00000024     sysbios.lib : BIOS.obj (.text:ti_sysbios_knl_Swi_Module_startup__F)
                  0020909c    00000024     ti.uia.runtime.aem3 : LoggerStopMode.oem3 (.text:ti_uia_runtime_LoggerStopMode_Instance_finalize__F)
                  002090c0    00000022     modbus_comm_pem3.oem3 (.text:xdc_runtime_SysMin_output__I)
                  002090e2    00000002     --HOLE-- [fill = 0]
                  002090e4    00000020     ti.sysbios.fatfs.aem3 : ffcio.oem3 (.text:ffcio_read)
                  00209104    00000020                           : ffcio.oem3 (.text:ffcio_write)
                  00209124    00000020     modbus_comm_pem3.oem3 (.text:ti_sysbios_gates_GateHwi_Object__delete__S)
                  00209144    00000020     modbus_comm_pem3.oem3 (.text:ti_sysbios_heaps_HeapMem_Object__delete__S)
                  00209164    00000020     modbus_comm_pem3.oem3 (.text:ti_sysbios_knl_Clock_Object__destruct__S)
                  00209184    00000020     modbus_comm_pem3.oem3 (.text:ti_sysbios_knl_Semaphore_Object__destruct__S)
                  002091a4    00000020     sysbios.lib : BIOS.obj (.text:ti_sysbios_knl_Task_enter__I)
                  002091c4    00000020     modbus_comm_pem3.oem3 (.text:ti_uia_runtime_LoggerStopMode_Object__delete__S)
                  002091e4    00000020     ti.targets.arm.rtsarm.aem3 : Registry.oem3 (.text:xdc_runtime_Registry_findById__F)
                  00209204    00000020                                : SysMin.oem3 (.text:xdc_runtime_SysMin_Module_startup__F)
                  00209224    00000020                                : System.oem3 (.text:xdc_runtime_System_avprintf__F)
                  00209244    00000020                                : System.oem3 (.text:xdc_runtime_System_putchar__I)
                  00209264    00000020                                : System.oem3 (.text:xdc_runtime_System_vprintf__F)
                  00209284    0000001c     ti.sysbios.fatfs.aem3 : diskio.oem3 (.text:disk_initialize)
                  002092a0    0000001c                           : diskio.oem3 (.text:disk_ioctl)
                  002092bc    0000001c                           : diskio.oem3 (.text:disk_read)
                  002092d8    0000001c                           : diskio.oem3 (.text:disk_status)
                  002092f4    0000001c                           : diskio.oem3 (.text:disk_write)
                  00209310    0000001c     modbus_comm_pem3.oem3 (.text:free)
                  0020932c    0000001c     sysbios.lib : BIOS.obj (.text:rtsLock$0)
                  00209348    0000001c     modbus_comm_pem3.oem3 (.text:ti_sysbios_knl_Queue_Object__destruct__S)
                  00209364    0000001c     ti.targets.arm.rtsarm.aem3 : Error.oem3 (.text:xdc_runtime_Error_check__F)
                  00209380    0000001c                                : Memory.oem3 (.text:xdc_runtime_Memory_valloc__F)
                  0020939c    0000001c                                : SysMin.oem3 (.text:xdc_runtime_SysMin_exit__F)
                  002093b8    0000001a     modbus_comm_pem3.oem3 (.text:ti_sysbios_gates_GateHwi_Handle__label__S)
                  002093d2    0000001a     modbus_comm_pem3.oem3 (.text:ti_sysbios_gates_GateMutex_Handle__label__S)
                  002093ec    0000001a     modbus_comm_pem3.oem3 (.text:ti_sysbios_heaps_HeapMem_Handle__label__S)
                  00209406    0000001a     modbus_comm_pem3.oem3 (.text:ti_uia_runtime_LoggerStopMode_Handle__label__S)
                  00209420    0000001a     modbus_comm_pem3.oem3 (.text:xdc_runtime_System_aprintf__E)
                  0020943a    0000001a     modbus_comm_pem3.oem3 (.text:xdc_runtime_System_printf__E)
                  00209454    00000018     ti.sysbios.fatfs.aem3 : ff.oem3 (.text:clust2sect)
                  0020946c    00000018     rtsv7M3_T_le_eabi.lib : _lock.obj (.text)
                  00209484    00000018                           : args_main.obj (.text)
                  0020949c    00000018                           : strcmp.obj (.text)
                  002094b4    00000018     modbus_comm_pem3.oem3 (.text:ti_sysbios_family_arm_lm3_Timer_Module__startupDone__F)
                  002094cc    00000018     modbus_comm_pem3.oem3 (.text:ti_sysbios_family_arm_m3_Hwi_Module__startupDone__F)
                  002094e4    00000018     sysbios.lib : BIOS.obj (.text:ti_sysbios_gates_GateMutex_leave__E)
                  002094fc    00000018     modbus_comm_pem3.oem3 (.text:ti_sysbios_hal_Timer_Module__startupDone__F)
                  00209514    00000018     ti.sysbios.fatfs.aem3 : ff.oem3 (.text:unlock_fs)
                  0020952c    00000018     ti.targets.arm.rtsarm.aem3 : Text.oem3 (.text:xdc_runtime_Text_ropeText__F)
                  00209544    00000016     rtsv7M3_T_le_eabi.lib : strchr.obj (.text)
                  0020955a    00000016     modbus_main.obj (.text:ti_sysbios_knl_Task_Params_init)
                  00209570    00000016     ti.uia.runtime.aem3 : LoggerStopMode.oem3 (.text:ti_uia_runtime_LoggerStopMode_getFreeSize__E)
                  00209586    00000016                         : LoggerStopMode.oem3 (.text:ti_uia_runtime_LoggerStopMode_getUnreadSize__E)
                  0020959c    00000014     rtsv7M3_T_le_eabi.lib : strlen.obj (.text)
                  002095b0    00000014     sysbios.lib : BIOS.obj (.text:ti_sysbios_family_arm_m3_Hwi_switchFromBootStack__E)
                  002095c4    00000014                 : BIOS.obj (.text:ti_sysbios_gates_GateHwi_enter__E)
                  002095d8    00000014     modbus_comm_pem3.oem3 (.text:ti_sysbios_heaps_HeapMem_Object__get__S)
                  002095ec    00000014     modbus_comm_pem3.oem3 (.text:ti_sysbios_knl_Swi_Object__get__S)
                  00209600    00000014     modbus_comm_pem3.oem3 (.text:ti_sysbios_knl_Task_Object__first__S)
                  00209614    00000014     modbus_comm_pem3.oem3 (.text:ti_sysbios_knl_Task_Object__get__S)
                  00209628    00000014     modbus_comm_pem3.oem3 (.text:ti_sysbios_knl_Task_Object__next__S)
                  0020963c    00000014     ti.uia.runtime.aem3 : LoggerStopMode.oem3 (.text:ti_uia_runtime_LoggerStopMode_write2__E)
                  00209650    00000014     ti.targets.arm.rtsarm.aem3 : System.oem3 (.text:xdc_runtime_System_abort__F)
                  00209664    00000012     rtsv7M3_T_le_eabi.lib : copy_zero_init.obj (.text:decompress:ZI)
                  00209676    00000012     ti.sysbios.fatfs.aem3 : ffcio.oem3 (.text:ffcio_rename)
                  00209688    00000012                           : ffcio.oem3 (.text:ffcio_unlink)
                  0020969a    00000012     rtsv7M3_T_le_eabi.lib : strcpy.obj (.text)
                  002096ac    00000012     sysbios.lib : BIOS.obj (.text:ti_sysbios_hal_Hwi_Module_startup__F)
                  002096be    00000012                 : BIOS.obj (.text:ti_sysbios_hal_Timer_Module_startup__F)
                  002096d0    00000012     ti.uia.runtime.aem3 : LoggerStopMode.oem3 (.text:ti_uia_runtime_LoggerStopMode_write1__E)
                  002096e2    00000012     modbus_comm_pem3.oem3 (.text:xdc_runtime_Startup_exec__I)
                  002096f4    00000010     modbus_main.obj (.text:SEM_pend)
                  00209704    00000010     sysbios.lib : m3_TaskSupport_asm.obj (.text:_ti_sysbios_family_arm_m3_TaskSupport_glue)
                  00209714    00000010                 : m3_TaskSupport_asm.obj (.text:_ti_sysbios_family_arm_m3_TaskSupport_swap__E)
                  00209724    00000010     ti.sysbios.fatfs.aem3 : ff.oem3 (.text:chk_chr)
                  00209734    00000010                           : ff.oem3 (.text:f_close)
                  00209744    00000010                           : ff.oem3 (.text:mem_cpy)
                  00209754    00000010     sysbios.lib : BIOS.obj (.text:ti_sysbios_BIOS_setThreadType__E)
                  00209764    00000010                 : BIOS.obj (.text:ti_sysbios_BIOS_start__E)
                  00209774    00000010                 : BIOS.obj (.text:ti_sysbios_family_arm_f28m35x_TimestampProvider_getFreq__E)
                  00209784    00000010                 : BIOS.obj (.text:ti_sysbios_family_arm_m3_Hwi_excHandler__I)
                  00209794    00000010                 : BIOS.obj (.text:ti_sysbios_gates_GateMutex_Instance_finalize__F)
                  002097a4    00000010                 : BIOS.obj (.text:ti_sysbios_knl_Semaphore_Instance_finalize__F)
                  002097b4    00000010                 : BIOS.obj (.text:ti_sysbios_knl_Swi_disable__E)
                  002097c4    00000010                 : BIOS.obj (.text:ti_sysbios_knl_Task_disable__E)
                  002097d4    00000010     modbus_comm_pem3.oem3 (.text:ti_uia_runtime_LoggerStopMode_Object__get__S)
                  002097e4    00000010     ti.uia.runtime.aem3 : LoggerStopMode.oem3 (.text:ti_uia_runtime_LoggerStopMode_isEmpty__E)
                  002097f4    00000010                         : LoggerStopMode.oem3 (.text:ti_uia_runtime_LoggerStopMode_write0__E)
                  00209804    00000010     ti.targets.arm.rtsarm.aem3 : Gate.oem3 (.text:xdc_runtime_Gate_leaveSystem__F)
                  00209814    00000010                                : Memory.oem3 (.text:xdc_runtime_Memory_free__F)
                  00209824    00000010                                : SysMin.oem3 (.text:xdc_runtime_SysMin_ready__F)
                  00209834    00000010     modbus_comm_pem3.oem3 (.text:xdc_runtime_Text_visitRope__I)
                  00209844    0000000e     rtsv7M3_T_le_eabi.lib : copy_decompress_none.obj (.text:decompress:none)
                  00209852    0000000e     ti.sysbios.fatfs.aem3 : ff.oem3 (.text:mem_set)
                  00209860    0000000e     sysbios.lib : BIOS.obj (.text:ti_sysbios_family_arm_m3_TaskSupport_checkStack__E)
                  0020986e    0000000e                 : BIOS.obj (.text:ti_sysbios_knl_Queue_empty__E)
                  0020987c    0000000e     ti.targets.arm.rtsarm.aem3 : System.oem3 (.text:xdc_runtime_System_vsprintf__F)
                  0020988a    0000000c     modbus_comm_pem3.oem3 (.text:.bootCodeSection:ti_catalog_arm_cortexm3_concertoInit_Boot_init)
                  00209896    0000000c     modbus_comm_pem3.oem3 (.text:.bootCodeSection:ti_catalog_arm_cortexm3_concertoInit_Boot_initStartup)
                  002098a2    0000000c     modbus_main.obj (.text:SEM_post)
                  002098ae    00000002     --HOLE-- [fill = 0]
                  002098b0    0000000c     sysbios.lib : BIOS.obj (.text:ti_sysbios_family_arm_f28m35x_TimestampProvider_get32__E)
                  002098bc    0000000c                 : BIOS.obj (.text:ti_sysbios_family_arm_m3_TaskSupport_getStackAlignment__E)
                  002098c8    0000000c     modbus_comm_pem3.oem3 (.text:ti_sysbios_knl_Clock_Params__init__S)
                  002098d4    0000000c     modbus_comm_pem3.oem3 (.text:ti_sysbios_knl_Queue_Object__get__S)
                  002098e0    0000000c     modbus_comm_pem3.oem3 (.text:ti_sysbios_knl_Task_Params__init__S)
                  002098ec    0000000c     sysbios.lib : BIOS.obj (.text:ti_sysbios_utils_Load_taskRegHook__E)
                  002098f8    0000000c     ti.targets.arm.rtsarm.aem3 : Error.oem3 (.text:xdc_runtime_Error_init__F)
                  00209904    0000000c                                : Gate.oem3 (.text:xdc_runtime_Gate_enterSystem__F)
                  00209910    0000000c                                : Memory.oem3 (.text:xdc_runtime_Memory_calloc__F)
                  0020991c    0000000c                                : Memory.oem3 (.text:xdc_runtime_Memory_getMaxDefaultTypeAlign__F)
                  00209928    0000000c                                : System.oem3 (.text:xdc_runtime_System_exit__F)
                  00209934    0000000c                                : System.oem3 (.text:xdc_runtime_System_lastFxn__I)
                  00209940    0000000a     sysbios.lib : m3_IntrinsicsSupport_asm.obj (.text:_ti_sysbios_family_arm_m3_IntrinsicsSupport_maxbit)
                  0020994a    0000000a     modbus_comm_pem3.oem3 (.text:xdc_runtime_IHeap_alloc)
                  00209954    0000000a     modbus_comm_pem3.oem3 (.text:xdc_runtime_IHeap_free)
                  0020995e    00000008     ti.sysbios.fatfs.aem3 : syncsysbios.oem3 (.text:ff_req_grant)
                  00209966    00000008     sysbios.lib : BIOS.obj (.text:ti_sysbios_family_arm_m3_Hwi_startup__E)
                  0020996e    00000002     --HOLE-- [fill = 0]
                  00209970    00000008     modbus_comm_pem3.oem3 (.text:ti_sysbios_fatfs_getFatTime)
                  00209978    00000006     Boot.aem3 : Boot.oem3 (.text)
                  0020997e    00000002     --HOLE-- [fill = 0]
                  00209980    00000006     driverlib.lib : sysctl.obj (.text:SysCtlDelay)
                  00209986    00000006     ti.targets.arm.rtsarm.aem3 : xdc_noinit.oem3 (.text:__xdc__init)
                  0020998c    00000006     rtsv7M3_T_le_eabi.lib : copy_decompress_rle.obj (.text:decompress:rle24)
                  00209992    00000006     ti.sysbios.fatfs.aem3 : ff.oem3 (.text:lock_fs)
                  00209998    00000006     sysbios.lib : BIOS.obj (.text:ti_sysbios_family_arm_m3_Hwi_doSwiRestore__I)
                  0020999e    00000006                 : BIOS.obj (.text:ti_sysbios_gates_GateHwi_leave__E)
                  002099a4    00000006                 : BIOS.obj (.text:ti_sysbios_heaps_HeapMem_isBlocking__E)
                  002099aa    00000006                 : BIOS.obj (.text:ti_sysbios_knl_Queue_Instance_init__F)
                  002099b0    00000006     ti.uia.runtime.aem3 : LoggerStopMode.oem3 (.text:ti_uia_runtime_LoggerStopMode_getPriority__E)
                  002099b6    00000006                         : LoggerStopMode.oem3 (.text:ti_uia_runtime_LoggerStopMode_getTransferType__F)
                  002099bc    00000006     ti.targets.arm.rtsarm.aem3 : System.oem3 (.text:xdc_runtime_System_Module_startup__F)
                  002099c2    00000004     modbus_comm_pem3.oem3 (.text:.bootCodeSection:ti_catalog_arm_cortexm3_concertoInit_Boot_limpAbort)
                  002099c6    00000004     ti.sysbios.fatfs.aem3 : syncsysbios.oem3 (.text:ff_rel_grant)
                  002099ca    00000004     modbus_comm_pem3.oem3 (.text:ti_sysbios_BIOS_RtsGateProxy_enter__E)
                  002099ce    00000004     modbus_comm_pem3.oem3 (.text:ti_sysbios_BIOS_RtsGateProxy_leave__E)
                  002099d2    00000004     sysbios.lib : BIOS.obj (.text:ti_sysbios_family_arm_lm3_Timer_getPeriod__E)
                  002099d6    00000004     modbus_comm_pem3.oem3 (.text:ti_sysbios_family_arm_m3_TaskSupport_Module__startupDone__S)
                  002099da    00000004     sysbios.lib : BIOS.obj (.text:ti_sysbios_gates_GateHwi_query__F)
                  002099de    00000004                 : BIOS.obj (.text:ti_sysbios_gates_GateMutex_query__F)
                  002099e2    00000004     modbus_comm_pem3.oem3 (.text:ti_sysbios_hal_Hwi_HwiProxy_Module__startupDone__S)
                  002099e6    00000004     modbus_comm_pem3.oem3 (.text:ti_sysbios_hal_Timer_TimerProxy_Module__startupDone__S)
                  002099ea    00000004     modbus_comm_pem3.oem3 (.text:ti_sysbios_hal_Timer_TimerProxy_getExpiredCounts__E)
                  002099ee    00000004     modbus_comm_pem3.oem3 (.text:ti_sysbios_hal_Timer_TimerProxy_getPeriod__E)
                  002099f2    00000004     modbus_comm_pem3.oem3 (.text:ti_sysbios_hal_Timer_TimerProxy_setNextTick__E)
                  002099f6    00000004     modbus_comm_pem3.oem3 (.text:ti_sysbios_heaps_HeapMem_Module_GateProxy_enter__E)
                  002099fa    00000004     modbus_comm_pem3.oem3 (.text:ti_sysbios_heaps_HeapMem_Module_GateProxy_leave__E)
                  002099fe    00000004     modbus_comm_pem3.oem3 (.text:ti_sysbios_knl_Task_SupportProxy_Module__startupDone__S)
                  00209a02    00000004     modbus_comm_pem3.oem3 (.text:ti_uia_runtime_LogSync_CpuTimestampProxy_Module__startupDone__S)
                  00209a06    00000004     modbus_comm_pem3.oem3 (.text:ti_uia_runtime_LogSync_GlobalTimestampProxy_Module__startupDone__S)
                  00209a0a    00000004     ti.uia.runtime.aem3 : LoggerStopMode.oem3 (.text:ti_uia_runtime_LoggerStopMode_getInstanceId__E)
                  00209a0e    00000004                         : LoggerStopMode.oem3 (.text:ti_uia_runtime_LoggerStopMode_getMaxLength__E)
                  00209a12    00000004                         : LoggerStopMode.oem3 (.text:ti_uia_runtime_LoggerStopMode_setPriority__E)
                  00209a16    00000004     ti.targets.arm.rtsarm.aem3 : Error.oem3 (.text:xdc_runtime_Error_getSite__F)
                  00209a1a    00000004     modbus_comm_pem3.oem3 (.text:xdc_runtime_Memory_HeapProxy_alloc__E)
                  00209a1e    00000004     modbus_comm_pem3.oem3 (.text:xdc_runtime_Memory_HeapProxy_free__E)
                  00209a22    00000004     modbus_comm_pem3.oem3 (.text:xdc_runtime_Startup_reset__I)
                  00209a26    00000004     modbus_comm_pem3.oem3 (.text:xdc_runtime_System_Module_GateProxy_enter__E)
                  00209a2a    00000004     modbus_comm_pem3.oem3 (.text:xdc_runtime_System_Module_GateProxy_leave__E)
                  00209a2e    00000004     ti.targets.arm.rtsarm.aem3 : System.oem3 (.text:xdc_runtime_System_aprintf_va__F)
                  00209a32    00000004                                : System.oem3 (.text:xdc_runtime_System_printf_va__F)
                  00209a36    00000004     modbus_comm_pem3.oem3 (.text:xdc_runtime_System_vsprintf__E)
                  00209a3a    00000004     modbus_comm_pem3.oem3 (.text:xdc_runtime_TimestampNull_Module__startupDone__S)
                  00209a3e    00000004     modbus_comm_pem3.oem3 (.text:xdc_runtime_Timestamp_Module__startupDone__S)
                  00209a42    00000002     --HOLE-- [fill = 0]
                  00209a44    0000000a     Boot.aem3 : Boot.oem3 (.tramp.$.flashfuncs:D:\ti\mcusdk_1_00_00_68\products\xdctools_3_23_04_60\packages\ti\catalog\arm\cortexm3\concertoInit\lib\Boot.aem3<Boot.oem3>$0x0.1)

.const     0    00209a50    00002789     
                  00209a50    00001d7f     modbus_comm_pem3.oem3 (.const:xdc_runtime_Text_charTab__A)
                  0020b7cf    00000001     --HOLE-- [fill = 0]
                  0020b7d0    00000100     modbus_comm_pem3.oem3 (.const:xdc_runtime_Text_nodeTab__A)
                  0020b8d0    00000068     TMDXDOCKH52C1.obj (.const)
                  0020b938    00000060     modbus_comm_pem3.oem3 (.const:ti_uia_runtime_LoggerStopMode_Module__FXNS__C)
                  0020b998    00000054     driverlib.lib : sysctl.obj (.const)
                  0020b9ec    00000048                   : gpio.obj (.const:g_pulGPIOBaseAddrs)
                  0020ba34    00000048                   : interrupt.obj (.const:g_pulRegs)
                  0020ba7c    00000047     modbus_comm_pem3.oem3 (.const:.string)
                  0020bac3    00000001     --HOLE-- [fill = 0]
                  0020bac4    00000038     modbus_comm_pem3.oem3 (.const:ti_sysbios_knl_Task_Object__PARAMS__C)
                  0020bafc    00000030     modbus_comm_pem3.oem3 (.const:ti_sysbios_knl_Task_hooks__A)
                  0020bb2c    00000030     modbus_comm_pem3.oem3 (.const:ti_uia_runtime_LoggerStopMode_Object__PARAMS__C)
                  0020bb5c    0000002c     modbus_comm_pem3.oem3 (.const:xdc_runtime_Startup_sfxnTab__A)
                  0020bb88    00000028     TMDXDOCKH52C1.obj (.const:sdspiHWAttrs)
                  0020bbb0    00000028     modbus_comm_pem3.oem3 (.const:ti_sysbios_heaps_HeapMem_Module__FXNS__C)
                  0020bbd8    00000024     TMDXDOCKH52C1.obj (.const:gpioHWAttrs)
                  0020bbfc    00000024     modbus_comm_pem3.oem3 (.const:ti_sysbios_gates_GateHwi_Module__FXNS__C)
                  0020bc20    00000024     modbus_comm_pem3.oem3 (.const:ti_sysbios_gates_GateMutex_Module__FXNS__C)
                  0020bc44    00000024     modbus_comm_pem3.oem3 (.const:ti_sysbios_knl_Clock_Object__PARAMS__C)
                  0020bc68    00000024     modbus_comm_pem3.oem3 (.const:ti_sysbios_knl_Semaphore_Object__PARAMS__C)
                  0020bc8c    00000020     driverlib.lib : interrupt.obj (.const)
                  0020bcac    00000020                   : ssi.obj (.const)
                  0020bccc    00000020     modbus_comm_pem3.oem3 (.const:ti_sysbios_gates_GateHwi_Object__DESC__C)
                  0020bcec    00000020     modbus_comm_pem3.oem3 (.const:ti_sysbios_gates_GateMutex_Object__DESC__C)
                  0020bd0c    00000020     modbus_comm_pem3.oem3 (.const:ti_sysbios_heaps_HeapMem_Object__DESC__C)
                  0020bd2c    00000020     modbus_comm_pem3.oem3 (.const:ti_sysbios_heaps_HeapMem_Object__PARAMS__C)
                  0020bd4c    00000020     modbus_comm_pem3.oem3 (.const:ti_sysbios_knl_Clock_Object__DESC__C)
                  0020bd6c    00000020     modbus_comm_pem3.oem3 (.const:ti_sysbios_knl_Queue_Object__DESC__C)
                  0020bd8c    00000020     modbus_comm_pem3.oem3 (.const:ti_sysbios_knl_Semaphore_Object__DESC__C)
                  0020bdac    00000020     modbus_comm_pem3.oem3 (.const:ti_sysbios_knl_Task_Object__DESC__C)
                  0020bdcc    00000020     modbus_comm_pem3.oem3 (.const:ti_uia_runtime_LoggerStopMode_Object__DESC__C)
                  0020bdec    00000018     modbus_comm_pem3.oem3 (.const:ti_sysbios_gates_GateHwi_Object__PARAMS__C)
                  0020be04    00000018     modbus_comm_pem3.oem3 (.const:ti_sysbios_gates_GateMutex_Object__PARAMS__C)
                  0020be1c    00000018     modbus_comm_pem3.oem3 (.const:ti_sysbios_knl_Queue_Object__PARAMS__C)
                  0020be34    00000016     modbus_comm_pem3.oem3 (.const:xdc_runtime_Startup_sfxnRts__A)
                  0020be4a    00000002     --HOLE-- [fill = 0]
                  0020be4c    00000014     modbus_comm_pem3.oem3 (.const:xdc_runtime_Startup_firstFxns__A)
                  0020be60    00000011     ti.targets.arm.rtsarm.aem3 : System.oem3 (.const)
                  0020be71    00000003     --HOLE-- [fill = 0]
                  0020be74    00000008     modbus_comm_pem3.oem3 (.const:ti_sysbios_knl_Idle_funcList__A)
                  0020be7c    00000008     modbus_comm_pem3.oem3 (.const:ti_sysbios_knl_Idle_funcList__C)
                  0020be84    00000008     modbus_comm_pem3.oem3 (.const:ti_sysbios_knl_Task_hooks__C)
                  0020be8c    00000008     modbus_comm_pem3.oem3 (.const:xdc_runtime_Startup_firstFxns__C)
                  0020be94    00000008     modbus_comm_pem3.oem3 (.const:xdc_runtime_Startup_lastFxns__C)
                  0020be9c    00000004     modbus_comm_pem3.oem3 (.const:ti_sysbios_BIOS_Module__diagsEnabled__C)
                  0020bea0    00000004     modbus_comm_pem3.oem3 (.const:ti_sysbios_BIOS_Module__diagsIncluded__C)
                  0020bea4    00000004     modbus_comm_pem3.oem3 (.const:ti_sysbios_BIOS_Module__diagsMask__C)
                  0020bea8    00000004     modbus_comm_pem3.oem3 (.const:ti_sysbios_BIOS_installedErrorHook__C)
                  0020beac    00000004     modbus_comm_pem3.oem3 (.const:ti_sysbios_family_arm_lm3_Timer_WRALLOW__C)
                  0020beb0    00000004     modbus_comm_pem3.oem3 (.const:ti_sysbios_family_arm_lm3_Timer_numTimerDevices__C)
                  0020beb4    00000004     modbus_comm_pem3.oem3 (.const:ti_sysbios_family_arm_lm3_Timer_startupNeeded__C)
                  0020beb8    00000004     modbus_comm_pem3.oem3 (.const:ti_sysbios_family_arm_m3_Hwi_E_NMI__C)
                  0020bebc    00000004     modbus_comm_pem3.oem3 (.const:ti_sysbios_family_arm_m3_Hwi_E_busFault__C)
                  0020bec0    00000004     modbus_comm_pem3.oem3 (.const:ti_sysbios_family_arm_m3_Hwi_E_debugMon__C)
                  0020bec4    00000004     modbus_comm_pem3.oem3 (.const:ti_sysbios_family_arm_m3_Hwi_E_hardFault__C)
                  0020bec8    00000004     modbus_comm_pem3.oem3 (.const:ti_sysbios_family_arm_m3_Hwi_E_memFault__C)
                  0020becc    00000004     modbus_comm_pem3.oem3 (.const:ti_sysbios_family_arm_m3_Hwi_E_noIsr__C)
                  0020bed0    00000004     modbus_comm_pem3.oem3 (.const:ti_sysbios_family_arm_m3_Hwi_E_reserved__C)
                  0020bed4    00000004     modbus_comm_pem3.oem3 (.const:ti_sysbios_family_arm_m3_Hwi_E_svCall__C)
                  0020bed8    00000004     modbus_comm_pem3.oem3 (.const:ti_sysbios_family_arm_m3_Hwi_E_usageFault__C)
                  0020bedc    00000004     modbus_comm_pem3.oem3 (.const:ti_sysbios_family_arm_m3_Hwi_LD_end__C)
                  0020bee0    00000004     modbus_comm_pem3.oem3 (.const:ti_sysbios_family_arm_m3_Hwi_LM_begin__C)
                  0020bee4    00000004     modbus_comm_pem3.oem3 (.const:ti_sysbios_family_arm_m3_Hwi_Module__diagsEnabled__C)
                  0020bee8    00000004     modbus_comm_pem3.oem3 (.const:ti_sysbios_family_arm_m3_Hwi_Module__diagsIncluded__C)
                  0020beec    00000004     modbus_comm_pem3.oem3 (.const:ti_sysbios_family_arm_m3_Hwi_Module__diagsMask__C)
                  0020bef0    00000004     modbus_comm_pem3.oem3 (.const:ti_sysbios_family_arm_m3_Hwi_Module__loggerFxn1__C)
                  0020bef4    00000004     modbus_comm_pem3.oem3 (.const:ti_sysbios_family_arm_m3_Hwi_Module__loggerFxn8__C)
                  0020bef8    00000004     modbus_comm_pem3.oem3 (.const:ti_sysbios_family_arm_m3_Hwi_Module__loggerObj__C)
                  0020befc    00000004     modbus_comm_pem3.oem3 (.const:ti_sysbios_family_arm_m3_Hwi_NUM_INTERRUPTS__C)
                  0020bf00    00000004     modbus_comm_pem3.oem3 (.const:ti_sysbios_family_arm_m3_Hwi_ccr__C)
                  0020bf04    00000004     modbus_comm_pem3.oem3 (.const:ti_sysbios_family_arm_m3_Hwi_disablePriority__C)
                  0020bf08    00000004     modbus_comm_pem3.oem3 (.const:ti_sysbios_family_arm_m3_Hwi_excHandlerFunc__C)
                  0020bf0c    00000004     modbus_comm_pem3.oem3 (.const:ti_sysbios_family_arm_m3_Hwi_excHookFunc__C)
                  0020bf10    00000004     modbus_comm_pem3.oem3 (.const:ti_sysbios_family_arm_m3_Hwi_priGroup__C)
                  0020bf14    00000004     modbus_comm_pem3.oem3 (.const:ti_sysbios_family_arm_m3_TaskSupport_stackAlignment__C)
                  0020bf18    00000004     modbus_comm_pem3.oem3 (.const:ti_sysbios_gates_GateMutex_A_badContext__C)
                  0020bf1c    00000004     modbus_comm_pem3.oem3 (.const:ti_sysbios_gates_GateMutex_Instance_State_sem__O)
                  0020bf20    00000004     modbus_comm_pem3.oem3 (.const:ti_sysbios_gates_GateMutex_Module__diagsEnabled__C)
                  0020bf24    00000004     modbus_comm_pem3.oem3 (.const:ti_sysbios_gates_GateMutex_Module__diagsIncluded__C)
                  0020bf28    00000004     modbus_comm_pem3.oem3 (.const:ti_sysbios_gates_GateMutex_Module__diagsMask__C)
                  0020bf2c    00000004     modbus_comm_pem3.oem3 (.const:ti_sysbios_hal_Hwi_E_stackOverflow__C)
                  0020bf30    00000004     modbus_comm_pem3.oem3 (.const:ti_sysbios_heaps_HeapMem_A_align__C)
                  0020bf34    00000004     modbus_comm_pem3.oem3 (.const:ti_sysbios_heaps_HeapMem_A_heapSize__C)
                  0020bf38    00000004     modbus_comm_pem3.oem3 (.const:ti_sysbios_heaps_HeapMem_A_invalidFree__C)
                  0020bf3c    00000004     modbus_comm_pem3.oem3 (.const:ti_sysbios_heaps_HeapMem_A_zeroBlock__C)
                  0020bf40    00000004     modbus_comm_pem3.oem3 (.const:ti_sysbios_heaps_HeapMem_E_memory__C)
                  0020bf44    00000004     modbus_comm_pem3.oem3 (.const:ti_sysbios_heaps_HeapMem_Module__diagsEnabled__C)
                  0020bf48    00000004     modbus_comm_pem3.oem3 (.const:ti_sysbios_heaps_HeapMem_Module__diagsIncluded__C)
                  0020bf4c    00000004     modbus_comm_pem3.oem3 (.const:ti_sysbios_heaps_HeapMem_Module__diagsMask__C)
                  0020bf50    00000004     modbus_comm_pem3.oem3 (.const:ti_sysbios_heaps_HeapMem_Module__gateObj__C)
                  0020bf54    00000004     modbus_comm_pem3.oem3 (.const:ti_sysbios_heaps_HeapMem_Object__count__C)
                  0020bf58    00000004     modbus_comm_pem3.oem3 (.const:ti_sysbios_heaps_HeapMem_reqAlignMask__C)
                  0020bf5c    00000004     modbus_comm_pem3.oem3 (.const:ti_sysbios_heaps_HeapMem_reqAlign__C)
                  0020bf60    00000004     modbus_comm_pem3.oem3 (.const:ti_sysbios_knl_Clock_A_badThreadType__C)
                  0020bf64    00000004     modbus_comm_pem3.oem3 (.const:ti_sysbios_knl_Clock_LM_begin__C)
                  0020bf68    00000004     modbus_comm_pem3.oem3 (.const:ti_sysbios_knl_Clock_LM_tick__C)
                  0020bf6c    00000004     modbus_comm_pem3.oem3 (.const:ti_sysbios_knl_Clock_LW_delayed__C)
                  0020bf70    00000004     modbus_comm_pem3.oem3 (.const:ti_sysbios_knl_Clock_Module_State_clockQ__O)
                  0020bf74    00000004     modbus_comm_pem3.oem3 (.const:ti_sysbios_knl_Clock_Module__diagsEnabled__C)
                  0020bf78    00000004     modbus_comm_pem3.oem3 (.const:ti_sysbios_knl_Clock_Module__diagsIncluded__C)
                  0020bf7c    00000004     modbus_comm_pem3.oem3 (.const:ti_sysbios_knl_Clock_Module__diagsMask__C)
                  0020bf80    00000004     modbus_comm_pem3.oem3 (.const:ti_sysbios_knl_Clock_Module__loggerFxn1__C)
                  0020bf84    00000004     modbus_comm_pem3.oem3 (.const:ti_sysbios_knl_Clock_Module__loggerFxn2__C)
                  0020bf88    00000004     modbus_comm_pem3.oem3 (.const:ti_sysbios_knl_Clock_Module__loggerObj__C)
                  0020bf8c    00000004     modbus_comm_pem3.oem3 (.const:ti_sysbios_knl_Semaphore_A_badContext__C)
                  0020bf90    00000004     modbus_comm_pem3.oem3 (.const:ti_sysbios_knl_Semaphore_A_noEvents__C)
                  0020bf94    00000004     modbus_comm_pem3.oem3 (.const:ti_sysbios_knl_Semaphore_Instance_State_pendQ__O)
                  0020bf98    00000004     modbus_comm_pem3.oem3 (.const:ti_sysbios_knl_Semaphore_LM_pend__C)
                  0020bf9c    00000004     modbus_comm_pem3.oem3 (.const:ti_sysbios_knl_Semaphore_LM_post__C)
                  0020bfa0    00000004     modbus_comm_pem3.oem3 (.const:ti_sysbios_knl_Semaphore_Module__diagsEnabled__C)
                  0020bfa4    00000004     modbus_comm_pem3.oem3 (.const:ti_sysbios_knl_Semaphore_Module__diagsIncluded__C)
                  0020bfa8    00000004     modbus_comm_pem3.oem3 (.const:ti_sysbios_knl_Semaphore_Module__diagsMask__C)
                  0020bfac    00000004     modbus_comm_pem3.oem3 (.const:ti_sysbios_knl_Semaphore_Module__loggerFxn2__C)
                  0020bfb0    00000004     modbus_comm_pem3.oem3 (.const:ti_sysbios_knl_Semaphore_Module__loggerFxn4__C)
                  0020bfb4    00000004     modbus_comm_pem3.oem3 (.const:ti_sysbios_knl_Semaphore_Module__loggerObj__C)
                  0020bfb8    00000004     modbus_comm_pem3.oem3 (.const:ti_sysbios_knl_Swi_LD_end__C)
                  0020bfbc    00000004     modbus_comm_pem3.oem3 (.const:ti_sysbios_knl_Swi_LM_begin__C)
                  0020bfc0    00000004     modbus_comm_pem3.oem3 (.const:ti_sysbios_knl_Swi_LM_post__C)
                  0020bfc4    00000004     modbus_comm_pem3.oem3 (.const:ti_sysbios_knl_Swi_Module__diagsEnabled__C)
                  0020bfc8    00000004     modbus_comm_pem3.oem3 (.const:ti_sysbios_knl_Swi_Module__diagsIncluded__C)
                  0020bfcc    00000004     modbus_comm_pem3.oem3 (.const:ti_sysbios_knl_Swi_Module__diagsMask__C)
                  0020bfd0    00000004     modbus_comm_pem3.oem3 (.const:ti_sysbios_knl_Swi_Module__loggerFxn1__C)
                  0020bfd4    00000004     modbus_comm_pem3.oem3 (.const:ti_sysbios_knl_Swi_Module__loggerFxn4__C)
                  0020bfd8    00000004     modbus_comm_pem3.oem3 (.const:ti_sysbios_knl_Swi_Module__loggerObj__C)
                  0020bfdc    00000004     modbus_comm_pem3.oem3 (.const:ti_sysbios_knl_Swi_Object__count__C)
                  0020bfe0    00000004     modbus_comm_pem3.oem3 (.const:ti_sysbios_knl_Task_A_badPriority__C)
                  0020bfe4    00000004     modbus_comm_pem3.oem3 (.const:ti_sysbios_knl_Task_A_badTaskState__C)
                  0020bfe8    00000004     modbus_comm_pem3.oem3 (.const:ti_sysbios_knl_Task_A_badThreadType__C)
                  0020bfec    00000004     modbus_comm_pem3.oem3 (.const:ti_sysbios_knl_Task_A_noPendElem__C)
                  0020bff0    00000004     modbus_comm_pem3.oem3 (.const:ti_sysbios_knl_Task_E_spOutOfBounds__C)
                  0020bff4    00000004     modbus_comm_pem3.oem3 (.const:ti_sysbios_knl_Task_E_stackOverflow__C)
                  0020bff8    00000004     modbus_comm_pem3.oem3 (.const:ti_sysbios_knl_Task_LD_block__C)
                  0020bffc    00000004     modbus_comm_pem3.oem3 (.const:ti_sysbios_knl_Task_LD_exit__C)
                  0020c000    00000004     modbus_comm_pem3.oem3 (.const:ti_sysbios_knl_Task_LD_ready__C)
                  0020c004    00000004     modbus_comm_pem3.oem3 (.const:ti_sysbios_knl_Task_LM_switch__C)
                  0020c008    00000004     modbus_comm_pem3.oem3 (.const:ti_sysbios_knl_Task_Module_State_inactiveQ__O)
                  0020c00c    00000004     modbus_comm_pem3.oem3 (.const:ti_sysbios_knl_Task_Module_State_terminatedQ__O)
                  0020c010    00000004     modbus_comm_pem3.oem3 (.const:ti_sysbios_knl_Task_Module__diagsEnabled__C)
                  0020c014    00000004     modbus_comm_pem3.oem3 (.const:ti_sysbios_knl_Task_Module__diagsIncluded__C)
                  0020c018    00000004     modbus_comm_pem3.oem3 (.const:ti_sysbios_knl_Task_Module__diagsMask__C)
                  0020c01c    00000004     modbus_comm_pem3.oem3 (.const:ti_sysbios_knl_Task_Module__loggerFxn2__C)
                  0020c020    00000004     modbus_comm_pem3.oem3 (.const:ti_sysbios_knl_Task_Module__loggerFxn4__C)
                  0020c024    00000004     modbus_comm_pem3.oem3 (.const:ti_sysbios_knl_Task_Module__loggerObj__C)
                  0020c028    00000004     modbus_comm_pem3.oem3 (.const:ti_sysbios_knl_Task_Object__count__C)
                  0020c02c    00000004     modbus_comm_pem3.oem3 (.const:ti_sysbios_knl_Task_Object__heap__C)
                  0020c030    00000004     modbus_comm_pem3.oem3 (.const:ti_sysbios_knl_Task_allBlockedFunc__C)
                  0020c034    00000004     modbus_comm_pem3.oem3 (.const:ti_sysbios_knl_Task_defaultStackHeap__C)
                  0020c038    00000004     modbus_comm_pem3.oem3 (.const:ti_sysbios_knl_Task_defaultStackSize__C)
                  0020c03c    00000004     modbus_comm_pem3.oem3 (.const:ti_sysbios_knl_Task_numConstructedTasks__C)
                  0020c040    00000004     modbus_comm_pem3.oem3 (.const:ti_sysbios_knl_Task_numPriorities__C)
                  0020c044    00000004     modbus_comm_pem3.oem3 (.const:ti_sysbios_utils_Load_LS_cpuLoad__C)
                  0020c048    00000004     modbus_comm_pem3.oem3 (.const:ti_sysbios_utils_Load_LS_hwiLoad__C)
                  0020c04c    00000004     modbus_comm_pem3.oem3 (.const:ti_sysbios_utils_Load_LS_swiLoad__C)
                  0020c050    00000004     modbus_comm_pem3.oem3 (.const:ti_sysbios_utils_Load_LS_taskLoad__C)
                  0020c054    00000004     modbus_comm_pem3.oem3 (.const:ti_sysbios_utils_Load_Module_State_gate__O)
                  0020c058    00000004     modbus_comm_pem3.oem3 (.const:ti_sysbios_utils_Load_Module_State_taskList__O)
                  0020c05c    00000004     modbus_comm_pem3.oem3 (.const:ti_sysbios_utils_Load_Module__diagsEnabled__C)
                  0020c060    00000004     modbus_comm_pem3.oem3 (.const:ti_sysbios_utils_Load_Module__diagsIncluded__C)
                  0020c064    00000004     modbus_comm_pem3.oem3 (.const:ti_sysbios_utils_Load_Module__diagsMask__C)
                  0020c068    00000004     modbus_comm_pem3.oem3 (.const:ti_sysbios_utils_Load_Module__loggerFxn1__C)
                  0020c06c    00000004     modbus_comm_pem3.oem3 (.const:ti_sysbios_utils_Load_Module__loggerFxn2__C)
                  0020c070    00000004     modbus_comm_pem3.oem3 (.const:ti_sysbios_utils_Load_Module__loggerFxn4__C)
                  0020c074    00000004     modbus_comm_pem3.oem3 (.const:ti_sysbios_utils_Load_Module__loggerObj__C)
                  0020c078    00000004     modbus_comm_pem3.oem3 (.const:ti_sysbios_utils_Load_postUpdate__C)
                  0020c07c    00000004     modbus_comm_pem3.oem3 (.const:ti_sysbios_utils_Load_windowInMs__C)
                  0020c080    00000004     modbus_comm_pem3.oem3 (.const:ti_uia_runtime_ILoggerSnapshot_Interface__BASE__C)
                  0020c084    00000004     modbus_comm_pem3.oem3 (.const:ti_uia_runtime_IUIATransfer_Interface__BASE__C)
                  0020c088    00000004     modbus_comm_pem3.oem3 (.const:ti_uia_runtime_LoggerStopMode_E_badLevel__C)
                  0020c08c    00000004     modbus_comm_pem3.oem3 (.const:ti_uia_runtime_LoggerStopMode_Object__count__C)
                  0020c090    00000004     modbus_comm_pem3.oem3 (.const:ti_uia_runtime_LoggerStopMode_overflowLogger__C)
                  0020c094    00000004     modbus_comm_pem3.oem3 (.const:ti_uia_runtime_LoggerStopMode_statusLogger__C)
                  0020c098    00000004     modbus_comm_pem3.oem3 (.const:xdc_runtime_Assert_E_assertFailed__C)
                  0020c09c    00000004     modbus_comm_pem3.oem3 (.const:xdc_runtime_Core_A_initializedParams__C)
                  0020c0a0    00000004     modbus_comm_pem3.oem3 (.const:xdc_runtime_Core_Module__diagsEnabled__C)
                  0020c0a4    00000004     modbus_comm_pem3.oem3 (.const:xdc_runtime_Core_Module__diagsIncluded__C)
                  0020c0a8    00000004     modbus_comm_pem3.oem3 (.const:xdc_runtime_Core_Module__diagsMask__C)
                  0020c0ac    00000004     modbus_comm_pem3.oem3 (.const:xdc_runtime_Error_E_generic__C)
                  0020c0b0    00000004     modbus_comm_pem3.oem3 (.const:xdc_runtime_Error_E_memory__C)
                  0020c0b4    00000004     modbus_comm_pem3.oem3 (.const:xdc_runtime_Error_Module__diagsEnabled__C)
                  0020c0b8    00000004     modbus_comm_pem3.oem3 (.const:xdc_runtime_Error_Module__diagsIncluded__C)
                  0020c0bc    00000004     modbus_comm_pem3.oem3 (.const:xdc_runtime_Error_Module__diagsMask__C)
                  0020c0c0    00000004     modbus_comm_pem3.oem3 (.const:xdc_runtime_Error_Module__loggerFxn8__C)
                  0020c0c4    00000004     modbus_comm_pem3.oem3 (.const:xdc_runtime_Error_Module__loggerObj__C)
                  0020c0c8    00000004     modbus_comm_pem3.oem3 (.const:xdc_runtime_Error_raiseHook__C)
                  0020c0cc    00000004     modbus_comm_pem3.oem3 (.const:xdc_runtime_IFilterLogger_Interface__BASE__C)
                  0020c0d0    00000004     modbus_comm_pem3.oem3 (.const:xdc_runtime_IGateProvider_Interface__BASE__C)
                  0020c0d4    00000004     modbus_comm_pem3.oem3 (.const:xdc_runtime_IHeap_Interface__BASE__C)
                  0020c0d8    00000004     modbus_comm_pem3.oem3 (.const:xdc_runtime_ILogger_Interface__BASE__C)
                  0020c0dc    00000004     modbus_comm_pem3.oem3 (.const:xdc_runtime_IModule_Interface__BASE__C)
                  0020c0e0    00000004     modbus_comm_pem3.oem3 (.const:xdc_runtime_Log_L_error__C)
                  0020c0e4    00000004     modbus_comm_pem3.oem3 (.const:xdc_runtime_Main_Module__diagsEnabled__C)
                  0020c0e8    00000004     modbus_comm_pem3.oem3 (.const:xdc_runtime_Main_Module__diagsIncluded__C)
                  0020c0ec    00000004     modbus_comm_pem3.oem3 (.const:xdc_runtime_Main_Module__diagsMask__C)
                  0020c0f0    00000004     modbus_comm_pem3.oem3 (.const:xdc_runtime_Main_Module__loggerFxn4__C)
                  0020c0f4    00000004     modbus_comm_pem3.oem3 (.const:xdc_runtime_Main_Module__loggerObj__C)
                  0020c0f8    00000004     modbus_comm_pem3.oem3 (.const:xdc_runtime_Memory_defaultHeapInstance__C)
                  0020c0fc    00000004     modbus_comm_pem3.oem3 (.const:xdc_runtime_Startup_execImpl__C)
                  0020c100    00000004     modbus_comm_pem3.oem3 (.const:xdc_runtime_Startup_lastFxns__A)
                  0020c104    00000004     modbus_comm_pem3.oem3 (.const:xdc_runtime_Startup_maxPasses__C)
                  0020c108    00000004     modbus_comm_pem3.oem3 (.const:xdc_runtime_Startup_sfxnRts__C)
                  0020c10c    00000004     modbus_comm_pem3.oem3 (.const:xdc_runtime_Startup_sfxnTab__C)
                  0020c110    00000004     modbus_comm_pem3.oem3 (.const:xdc_runtime_SysMin_bufSize__C)
                  0020c114    00000004     modbus_comm_pem3.oem3 (.const:xdc_runtime_SysMin_outputFunc__C)
                  0020c118    00000004     modbus_comm_pem3.oem3 (.const:xdc_runtime_System_Module__gateObj__C)
                  0020c11c    00000004     modbus_comm_pem3.oem3 (.const:xdc_runtime_System_extendFxn__C)
                  0020c120    00000004     modbus_comm_pem3.oem3 (.const:xdc_runtime_System_maxAtexitHandlers__C)
                  0020c124    00000004     modbus_comm_pem3.oem3 (.const:xdc_runtime_Text_charTab__C)
                  0020c128    00000004     modbus_comm_pem3.oem3 (.const:xdc_runtime_Text_nameEmpty__C)
                  0020c12c    00000004     modbus_comm_pem3.oem3 (.const:xdc_runtime_Text_nameStatic__C)
                  0020c130    00000004     modbus_comm_pem3.oem3 (.const:xdc_runtime_Text_nameUnknown__C)
                  0020c134    00000004     modbus_comm_pem3.oem3 (.const:xdc_runtime_Text_nodeTab__C)
                  0020c138    00000004     modbus_comm_pem3.oem3 (.const:xdc_runtime_Text_visitRopeFxn__C)
                  0020c13c    00000002     modbus_comm_pem3.oem3 (.const:ti_sysbios_BIOS_Module__id__C)
                  0020c13e    00000002     --HOLE-- [fill = 0]
                  0020c140    00000002     modbus_comm_pem3.oem3 (.const:ti_sysbios_family_arm_m3_Hwi_Module__id__C)
                  0020c142    00000002     --HOLE-- [fill = 0]
                  0020c144    00000002     modbus_comm_pem3.oem3 (.const:ti_sysbios_family_arm_m3_Hwi_Module__loggerDefined__C)
                  0020c146    00000002     --HOLE-- [fill = 0]
                  0020c148    00000002     modbus_comm_pem3.oem3 (.const:ti_sysbios_gates_GateMutex_Module__id__C)
                  0020c14a    00000002     --HOLE-- [fill = 0]
                  0020c14c    00000002     modbus_comm_pem3.oem3 (.const:ti_sysbios_hal_Hwi_Module__id__C)
                  0020c14e    00000002     --HOLE-- [fill = 0]
                  0020c150    00000002     modbus_comm_pem3.oem3 (.const:ti_sysbios_heaps_HeapMem_Module__id__C)
                  0020c152    00000002     --HOLE-- [fill = 0]
                  0020c154    00000002     modbus_comm_pem3.oem3 (.const:ti_sysbios_knl_Clock_Module__id__C)
                  0020c156    00000002     --HOLE-- [fill = 0]
                  0020c158    00000002     modbus_comm_pem3.oem3 (.const:ti_sysbios_knl_Clock_Module__loggerDefined__C)
                  0020c15a    00000002     --HOLE-- [fill = 0]
                  0020c15c    00000002     modbus_comm_pem3.oem3 (.const:ti_sysbios_knl_Semaphore_Module__id__C)
                  0020c15e    00000002     --HOLE-- [fill = 0]
                  0020c160    00000002     modbus_comm_pem3.oem3 (.const:ti_sysbios_knl_Semaphore_Module__loggerDefined__C)
                  0020c162    00000002     --HOLE-- [fill = 0]
                  0020c164    00000002     modbus_comm_pem3.oem3 (.const:ti_sysbios_knl_Swi_Module__id__C)
                  0020c166    00000002     --HOLE-- [fill = 0]
                  0020c168    00000002     modbus_comm_pem3.oem3 (.const:ti_sysbios_knl_Swi_Module__loggerDefined__C)
                  0020c16a    00000002     --HOLE-- [fill = 0]
                  0020c16c    00000002     modbus_comm_pem3.oem3 (.const:ti_sysbios_knl_Task_Module__id__C)
                  0020c16e    00000002     --HOLE-- [fill = 0]
                  0020c170    00000002     modbus_comm_pem3.oem3 (.const:ti_sysbios_knl_Task_Module__loggerDefined__C)
                  0020c172    00000002     --HOLE-- [fill = 0]
                  0020c174    00000002     modbus_comm_pem3.oem3 (.const:ti_sysbios_knl_Task_deleteTerminatedTasks__C)
                  0020c176    00000002     --HOLE-- [fill = 0]
                  0020c178    00000002     modbus_comm_pem3.oem3 (.const:ti_sysbios_knl_Task_initStackFlag__C)
                  0020c17a    00000002     --HOLE-- [fill = 0]
                  0020c17c    00000002     modbus_comm_pem3.oem3 (.const:ti_sysbios_utils_Load_Module__id__C)
                  0020c17e    00000002     --HOLE-- [fill = 0]
                  0020c180    00000002     modbus_comm_pem3.oem3 (.const:ti_sysbios_utils_Load_Module__loggerDefined__C)
                  0020c182    00000002     --HOLE-- [fill = 0]
                  0020c184    00000002     modbus_comm_pem3.oem3 (.const:ti_sysbios_utils_Load_autoAddTasks__C)
                  0020c186    00000002     --HOLE-- [fill = 0]
                  0020c188    00000002     modbus_comm_pem3.oem3 (.const:ti_sysbios_utils_Load_hwiEnabled__C)
                  0020c18a    00000002     --HOLE-- [fill = 0]
                  0020c18c    00000002     modbus_comm_pem3.oem3 (.const:ti_sysbios_utils_Load_swiEnabled__C)
                  0020c18e    00000002     --HOLE-- [fill = 0]
                  0020c190    00000002     modbus_comm_pem3.oem3 (.const:ti_sysbios_utils_Load_taskEnabled__C)
                  0020c192    00000002     --HOLE-- [fill = 0]
                  0020c194    00000002     modbus_comm_pem3.oem3 (.const:ti_sysbios_utils_Load_updateInIdle__C)
                  0020c196    00000002     --HOLE-- [fill = 0]
                  0020c198    00000002     modbus_comm_pem3.oem3 (.const:ti_uia_runtime_LoggerStopMode_Module__id__C)
                  0020c19a    00000002     --HOLE-- [fill = 0]
                  0020c19c    00000002     modbus_comm_pem3.oem3 (.const:ti_uia_runtime_LoggerStopMode_filterByLevel__C)
                  0020c19e    00000002     --HOLE-- [fill = 0]
                  0020c1a0    00000002     modbus_comm_pem3.oem3 (.const:ti_uia_runtime_LoggerStopMode_isTimestampEnabled__C)
                  0020c1a2    00000002     --HOLE-- [fill = 0]
                  0020c1a4    00000002     modbus_comm_pem3.oem3 (.const:xdc_runtime_Core_Module__id__C)
                  0020c1a6    00000002     --HOLE-- [fill = 0]
                  0020c1a8    00000002     modbus_comm_pem3.oem3 (.const:xdc_runtime_Error_Module__loggerDefined__C)
                  0020c1aa    00000002     --HOLE-- [fill = 0]
                  0020c1ac    00000002     modbus_comm_pem3.oem3 (.const:xdc_runtime_Error_maxDepth__C)
                  0020c1ae    00000002     --HOLE-- [fill = 0]
                  0020c1b0    00000002     modbus_comm_pem3.oem3 (.const:xdc_runtime_Main_Module__id__C)
                  0020c1b2    00000002     --HOLE-- [fill = 0]
                  0020c1b4    00000002     modbus_comm_pem3.oem3 (.const:xdc_runtime_Main_Module__loggerDefined__C)
                  0020c1b6    00000002     --HOLE-- [fill = 0]
                  0020c1b8    00000002     modbus_comm_pem3.oem3 (.const:xdc_runtime_Memory_Module__id__C)
                  0020c1ba    00000002     --HOLE-- [fill = 0]
                  0020c1bc    00000002     modbus_comm_pem3.oem3 (.const:xdc_runtime_SysMin_flushAtExit__C)
                  0020c1be    00000002     --HOLE-- [fill = 0]
                  0020c1c0    00000002     modbus_comm_pem3.oem3 (.const:xdc_runtime_Text_charCnt__C)
                  0020c1c2    00000002     --HOLE-- [fill = 0]
                  0020c1c4    00000002     modbus_comm_pem3.oem3 (.const:xdc_runtime_Text_isLoaded__C)
                  0020c1c6    00000002     --HOLE-- [fill = 0]
                  0020c1c8    00000002     modbus_comm_pem3.oem3 (.const:xdc_runtime_Text_registryModsLastId__C)
                  0020c1ca    00000002     --HOLE-- [fill = 0]
                  0020c1cc    00000002     modbus_comm_pem3.oem3 (.const:xdc_runtime_Text_unnamedModsLastId__C)
                  0020c1ce    00000002     --HOLE-- [fill = 0]
                  0020c1d0    00000001     modbus_comm_pem3.oem3 (.const:ti_sysbios_knl_Clock_tickMode__C)
                  0020c1d1    00000003     --HOLE-- [fill = 0]
                  0020c1d4    00000001     modbus_comm_pem3.oem3 (.const:ti_sysbios_knl_Clock_tickSource__C)
                  0020c1d5    00000003     --HOLE-- [fill = 0]
                  0020c1d8    00000001     modbus_comm_pem3.oem3 (.const:xdc_runtime_Error_policy__C)

.flashfuncs 
*          0    0020c1dc    0000003c     RUN ADDR = 200001ac
                  0020c1dc    0000003c     Boot.aem3 : Boot.oem3 (.flashfuncs)

.cinit     0    0020c218    000004f0     
                  0020c218    000004b8     (.cinit..data.load) [load image, compression = rle]
                  0020c6d0    0000000c     (__TI_handler_table)
                  0020c6dc    00000004     --HOLE-- [fill = 0]
                  0020c6e0    00000008     (.cinit..bss.load) [load image, compression = zero_init]
                  0020c6e8    00000008     (.cinit..vecs.load) [load image, compression = zero_init]
                  0020c6f0    00000018     (__TI_cinit_table)

.binit     0    0020c708    00000010     
                  0020c708    00000010     (.binit)

.vecs      0    20000000    000001ac     UNINITIALIZED
                  20000000    000001ac     modbus_comm_pem3.oem3 (.vecs)

.bss       0    200001e8    00002b10     UNINITIALIZED
                  200001e8    00001000     modbus_comm_pem3.oem3 (.bss:ti_sysbios_heaps_HeapMem_Instance_State_0_buf__A)
                  200011e8    00000800     modbus_comm_pem3.oem3 (.bss:taskStackSection)
                  200019e8    00000480     modbus_comm_pem3.oem3 (.bss:ti_uia_runtime_LoggerStopMode_Instance_State_1_bufferArray__A)
                  20001e68    00000480     modbus_comm_pem3.oem3 (.bss:ti_uia_runtime_LoggerStopMode_Instance_State_2_bufferArray__A)
                  200022e8    00000400     modbus_comm_pem3.oem3 (.bss:xdc_runtime_SysMin_Module_State_0_outbuf__A)
                  200026e8    00000280     modbus_comm_pem3.oem3 (.bss:ti_uia_runtime_LoggerStopMode_Instance_State_0_bufferArray__A)
                  20002968    00000120     rtsv7M3_T_le_eabi.lib : trgmsg.obj (.bss:__CIOBUF_)
                  20002a88    000000c8                           : trgdrv.obj (.bss:result$1)
                  20002b50    00000070     TMDXDOCKH52C1.obj (.bss:I2CObjects)
                  20002bc0    0000004c     TMDXDOCKH52C1.obj (.bss:uartObjects)
                  20002c0c    00000038     modbus_main.obj (.bss:taskParams)
                  20002c44    00000033     modbus_main.obj (.bss)
                  20002c77    00000001     --HOLE--
                  20002c78    00000030     modbus_main.obj (.bss:eb)
                  20002ca8    00000028     ti.sysbios.fatfs.aem3 : ffcio.oem3 (.bss:filTable)
                  20002cd0    00000018     TMDXDOCKH52C1.obj (.bss)
                  20002ce8    00000008     modbus_comm_pem3.oem3 (.bss)
                  20002cf0    00000008     rtsv7M3_T_le_eabi.lib : trgdrv.obj (.bss)

.stack     0    20008000    00001000     UNINITIALIZED
                  20008000    00001000     --HOLE--

.data      0    20009000    00000956     
                  20009000    000001ac     modbus_comm_pem3.oem3 (.data)
                  200091ac    000001ac     modbus_comm_pem3.oem3 (.data:ti_sysbios_family_arm_m3_Hwi_Module_State_0_dispatchTable__A)
                  20009358    00000108     modbus_comm_pem3.oem3 (.data:ti_uia_runtime_LoggerStopMode_Object__table__V)
                  20009460    00000098     modbus_comm_pem3.oem3 (.data:ti_sysbios_utils_Load_Module__state__V)
                  200094f8    00000080     modbus_comm_pem3.oem3 (.data:ti_sysbios_knl_Swi_Module_State_0_readyQ__A)
                  20009578    00000080     modbus_comm_pem3.oem3 (.data:ti_sysbios_knl_Task_Module_State_0_readyQ__A)
                  200095f8    00000078     rtsv7M3_T_le_eabi.lib : lowlev.obj (.data:_device)
                  20009670    0000006b     modbus_comm_pem3.oem3 (.data:ti_sysbios_family_arm_m3_Hwi_Module_State_0_priorities__A)
                  200096db    00000001     --HOLE--
                  200096dc    00000050     rtsv7M3_T_le_eabi.lib : lowlev.obj (.data:_stream)
                  2000972c    00000050     ti.sysbios.fatfs.aem3 : diskio.oem3 (.data:drive_fxn_table)
                  2000977c    00000050     modbus_comm_pem3.oem3 (.data:ti_sysbios_family_arm_m3_Hwi_Module__state__V)
                  200097cc    00000048     modbus_comm_pem3.oem3 (.data:ti_sysbios_knl_Task_Object__table__V)
                  20009814    00000038     modbus_comm_pem3.oem3 (.data:ti_sysbios_gates_GateMutex_Object__table__V)
                  2000984c    00000034     modbus_comm_pem3.oem3 (.data:ti_sysbios_knl_Task_Module__state__V)
                  20009880    00000030     modbus_comm_pem3.oem3 (.data:ti_sysbios_family_arm_lm3_Timer_Object__table__V)
                  200098b0    00000030     modbus_comm_pem3.oem3 (.data:ti_sysbios_knl_Swi_Object__table__V)
                  200098e0    0000002c     modbus_comm_pem3.oem3 (.data:ti_sysbios_knl_Clock_Module__state__V)
                  2000990c    00000012     ti.sysbios.fatfs.aem3 : ff.oem3 (.data)
                  2000991e    00000002     --HOLE--
                  20009920    00000008     rtsv7M3_T_le_eabi.lib : _lock.obj (.data)
                  20009928    00000008                           : exit.obj (.data)
                  20009930    00000008     ti.uia.runtime.aem3 : QueueDescriptor.oem3 (.data)
                  20009938    00000006     TMDXDOCKH52C1.obj (.data)
                  2000993e    00000002     --HOLE--
                  20009940    00000004     rtsv7M3_T_le_eabi.lib : dtor_list.obj (.data)
                  20009944    00000004                           : lowlev.obj (.data)
                  20009948    00000004                           : stkdepth_vars.obj (.data)
                  2000994c    00000004     ti.sysbios.fatfs.aem3 : ffcio.oem3 (.data)
                  20009950    00000002     gpio_mware.aem3 : GPIO.oem3 (.data)
                  20009952    00000002     --HOLE--
                  20009954    00000002     uart_mware.aem3 : UART.oem3 (.data)


LINKER GENERATED COPY TABLES

__TI_cinit_table @ 0020c6f0 records: 3, size/record: 8, table size: 24
	.data: load addr=0020c218, load size=000004b8 bytes, run addr=20009000, run size=00000956 bytes, compression=rle
	.bss: load addr=0020c6e0, load size=00000008 bytes, run addr=200001e8, run size=00002b10 bytes, compression=zero_init
	.vecs: load addr=0020c6e8, load size=00000008 bytes, run addr=20000000, run size=000001ac bytes, compression=zero_init
binit @ 0020c708 records: 1, size/record: 12, table size: 16
	.flashfuncs: load addr=0020c1dc, load size=0000003c, run addr=200001ac, run size=0000003c, compression=none


LINKER GENERATED HANDLER TABLE

__TI_handler_table @ 0020c6d0 records: 3, size/record: 4, table size: 12
	index: 0, handler: __TI_zero_init
	index: 1, handler: __TI_decompress_rle24
	index: 2, handler: __TI_decompress_none


FAR CALL TRAMPOLINES

callee name               trampoline name
   callee addr  tramp addr   call addr  call info
--------------  -----------  ---------  ----------------
$.flashfuncs:D:\ti\mcusdk_1_00_00_68\products\xdctools_3_23_04_60\packages\ti\catalog\arm\cortexm3\concertoInit\lib\Boot.aem3<Boot.oem3>$0x0  $Tramp$TT$L$PI$$$.flashfuncs:D:\ti\mcusdk_1_00_00_68\products\xdctools_3_23_04_60\packages\ti\catalog\arm\cortexm3\concertoInit\lib\Boot.aem3<Boot.oem3>$0x0
   200001ad     00209a44     0020989e   modbus_comm_pem3.oem3 (.text:.bootCodeSection:ti_catalog_arm_cortexm3_concertoInit_Boot_initStartup)

[1 trampolines]
[1 trampoline calls]


GLOBAL SYMBOLS: SORTED ALPHABETICALLY BY Name 

address    name
--------   ----
00208401   C$$EXIT
00207c03   C$$IO$$
0020893d   CPUbasepriGet
00208937   CPUbasepriSet
00208911   CPUcpsid
00208927   CPUcpsie
0020891d   CPUprimask
00208933   CPUwfi
0020b8f4   EMAC_config
00200c2f   GPIODirModeGet
00200bff   GPIODirModeSet
00200c9f   GPIOIntTypeGet
00200c59   GPIOIntTypeSet
00200d33   GPIOPadConfigGet
00200cd9   GPIOPadConfigSet
00200ec1   GPIOPinConfigure
00200f2b   GPIOPinConfigureCoreSelect
00200d97   GPIOPinIntClear
00200d7b   GPIOPinIntDisable
00200d6f   GPIOPinIntEnable
00200d89   GPIOPinIntStatus
00200f55   GPIOPinLock
00200f4b   GPIOPinLockStatus
00200dc9   GPIOPinRead
00200dd5   GPIOPinTypeCAN
00200ead   GPIOPinTypeEPI
00200de9   GPIOPinTypeGPIOInput
00200dfd   GPIOPinTypeGPIOOutput
00200e19   GPIOPinTypeGPIOOutputOD
00200e2d   GPIOPinTypeI2C
00200e45   GPIOPinTypeSSI
00200e5d   GPIOPinTypeTimer
00200e71   GPIOPinTypeUART
00200e99   GPIOPinTypeUSBAnalog
00200e85   GPIOPinTypeUSBDigital
00200f7b   GPIOPinUnlock
00200dcf   GPIOPinWrite
00200d9d   GPIOPortIntRegister
00200db5   GPIOPortIntUnregister
0020b8d0   GPIO_config
00207b79   GPIO_init
00203a65   GPIO_write
00201f8d   HOSTclock
00201f49   HOSTclose
00201eed   HOSTlseek
00201e9d   HOSTopen
00201e4f   HOSTread
00201def   HOSTrename
00201db3   HOSTtime
00201d79   HOSTunlink
00201d2b   HOSTwrite
0020b91c   I2CHWAttrs
20002b50   I2CObjects
0020b92c   I2C_config
00202385   IntDisable
00202311   IntEnable
00202295   IntFlashVTable
0020228b   IntMasterDisable
00202281   IntMasterEnable
00202463   IntPendClear
002023fb   IntPendSet
002022f9   IntPriorityGet
002022ad   IntPriorityGroupingGet
0020229d   IntPriorityGroupingSet
0020893d   IntPriorityMaskGet
00208937   IntPriorityMaskSet
002022cd   IntPrioritySet
00202297   IntRAMVTable
00202299   IntRegister
0020229b   IntUnregister
0020b900   SDSPI_config
UNDEFED    SHT$$INIT_ARRAY$$Base
UNDEFED    SHT$$INIT_ARRAY$$Limit
00204dc9   SSIBusy
00204cdb   SSIConfigSetExpClk
00204dbf   SSIDMADisable
00204db7   SSIDMAEnable
00204d99   SSIDataGet
00204da5   SSIDataGetNonBlocking
00204d7f   SSIDataPut
00204d89   SSIDataPutNonBlocking
00204d29   SSIDisable
00204d1f   SSIEnable
00204d7b   SSIIntClear
00204d67   SSIIntDisable
00204d5f   SSIIntEnable
00204d33   SSIIntRegister
00204d71   SSIIntStatus
00204d4b   SSIIntUnregister
20002c48   Sem
002008c3   SysCtlC28Disable
002008ab   SysCtlC28Enable
002007e1   SysCtlClockConfigGet
002007ad   SysCtlClockConfigSet
00200549   SysCtlClockDividersSet
00200831   SysCtlClockGet
00200681   SysCtlClockPllConfig
00200489   SysCtlDeepSleep
00209981   SysCtlDelay
00200a1b   SysCtlEnableAERRNMI
00200a35   SysCtlEnableVREGWarnNMI
0020020b   SysCtlFlashSizeGet
002008f7   SysCtlGPIOAHBDisable
002008db   SysCtlGPIOAHBEnable
00200a4d   SysCtlGetNmiConfig
00200a61   SysCtlGetNmiFlagStatus
00200a53   SysCtlGetNmiInterruptStatus
00200ab7   SysCtlHoldSubSystemInReset
00200a81   SysCtlNmiFlgClr
00200a99   SysCtlNmiFlgClrAll
00200a69   SysCtlNmiIsSet
0020044d   SysCtlPeripheralClockGating
00200421   SysCtlPeripheralDeepSleepDisable
002003f7   SysCtlPeripheralDeepSleepEnable
00200367   SysCtlPeripheralDisable
00200341   SysCtlPeripheralEnable
0020038d   SysCtlPeripheralIsEnabled
00200217   SysCtlPeripheralPresent
00200279   SysCtlPeripheralReset
002003d1   SysCtlPeripheralSleepDisable
002003ab   SysCtlPeripheralSleepEnable
0020064f   SysCtlPowerOffPLL
00200add   SysCtlReleaseSubSystemFromReset
00200475   SysCtlReset
002004b5   SysCtlResetCauseClear
002004a9   SysCtlResetCauseGet
002001ed   SysCtlSRAMSizeGet
00208933   SysCtlSleep
00200b05   SysCtlSubSystemReset
002009fd   SysCtlUSBPLLConfigGet
00200965   SysCtlUSBPLLConfigSet
00200949   SysCtlUSBPLLDisable
00200915   SysCtlUSBPLLEnable
002004d1   SysCtlXPllClockDividerSet
00208949   TMDXDOCKH52C1_initGPIO
00207115   TMDXDOCKH52C1_initGeneral
00207ec1   TMDXDOCKH52C1_initUART
200097cc   TSK_idle
20002c50   TimerHd_Counter
00202197   UARTBreakCtl
002021ab   UARTBusy
00202173   UARTCharGet
00202163   UARTCharGetNonBlocking
0020218d   UARTCharPut
0020217d   UARTCharPutNonBlocking
0020214b   UARTCharsAvail
0020204d   UARTConfigGetExpClk
00202003   UARTConfigSetExpClk
00202253   UARTDMADisable
0020224b   UARTDMAEnable
00202089   UARTDisable
002020cb   UARTDisableSIR
00202075   UARTEnable
002020b5   UARTEnableSIR
002020ab   UARTFIFODisable
002020a1   UARTFIFOEnable
00201ff3   UARTFIFOLevelGet
00201fed   UARTFIFOLevelSet
0020212f   UARTFlowControlGet
00202123   UARTFlowControlSet
00202247   UARTIntClear
00202233   UARTIntDisable
0020222b   UARTIntEnable
002021b3   UARTIntRegister
0020223d   UARTIntStatus
002021ef   UARTIntUnregister
00202101   UARTModemControlClear
00202111   UARTModemControlGet
002020f5   UARTModemControlSet
00202119   UARTModemStatusGet
00201fe5   UARTParityModeGet
00201fd9   UARTParityModeSet
00202265   UARTRxErrorClear
0020225d   UARTRxErrorGet
002020eb   UARTSmartCardDisable
002020d5   UARTSmartCardEnable
00202157   UARTSpaceAvail
00202143   UARTTxIntModeGet
00202137   UARTTxIntModeSet
0020b8e0   UART_config
0020741d   UART_init
0020b90c   USBMSCHFatFsHWAttrs
20002ce0   USBMSCHFatFsObjects
0020b910   USBMSCHFatFs_config
0020406d   UartTask
00206701   WatchdogEnable
0020677f   WatchdogIntClear
0020676b   WatchdogIntEnable
0020674b   WatchdogIntRegister
00206775   WatchdogIntStatus
0020675b   WatchdogIntUnregister
0020671f   WatchdogLock
0020672f   WatchdogLockState
00206743   WatchdogReloadGet
0020673f   WatchdogReloadSet
00206715   WatchdogResetDisable
0020670b   WatchdogResetEnable
002066f9   WatchdogRunning
00206793   WatchdogStallDisable
00206785   WatchdogStallEnable
00206727   WatchdogUnlock
00206747   WatchdogValueGet
00000000   __ASM__
20002968   __CIOBUF_
00000062   __ISA__
00000074   __PLAT__
20009000   __STACK_END
00001000   __STACK_SIZE
20008100   __STACK_TOP
0000009b   __TARG__
0020c6f0   __TI_CINIT_Base
0020c708   __TI_CINIT_Limit
0020c6d0   __TI_Handler_Table_Base
0020c6dc   __TI_Handler_Table_Limit
00000001   __TI_args_main
00206cf1   __TI_auto_init
00209845   __TI_decompress_none
0020998d   __TI_decompress_rle24
0020c708   __TI_static_base__
0020c708   __TI_table_binit
00209665   __TI_zero_init
000000c0   __TRDR__
00205dc3   __aeabi_atexit
0020750d   __aeabi_memclr
0020750d   __aeabi_memclr4
0020750d   __aeabi_memclr8
00206e31   __aeabi_memcpy
00206e31   __aeabi_memcpy4
00206e31   __aeabi_memcpy8
0020750f   __aeabi_memset
0020750f   __aeabi_memset4
0020750f   __aeabi_memset8
0020c708   __binit__
ffffffff   __c_args__
00205d6d   __cxa_atexit
00205d7f   __cxa_finalize
00205dbd   __cxa_ia64_exit
20008000   __stack
00209987   __xdc__init
200091a8   __xdc__init__addr
00209485   _args_main
00208379   _c_int00
20009928   _cleanup_ptr
2000992c   _dtors_ptr
20009920   _lock
00209479   _nop
00209473   _register_lock
0020946d   _register_unlock
00200031   _ti_catalog_arm_cortexm3_concertoInit_Boot_entry
20009924   _unlock
20002c54   a
00208405   abort
00201663   add_device
00205d71   atexit
0020c708   binit
00201615   close
00209455   clust2sect
002081c9   copy_in
00209285   disk_initialize
002092a1   disk_ioctl
002092bd   disk_read
002092d9   disk_status
002092f5   disk_write
20002c78   eb
20002c4c   echo
0020b8ec   emacHWAttrs
20002cd0   emacObjects
0020840d   exit
00209735   f_close
00203d7d   f_lseek
002041c1   f_open
002038c1   f_read
00204b8d   f_rename
00206139   f_sync
002061f7   f_unlink
00202de1   f_write
002099c7   ff_rel_grant
0020995f   ff_req_grant
00208fa1   ffcio_close
0020897d   ffcio_lseek
002067a5   ffcio_open
002090e5   ffcio_read
00209677   ffcio_rename
00209689   ffcio_unlink
00209105   ffcio_write
002015ff   find_registered_device
00209311   free
00205c9d   get_fat
00209971   get_fattime
00201ced   getenv
0020bbd8   gpioHWAttrs
20002c67   input
002015bf   lseek
20009938   macAddress
0020511d   main
20009948   main_func_sp
00208cd1   malloc
20002c66   mb_tx_data
00206e31   memcpy
00207515   memset
20002c65   n
00201537   open
20002c64   pt
00205a0d   put_fat
002014bb   read
00207c07   readmsg
00201493   remove_device
00201457   rename
0020bb88   sdspiHWAttrs
20002cd4   sdspiObjects
00209545   strchr
0020949d   strcmp
0020969b   strcpy
0020959d   strlen
00208b4f   strncpy
20002c44   tMB_State
20002c0c   taskParams
00203339   ti_catalog_arm_cortexm3_concertoInit_Boot_bootC28
0020324b   ti_catalog_arm_cortexm3_concertoInit_Boot_configurePllDivs
00203249   ti_catalog_arm_cortexm3_concertoInit_Boot_defaultLimpAbortFunction
0020988b   ti_catalog_arm_cortexm3_concertoInit_Boot_init
0020319d   ti_catalog_arm_cortexm3_concertoInit_Boot_initC28RAMs
200001ad   ti_catalog_arm_cortexm3_concertoInit_Boot_initFlash
00209897   ti_catalog_arm_cortexm3_concertoInit_Boot_initStartup
002099c3   ti_catalog_arm_cortexm3_concertoInit_Boot_limpAbort
00209979   ti_catalog_arm_cortexm3_concertoInit_Boot_stepDelay
0020be9c   ti_sysbios_BIOS_Module__diagsEnabled__C
0020bea0   ti_sysbios_BIOS_Module__diagsIncluded__C
0020bea4   ti_sysbios_BIOS_Module__diagsMask__C
0020c13c   ti_sysbios_BIOS_Module__id__C
20009000   ti_sysbios_BIOS_Module__state__V
002099cb   ti_sysbios_BIOS_RtsGateProxy_enter__E
002099cf   ti_sysbios_BIOS_RtsGateProxy_leave__E
002099df   ti_sysbios_BIOS_RtsGateProxy_query__E
00208445   ti_sysbios_BIOS_errorRaiseHook__I
00208b81   ti_sysbios_BIOS_exitFunc__I
0020bea8   ti_sysbios_BIOS_installedErrorHook__C
00208fe9   ti_sysbios_BIOS_registerRTSLock__I
00209755   ti_sysbios_BIOS_setThreadType__E
00208e8d   ti_sysbios_BIOS_startFunc__I
00209765   ti_sysbios_BIOS_start__E
40000400   ti_sysbios_family_arm_ducati_CTM_ctm
2000901c   ti_sysbios_family_arm_f28m35x_TimestampProvider_Module__state__V
002098b1   ti_sysbios_family_arm_f28m35x_TimestampProvider_get32__E
00208eb5   ti_sysbios_family_arm_f28m35x_TimestampProvider_get64__E
00209775   ti_sysbios_family_arm_f28m35x_TimestampProvider_getFreq__E
2000902c   ti_sysbios_family_arm_lm3_Timer_Module_State_0_device__A
2000904c   ti_sysbios_family_arm_lm3_Timer_Module_State_0_handles__A
20009024   ti_sysbios_family_arm_lm3_Timer_Module__root__V
002094b5   ti_sysbios_family_arm_lm3_Timer_Module__startupDone__F
002094b5   ti_sysbios_family_arm_lm3_Timer_Module__startupDone__S
2000905c   ti_sysbios_family_arm_lm3_Timer_Module__state__V
0020721d   ti_sysbios_family_arm_lm3_Timer_Module_startup__E
0020721d   ti_sysbios_family_arm_lm3_Timer_Module_startup__F
20009880   ti_sysbios_family_arm_lm3_Timer_Object__table__V
0020beac   ti_sysbios_family_arm_lm3_Timer_WRALLOW__C
00205af9   ti_sysbios_family_arm_lm3_Timer_enableTimers__I
00208bb1   ti_sysbios_family_arm_lm3_Timer_getExpiredCounts__E
002099d3   ti_sysbios_family_arm_lm3_Timer_getPeriod__E
0020900d   ti_sysbios_family_arm_lm3_Timer_isrStub__E
0020beb0   ti_sysbios_family_arm_lm3_Timer_numTimerDevices__C
00203f07   ti_sysbios_family_arm_lm3_Timer_setNextTick__E
0020beb4   ti_sysbios_family_arm_lm3_Timer_startupNeeded__C
00205ef9   ti_sysbios_family_arm_lm3_Timer_startup__E
0020beb8   ti_sysbios_family_arm_m3_Hwi_E_NMI__C
0020bebc   ti_sysbios_family_arm_m3_Hwi_E_busFault__C
0020bec0   ti_sysbios_family_arm_m3_Hwi_E_debugMon__C
0020bec4   ti_sysbios_family_arm_m3_Hwi_E_hardFault__C
0020bec8   ti_sysbios_family_arm_m3_Hwi_E_memFault__C
0020becc   ti_sysbios_family_arm_m3_Hwi_E_noIsr__C
0020bed0   ti_sysbios_family_arm_m3_Hwi_E_reserved__C
0020bed4   ti_sysbios_family_arm_m3_Hwi_E_svCall__C
0020bed8   ti_sysbios_family_arm_m3_Hwi_E_usageFault__C
0020bedc   ti_sysbios_family_arm_m3_Hwi_LD_end__C
0020bee0   ti_sysbios_family_arm_m3_Hwi_LM_begin__C
200091ac   ti_sysbios_family_arm_m3_Hwi_Module_State_0_dispatchTable__A
20009670   ti_sysbios_family_arm_m3_Hwi_Module_State_0_priorities__A
0020bee4   ti_sysbios_family_arm_m3_Hwi_Module__diagsEnabled__C
0020bee8   ti_sysbios_family_arm_m3_Hwi_Module__diagsIncluded__C
0020beec   ti_sysbios_family_arm_m3_Hwi_Module__diagsMask__C
0020c140   ti_sysbios_family_arm_m3_Hwi_Module__id__C
0020c144   ti_sysbios_family_arm_m3_Hwi_Module__loggerDefined__C
0020bef0   ti_sysbios_family_arm_m3_Hwi_Module__loggerFxn1__C
0020bef4   ti_sysbios_family_arm_m3_Hwi_Module__loggerFxn8__C
0020bef8   ti_sysbios_family_arm_m3_Hwi_Module__loggerObj__C
20009068   ti_sysbios_family_arm_m3_Hwi_Module__root__V
002094cd   ti_sysbios_family_arm_m3_Hwi_Module__startupDone__F
002094cd   ti_sysbios_family_arm_m3_Hwi_Module__startupDone__S
2000977c   ti_sysbios_family_arm_m3_Hwi_Module__state__V
00204dd5   ti_sysbios_family_arm_m3_Hwi_Module_startup__E
00204dd5   ti_sysbios_family_arm_m3_Hwi_Module_startup__F
0020befc   ti_sysbios_family_arm_m3_Hwi_NUM_INTERRUPTS__C
20009070   ti_sysbios_family_arm_m3_Hwi_Object__table__V
0020bf00   ti_sysbios_family_arm_m3_Hwi_ccr__C
00208695   ti_sysbios_family_arm_m3_Hwi_disableInterrupt__E
0020bf04   ti_sysbios_family_arm_m3_Hwi_disablePriority__C
002046ed   ti_sysbios_family_arm_m3_Hwi_dispatchC__I
0020533d   ti_sysbios_family_arm_m3_Hwi_dispatch__I
00209999   ti_sysbios_family_arm_m3_Hwi_doSwiRestore__I
00209031   ti_sysbios_family_arm_m3_Hwi_doTaskRestore__I
002086d1   ti_sysbios_family_arm_m3_Hwi_enableInterrupt__E
00206371   ti_sysbios_family_arm_m3_Hwi_excBusFault__I
00206649   ti_sysbios_family_arm_m3_Hwi_excDebugMon__I
00200fad   ti_sysbios_family_arm_m3_Hwi_excDumpRegs__I
00205421   ti_sysbios_family_arm_m3_Hwi_excHandlerAsm__I
0020bf08   ti_sysbios_family_arm_m3_Hwi_excHandlerFunc__C
00203bf1   ti_sysbios_family_arm_m3_Hwi_excHandlerMax__I
00209785   ti_sysbios_family_arm_m3_Hwi_excHandler__I
002064e1   ti_sysbios_family_arm_m3_Hwi_excHardFault__I
0020bf0c   ti_sysbios_family_arm_m3_Hwi_excHookFunc__C
00206c4d   ti_sysbios_family_arm_m3_Hwi_excMemFault__I
002089b1   ti_sysbios_family_arm_m3_Hwi_excNmi__I
002087c1   ti_sysbios_family_arm_m3_Hwi_excNoIsr__I
00208211   ti_sysbios_family_arm_m3_Hwi_excReserved__I
0020870d   ti_sysbios_family_arm_m3_Hwi_excSvCall__I
00205bcd   ti_sysbios_family_arm_m3_Hwi_excUsageFault__I
00208571   ti_sysbios_family_arm_m3_Hwi_getTaskSP__E
002087f9   ti_sysbios_family_arm_m3_Hwi_initVTOR__I
00208577   ti_sysbios_family_arm_m3_Hwi_init__I
e000e000   ti_sysbios_family_arm_m3_Hwi_nvic
002053ef   ti_sysbios_family_arm_m3_Hwi_pendSV__I
0020bf10   ti_sysbios_family_arm_m3_Hwi_priGroup__C
20000000   ti_sysbios_family_arm_m3_Hwi_ramVectors
00200040   ti_sysbios_family_arm_m3_Hwi_resetVectors
00205407   ti_sysbios_family_arm_m3_Hwi_return
00209967   ti_sysbios_family_arm_m3_Hwi_startup__E
002095b1   ti_sysbios_family_arm_m3_Hwi_switchFromBootStack__E
00209941   ti_sysbios_family_arm_m3_IntrinsicsSupport_maxbit__E
002099d7   ti_sysbios_family_arm_m3_TaskSupport_Module__startupDone__S
00208001   ti_sysbios_family_arm_m3_TaskSupport_buildTaskStack
00209861   ti_sysbios_family_arm_m3_TaskSupport_checkStack__E
002098bd   ti_sysbios_family_arm_m3_TaskSupport_getStackAlignment__E
00209705   ti_sysbios_family_arm_m3_TaskSupport_glue
0020bf14   ti_sysbios_family_arm_m3_TaskSupport_stackAlignment__C
00208831   ti_sysbios_family_arm_m3_TaskSupport_start__E
00209715   ti_sysbios_family_arm_m3_TaskSupport_swap__E
00208555   ti_sysbios_family_xxx_Hwi_switchToIsrStack
00208565   ti_sysbios_family_xxx_Hwi_switchToTaskStack
00209971   ti_sysbios_fatfs_getFatTime
0020804d   ti_sysbios_fatfs_startup
002093b9   ti_sysbios_gates_GateHwi_Handle__label__S
00204313   ti_sysbios_gates_GateHwi_Instance_init__F
0020bbfc   ti_sysbios_gates_GateHwi_Module__FXNS__C
20009088   ti_sysbios_gates_GateHwi_Module__root__V
0020bccc   ti_sysbios_gates_GateHwi_Object__DESC__C
0020bdec   ti_sysbios_gates_GateHwi_Object__PARAMS__C
002089e5   ti_sysbios_gates_GateHwi_Object__create__S
00209125   ti_sysbios_gates_GateHwi_Object__delete__S
20009090   ti_sysbios_gates_GateHwi_Object__table__V
002095c5   ti_sysbios_gates_GateHwi_enter__E
0020999f   ti_sysbios_gates_GateHwi_leave__E
002099db   ti_sysbios_gates_GateHwi_query__E
002099db   ti_sysbios_gates_GateHwi_query__F
0020bf18   ti_sysbios_gates_GateMutex_A_badContext__C
002093d3   ti_sysbios_gates_GateMutex_Handle__label__S
0020bf1c   ti_sysbios_gates_GateMutex_Instance_State_sem__O
00209795   ti_sysbios_gates_GateMutex_Instance_finalize__F
00208edd   ti_sysbios_gates_GateMutex_Instance_init__F
0020bc20   ti_sysbios_gates_GateMutex_Module__FXNS__C
0020bf20   ti_sysbios_gates_GateMutex_Module__diagsEnabled__C
0020bf24   ti_sysbios_gates_GateMutex_Module__diagsIncluded__C
0020bf28   ti_sysbios_gates_GateMutex_Module__diagsMask__C
0020c148   ti_sysbios_gates_GateMutex_Module__id__C
20009094   ti_sysbios_gates_GateMutex_Module__root__V
0020bcec   ti_sysbios_gates_GateMutex_Object__DESC__C
0020be04   ti_sysbios_gates_GateMutex_Object__PARAMS__C
00208a19   ti_sysbios_gates_GateMutex_Object__create__S
00209055   ti_sysbios_gates_GateMutex_Object__delete__S
20009814   ti_sysbios_gates_GateMutex_Object__table__V
00206595   ti_sysbios_gates_GateMutex_enter__E
002094e5   ti_sysbios_gates_GateMutex_leave__E
002099df   ti_sysbios_gates_GateMutex_query__E
002099df   ti_sysbios_gates_GateMutex_query__F
0020bf2c   ti_sysbios_hal_Hwi_E_stackOverflow__C
002099e3   ti_sysbios_hal_Hwi_HwiProxy_Module__startupDone__S
00208695   ti_sysbios_hal_Hwi_HwiProxy_disableInterrupt__E
002086d1   ti_sysbios_hal_Hwi_HwiProxy_enableInterrupt__E
00208571   ti_sysbios_hal_Hwi_HwiProxy_getTaskSP__E
00209967   ti_sysbios_hal_Hwi_HwiProxy_startup__E
002095b1   ti_sysbios_hal_Hwi_HwiProxy_switchFromBootStack__E
0020c14c   ti_sysbios_hal_Hwi_Module__id__C
2000909c   ti_sysbios_hal_Hwi_Module__root__V
002096ad   ti_sysbios_hal_Hwi_Module_startup__E
002096ad   ti_sysbios_hal_Hwi_Module_startup__F
00208be1   ti_sysbios_hal_Hwi_checkStack
00208695   ti_sysbios_hal_Hwi_disableInterrupt__E
002086d1   ti_sysbios_hal_Hwi_enableInterrupt__E
00208571   ti_sysbios_hal_Hwi_getTaskSP__E
00208d2d   ti_sysbios_hal_Hwi_initStack
00209967   ti_sysbios_hal_Hwi_startup__E
002095b1   ti_sysbios_hal_Hwi_switchFromBootStack__E
200090a4   ti_sysbios_hal_Timer_Module__root__V
002094fd   ti_sysbios_hal_Timer_Module__startupDone__F
002094fd   ti_sysbios_hal_Timer_Module__startupDone__S
002096bf   ti_sysbios_hal_Timer_Module_startup__E
002096bf   ti_sysbios_hal_Timer_Module_startup__F
200090ac   ti_sysbios_hal_Timer_Object__table__V
002099e7   ti_sysbios_hal_Timer_TimerProxy_Module__startupDone__S
002099eb   ti_sysbios_hal_Timer_TimerProxy_getExpiredCounts__E
002099ef   ti_sysbios_hal_Timer_TimerProxy_getPeriod__E
002099f3   ti_sysbios_hal_Timer_TimerProxy_setNextTick__E
00205ef9   ti_sysbios_hal_Timer_TimerProxy_startup__E
00205ef9   ti_sysbios_hal_Timer_startup__E
0020bf30   ti_sysbios_heaps_HeapMem_A_align__C
0020bf34   ti_sysbios_heaps_HeapMem_A_heapSize__C
0020bf38   ti_sysbios_heaps_HeapMem_A_invalidFree__C
0020bf3c   ti_sysbios_heaps_HeapMem_A_zeroBlock__C
0020bf40   ti_sysbios_heaps_HeapMem_E_memory__C
002093ed   ti_sysbios_heaps_HeapMem_Handle__label__S
200001e8   ti_sysbios_heaps_HeapMem_Instance_State_0_buf__A
00205fb9   ti_sysbios_heaps_HeapMem_Instance_init__F
002099f7   ti_sysbios_heaps_HeapMem_Module_GateProxy_enter__E
002099fb   ti_sysbios_heaps_HeapMem_Module_GateProxy_leave__E
002099df   ti_sysbios_heaps_HeapMem_Module_GateProxy_query__E
0020bbb0   ti_sysbios_heaps_HeapMem_Module__FXNS__C
0020bf44   ti_sysbios_heaps_HeapMem_Module__diagsEnabled__C
0020bf48   ti_sysbios_heaps_HeapMem_Module__diagsIncluded__C
0020bf4c   ti_sysbios_heaps_HeapMem_Module__diagsMask__C
0020bf50   ti_sysbios_heaps_HeapMem_Module__gateObj__C
0020c150   ti_sysbios_heaps_HeapMem_Module__id__C
200090b4   ti_sysbios_heaps_HeapMem_Module__root__V
0020bd0c   ti_sysbios_heaps_HeapMem_Object__DESC__C
0020bd2c   ti_sysbios_heaps_HeapMem_Object__PARAMS__C
0020bf54   ti_sysbios_heaps_HeapMem_Object__count__C
00208a4d   ti_sysbios_heaps_HeapMem_Object__create__S
00209145   ti_sysbios_heaps_HeapMem_Object__delete__S
002095d9   ti_sysbios_heaps_HeapMem_Object__get__S
200090bc   ti_sysbios_heaps_HeapMem_Object__table__V
0020297d   ti_sysbios_heaps_HeapMem_alloc__E
002024dd   ti_sysbios_heaps_HeapMem_free__E
00208259   ti_sysbios_heaps_HeapMem_getStats__E
00208749   ti_sysbios_heaps_HeapMem_init__I
002099a5   ti_sysbios_heaps_HeapMem_isBlocking__E
0020bf58   ti_sysbios_heaps_HeapMem_reqAlignMask__C
0020bf5c   ti_sysbios_heaps_HeapMem_reqAlign__C
0020bf60   ti_sysbios_knl_Clock_A_badThreadType__C
00206851   ti_sysbios_knl_Clock_Instance_finalize__F
00204815   ti_sysbios_knl_Clock_Instance_init__F
0020bf64   ti_sysbios_knl_Clock_LM_begin__C
0020bf68   ti_sysbios_knl_Clock_LM_tick__C
0020bf6c   ti_sysbios_knl_Clock_LW_delayed__C
0020bf70   ti_sysbios_knl_Clock_Module_State_clockQ__O
0020bf74   ti_sysbios_knl_Clock_Module__diagsEnabled__C
0020bf78   ti_sysbios_knl_Clock_Module__diagsIncluded__C
0020bf7c   ti_sysbios_knl_Clock_Module__diagsMask__C
0020c154   ti_sysbios_knl_Clock_Module__id__C
0020c158   ti_sysbios_knl_Clock_Module__loggerDefined__C
0020bf80   ti_sysbios_knl_Clock_Module__loggerFxn1__C
0020bf84   ti_sysbios_knl_Clock_Module__loggerFxn2__C
0020bf88   ti_sysbios_knl_Clock_Module__loggerObj__C
200090d0   ti_sysbios_knl_Clock_Module__root__V
200098e0   ti_sysbios_knl_Clock_Module__state__V
00208c11   ti_sysbios_knl_Clock_Module_startup__E
00208c11   ti_sysbios_knl_Clock_Module_startup__F
0020bd4c   ti_sysbios_knl_Clock_Object__DESC__C
0020bc44   ti_sysbios_knl_Clock_Object__PARAMS__C
00208785   ti_sysbios_knl_Clock_Object__create__S
00209165   ti_sysbios_knl_Clock_Object__destruct__S
002098c9   ti_sysbios_knl_Clock_Params__init__S
00208d59   ti_sysbios_knl_Clock_doTick__I
00208099   ti_sysbios_knl_Clock_getTicks__E
00207c39   ti_sysbios_knl_Clock_logTick__E
00207c99   ti_sysbios_knl_Clock_startI__E
00207751   ti_sysbios_knl_Clock_start__E
0020c1d0   ti_sysbios_knl_Clock_tickMode__C
0020c1d4   ti_sysbios_knl_Clock_tickSource__C
0020493d   ti_sysbios_knl_Clock_workFunc__E
200090d8   ti_sysbios_knl_Event_Module__root__V
0020be74   ti_sysbios_knl_Idle_funcList__A
0020be7c   ti_sysbios_knl_Idle_funcList__C
002085d5   ti_sysbios_knl_Idle_loop__E
00209941   ti_sysbios_knl_Intrinsics_SupportProxy_maxbit__E
00209941   ti_sysbios_knl_Intrinsics_maxbit__E
002099ab   ti_sysbios_knl_Queue_Instance_init__F
200090e4   ti_sysbios_knl_Queue_Module__root__V
0020bd6c   ti_sysbios_knl_Queue_Object__DESC__C
0020be1c   ti_sysbios_knl_Queue_Object__PARAMS__C
00208a81   ti_sysbios_knl_Queue_Object__create__S
00209349   ti_sysbios_knl_Queue_Object__destruct__S
002098d5   ti_sysbios_knl_Queue_Object__get__S
0020986f   ti_sysbios_knl_Queue_empty__E
0020bf8c   ti_sysbios_knl_Semaphore_A_badContext__C
0020bf90   ti_sysbios_knl_Semaphore_A_noEvents__C
0020bf94   ti_sysbios_knl_Semaphore_Instance_State_pendQ__O
002097a5   ti_sysbios_knl_Semaphore_Instance_finalize__F
00206a55   ti_sysbios_knl_Semaphore_Instance_init__F
0020bf98   ti_sysbios_knl_Semaphore_LM_pend__C
0020bf9c   ti_sysbios_knl_Semaphore_LM_post__C
0020bfa0   ti_sysbios_knl_Semaphore_Module__diagsEnabled__C
0020bfa4   ti_sysbios_knl_Semaphore_Module__diagsIncluded__C
0020bfa8   ti_sysbios_knl_Semaphore_Module__diagsMask__C
0020c15c   ti_sysbios_knl_Semaphore_Module__id__C
0020c160   ti_sysbios_knl_Semaphore_Module__loggerDefined__C
0020bfac   ti_sysbios_knl_Semaphore_Module__loggerFxn2__C
0020bfb0   ti_sysbios_knl_Semaphore_Module__loggerFxn4__C
0020bfb4   ti_sysbios_knl_Semaphore_Module__loggerObj__C
200090ec   ti_sysbios_knl_Semaphore_Module__root__V
0020bd8c   ti_sysbios_knl_Semaphore_Object__DESC__C
0020bc68   ti_sysbios_knl_Semaphore_Object__PARAMS__C
00208869   ti_sysbios_knl_Semaphore_Object__create__S
00209185   ti_sysbios_knl_Semaphore_Object__destruct__S
002088a1   ti_sysbios_knl_Semaphore_pendTimeout__I
00203549   ti_sysbios_knl_Semaphore_pend__E
002062b5   ti_sysbios_knl_Semaphore_post__E
0020bfb8   ti_sysbios_knl_Swi_LD_end__C
0020bfbc   ti_sysbios_knl_Swi_LM_begin__C
0020bfc0   ti_sysbios_knl_Swi_LM_post__C
200094f8   ti_sysbios_knl_Swi_Module_State_0_readyQ__A
0020bfc4   ti_sysbios_knl_Swi_Module__diagsEnabled__C
0020bfc8   ti_sysbios_knl_Swi_Module__diagsIncluded__C
0020bfcc   ti_sysbios_knl_Swi_Module__diagsMask__C
0020c164   ti_sysbios_knl_Swi_Module__id__C
0020c168   ti_sysbios_knl_Swi_Module__loggerDefined__C
0020bfd0   ti_sysbios_knl_Swi_Module__loggerFxn1__C
0020bfd4   ti_sysbios_knl_Swi_Module__loggerFxn4__C
0020bfd8   ti_sysbios_knl_Swi_Module__loggerObj__C
200090f8   ti_sysbios_knl_Swi_Module__root__V
20009100   ti_sysbios_knl_Swi_Module__state__V
00209079   ti_sysbios_knl_Swi_Module_startup__E
00209079   ti_sysbios_knl_Swi_Module_startup__F
0020bfdc   ti_sysbios_knl_Swi_Object__count__C
002095ed   ti_sysbios_knl_Swi_Object__get__S
200098b0   ti_sysbios_knl_Swi_Object__table__V
002097b5   ti_sysbios_knl_Swi_disable__E
002068fd   ti_sysbios_knl_Swi_post__E
00207e6d   ti_sysbios_knl_Swi_restoreHwi__E
00204ef5   ti_sysbios_knl_Swi_run__I
00206afd   ti_sysbios_knl_Swi_schedule__I
00208615   ti_sysbios_knl_Swi_startup__E
0020bfe0   ti_sysbios_knl_Task_A_badPriority__C
0020bfe4   ti_sysbios_knl_Task_A_badTaskState__C
0020bfe8   ti_sysbios_knl_Task_A_badThreadType__C
0020bfec   ti_sysbios_knl_Task_A_noPendElem__C
0020bff0   ti_sysbios_knl_Task_E_spOutOfBounds__C
0020bff4   ti_sysbios_knl_Task_E_stackOverflow__C
20002ce8   ti_sysbios_knl_Task_Instance_State_0_hookEnv__A
200011e8   ti_sysbios_knl_Task_Instance_State_0_stack__A
00202bb5   ti_sysbios_knl_Task_Instance_finalize__F
00202fc1   ti_sysbios_knl_Task_Instance_init__F
0020bff8   ti_sysbios_knl_Task_LD_block__C
0020bffc   ti_sysbios_knl_Task_LD_exit__C
0020c000   ti_sysbios_knl_Task_LD_ready__C
0020c004   ti_sysbios_knl_Task_LM_switch__C
20009578   ti_sysbios_knl_Task_Module_State_0_readyQ__A
0020c008   ti_sysbios_knl_Task_Module_State_inactiveQ__O
0020c00c   ti_sysbios_knl_Task_Module_State_terminatedQ__O
0020c010   ti_sysbios_knl_Task_Module__diagsEnabled__C
0020c014   ti_sysbios_knl_Task_Module__diagsIncluded__C
0020c018   ti_sysbios_knl_Task_Module__diagsMask__C
0020c16c   ti_sysbios_knl_Task_Module__id__C
0020c170   ti_sysbios_knl_Task_Module__loggerDefined__C
0020c01c   ti_sysbios_knl_Task_Module__loggerFxn2__C
0020c020   ti_sysbios_knl_Task_Module__loggerFxn4__C
0020c024   ti_sysbios_knl_Task_Module__loggerObj__C
2000911c   ti_sysbios_knl_Task_Module__root__V
2000984c   ti_sysbios_knl_Task_Module__state__V
0020729d   ti_sysbios_knl_Task_Module_startup__E
0020729d   ti_sysbios_knl_Task_Module_startup__F
0020bdac   ti_sysbios_knl_Task_Object__DESC__C
0020bac4   ti_sysbios_knl_Task_Object__PARAMS__C
0020c028   ti_sysbios_knl_Task_Object__count__C
002079e5   ti_sysbios_knl_Task_Object__create__S
00209601   ti_sysbios_knl_Task_Object__first__S
00209615   ti_sysbios_knl_Task_Object__get__S
0020c02c   ti_sysbios_knl_Task_Object__heap__C
00209629   ti_sysbios_knl_Task_Object__next__S
200097cc   ti_sysbios_knl_Task_Object__table__V
002098e1   ti_sysbios_knl_Task_Params__init__S
002099ff   ti_sysbios_knl_Task_SupportProxy_Module__startupDone__S
00209861   ti_sysbios_knl_Task_SupportProxy_checkStack__E
002098bd   ti_sysbios_knl_Task_SupportProxy_getStackAlignment__E
00208831   ti_sysbios_knl_Task_SupportProxy_start__E
00209715   ti_sysbios_knl_Task_SupportProxy_swap__E
0020c030   ti_sysbios_knl_Task_allBlockedFunc__C
00208d85   ti_sysbios_knl_Task_allBlockedFunction__I
00206d91   ti_sysbios_knl_Task_blockI__E
002069a9   ti_sysbios_knl_Task_checkStacks__E
0020c034   ti_sysbios_knl_Task_defaultStackHeap__C
0020c038   ti_sysbios_knl_Task_defaultStackSize__C
0020c174   ti_sysbios_knl_Task_deleteTerminatedTasks__C
002097c5   ti_sysbios_knl_Task_disable__E
002091a5   ti_sysbios_knl_Task_enter__I
00204a65   ti_sysbios_knl_Task_exit__E
0020bafc   ti_sysbios_knl_Task_hooks__A
0020be84   ti_sysbios_knl_Task_hooks__C
0020c178   ti_sysbios_knl_Task_initStackFlag__C
0020c03c   ti_sysbios_knl_Task_numConstructedTasks__C
0020c040   ti_sysbios_knl_Task_numPriorities__C
00205641   ti_sysbios_knl_Task_postInit__I
00208ab5   ti_sysbios_knl_Task_restore__E
0020522d   ti_sysbios_knl_Task_schedule__I
00205739   ti_sysbios_knl_Task_startup__E
00206079   ti_sysbios_knl_Task_unblockI__E
0020c044   ti_sysbios_utils_Load_LS_cpuLoad__C
0020c048   ti_sysbios_utils_Load_LS_hwiLoad__C
0020c04c   ti_sysbios_utils_Load_LS_swiLoad__C
0020c050   ti_sysbios_utils_Load_LS_taskLoad__C
0020c054   ti_sysbios_utils_Load_Module_State_gate__O
0020c058   ti_sysbios_utils_Load_Module_State_taskList__O
0020c05c   ti_sysbios_utils_Load_Module__diagsEnabled__C
0020c060   ti_sysbios_utils_Load_Module__diagsIncluded__C
0020c064   ti_sysbios_utils_Load_Module__diagsMask__C
0020c17c   ti_sysbios_utils_Load_Module__id__C
0020c180   ti_sysbios_utils_Load_Module__loggerDefined__C
0020c068   ti_sysbios_utils_Load_Module__loggerFxn1__C
0020c06c   ti_sysbios_utils_Load_Module__loggerFxn2__C
0020c070   ti_sysbios_utils_Load_Module__loggerFxn4__C
0020c074   ti_sysbios_utils_Load_Module__loggerObj__C
20009128   ti_sysbios_utils_Load_Module__root__V
20009460   ti_sysbios_utils_Load_Module__state__V
00206ba5   ti_sysbios_utils_Load_addTask__E
0020c184   ti_sysbios_utils_Load_autoAddTasks__C
0020c188   ti_sysbios_utils_Load_hwiEnabled__C
00206429   ti_sysbios_utils_Load_idleFxn__E
00203375   ti_sysbios_utils_Load_logLoads__I
0020c078   ti_sysbios_utils_Load_postUpdate__C
002077c1   ti_sysbios_utils_Load_removeTask__E
0020c18c   ti_sysbios_utils_Load_swiEnabled__C
00207089   ti_sysbios_utils_Load_taskCreateHook__E
00207585   ti_sysbios_utils_Load_taskDeleteHook__E
0020c190   ti_sysbios_utils_Load_taskEnabled__C
002098ed   ti_sysbios_utils_Load_taskRegHook__E
00207f11   ti_sysbios_utils_Load_taskSwitchHook__E
0020c194   ti_sysbios_utils_Load_updateInIdle__C
0020272d   ti_sysbios_utils_Load_update__E
0020c07c   ti_sysbios_utils_Load_windowInMs__C
0020c080   ti_uia_runtime_ILoggerSnapshot_Interface__BASE__C
0020c084   ti_uia_runtime_IUIATransfer_Interface__BASE__C
00209a03   ti_uia_runtime_LogSync_CpuTimestampProxy_Module__startupDone__S
002098b1   ti_uia_runtime_LogSync_CpuTimestampProxy_get32__E
00208eb5   ti_uia_runtime_LogSync_CpuTimestampProxy_get64__E
00209775   ti_uia_runtime_LogSync_CpuTimestampProxy_getFreq__E
00209a07   ti_uia_runtime_LogSync_GlobalTimestampProxy_Module__startupDone__S
2000912c   ti_uia_runtime_LogSync_Module__root__V
20009134   ti_uia_runtime_LogSync_Module__state__V
00208f2d   ti_uia_runtime_LogSync_Module_startup__E
00208f2d   ti_uia_runtime_LogSync_Module_startup__F
0020c088   ti_uia_runtime_LoggerStopMode_E_badLevel__C
00209407   ti_uia_runtime_LoggerStopMode_Handle__label__S
200026e8   ti_uia_runtime_LoggerStopMode_Instance_State_0_bufferArray__A
200019e8   ti_uia_runtime_LoggerStopMode_Instance_State_1_bufferArray__A
20001e68   ti_uia_runtime_LoggerStopMode_Instance_State_2_bufferArray__A
0020909d   ti_uia_runtime_LoggerStopMode_Instance_finalize__F
00208331   ti_uia_runtime_LoggerStopMode_Instance_init__F
0020b938   ti_uia_runtime_LoggerStopMode_Module__FXNS__C
0020c198   ti_uia_runtime_LoggerStopMode_Module__id__C
20009140   ti_uia_runtime_LoggerStopMode_Module__root__V
20009148   ti_uia_runtime_LoggerStopMode_Module__state__V
00208db1   ti_uia_runtime_LoggerStopMode_Module_startup__E
00208db1   ti_uia_runtime_LoggerStopMode_Module_startup__F
0020bdcc   ti_uia_runtime_LoggerStopMode_Object__DESC__C
0020bb2c   ti_uia_runtime_LoggerStopMode_Object__PARAMS__C
0020c08c   ti_uia_runtime_LoggerStopMode_Object__count__C
00207cf9   ti_uia_runtime_LoggerStopMode_Object__create__S
002091c5   ti_uia_runtime_LoggerStopMode_Object__delete__S
002097d5   ti_uia_runtime_LoggerStopMode_Object__get__S
20009358   ti_uia_runtime_LoggerStopMode_Object__table__V
00208ddd   ti_uia_runtime_LoggerStopMode_disable__E
00208e09   ti_uia_runtime_LoggerStopMode_enable__E
0020c19c   ti_uia_runtime_LoggerStopMode_filterByLevel__C
002080e5   ti_uia_runtime_LoggerStopMode_filterOutEvent__I
0020731d   ti_uia_runtime_LoggerStopMode_getContents__E
002075fd   ti_uia_runtime_LoggerStopMode_getFilterLevel__E
00209571   ti_uia_runtime_LoggerStopMode_getFreeSize__E
00209a0b   ti_uia_runtime_LoggerStopMode_getInstanceId__E
00209a0f   ti_uia_runtime_LoggerStopMode_getMaxLength__E
002099b1   ti_uia_runtime_LoggerStopMode_getPriority__E
002099b7   ti_uia_runtime_LoggerStopMode_getTransferType__E
002099b7   ti_uia_runtime_LoggerStopMode_getTransferType__F
00209587   ti_uia_runtime_LoggerStopMode_getUnreadSize__E
002097e5   ti_uia_runtime_LoggerStopMode_isEmpty__E
0020c1a0   ti_uia_runtime_LoggerStopMode_isTimestampEnabled__C
0020c090   ti_uia_runtime_LoggerStopMode_overflowLogger__C
00207db7   ti_uia_runtime_LoggerStopMode_readBlockOfMemory__I
00208489   ti_uia_runtime_LoggerStopMode_reset__E
00208489   ti_uia_runtime_LoggerStopMode_reset__F
0020739d   ti_uia_runtime_LoggerStopMode_setFilterLevel__E
00209a13   ti_uia_runtime_LoggerStopMode_setPriority__E
0020c094   ti_uia_runtime_LoggerStopMode_statusLogger__C
002097f5   ti_uia_runtime_LoggerStopMode_write0__E
002096d1   ti_uia_runtime_LoggerStopMode_write1__E
0020963d   ti_uia_runtime_LoggerStopMode_write2__E
00204465   ti_uia_runtime_LoggerStopMode_write4__E
00203715   ti_uia_runtime_LoggerStopMode_write8__E
0020790d   ti_uia_runtime_LoggerStopMode_writeBlockOfMemory__I
00203f09   ti_uia_runtime_LoggerStopMode_writeMemoryRange__E
002084cd   ti_uia_runtime_QueueDescriptor_addToList__E
20009930   ti_uia_runtime_QueueDescriptor_gPtrToFirstDescriptor
20009934   ti_uia_runtime_QueueDescriptor_gUpdateCount
00208f55   ti_uia_runtime_QueueDescriptor_initHeader__E
00208131   ti_uia_runtime_QueueDescriptor_removeFromList__E
00205441   uart1Isr
0020b8d8   uartHWAttrs
20002bc0   uartObjects
00201433   unlink
00201385   write
00207bd9   writemsg
0020c098   xdc_runtime_Assert_E_assertFailed__C
002082a1   xdc_runtime_Assert_raise__I
0020c09c   xdc_runtime_Core_A_initializedParams__C
0020c0a0   xdc_runtime_Core_Module__diagsEnabled__C
0020c0a4   xdc_runtime_Core_Module__diagsIncluded__C
0020c0a8   xdc_runtime_Core_Module__diagsMask__C
0020c1a4   xdc_runtime_Core_Module__id__C
00208c41   xdc_runtime_Core_assignLabel__I
002082e9   xdc_runtime_Core_assignParams__I
00204315   xdc_runtime_Core_createObject__I
00207a4d   xdc_runtime_Core_deleteObject__I
0020c0ac   xdc_runtime_Error_E_generic__C
0020c0b0   xdc_runtime_Error_E_memory__C
0020c0b4   xdc_runtime_Error_Module__diagsEnabled__C
0020c0b8   xdc_runtime_Error_Module__diagsIncluded__C
0020c0bc   xdc_runtime_Error_Module__diagsMask__C
0020c1a8   xdc_runtime_Error_Module__loggerDefined__C
0020c0c0   xdc_runtime_Error_Module__loggerFxn8__C
0020c0c4   xdc_runtime_Error_Module__loggerObj__C
20009150   xdc_runtime_Error_Module__state__V
00209365   xdc_runtime_Error_check__E
00209365   xdc_runtime_Error_check__F
00209a17   xdc_runtime_Error_getSite__E
00209a17   xdc_runtime_Error_getSite__F
002098f9   xdc_runtime_Error_init__E
002098f9   xdc_runtime_Error_init__F
0020c1ac   xdc_runtime_Error_maxDepth__C
0020c1d8   xdc_runtime_Error_policy__C
00207979   xdc_runtime_Error_print__E
00207979   xdc_runtime_Error_print__F
0020c0c8   xdc_runtime_Error_raiseHook__C
002045b1   xdc_runtime_Error_raiseX__E
002045b1   xdc_runtime_Error_raiseX__F
00209905   xdc_runtime_Gate_enterSystem__E
00209905   xdc_runtime_Gate_enterSystem__F
00209805   xdc_runtime_Gate_leaveSystem__E
00209805   xdc_runtime_Gate_leaveSystem__F
0020c0cc   xdc_runtime_IFilterLogger_Interface__BASE__C
0020c0d0   xdc_runtime_IGateProvider_Interface__BASE__C
0020c0d4   xdc_runtime_IHeap_Interface__BASE__C
0020c0d8   xdc_runtime_ILogger_Interface__BASE__C
0020c0dc   xdc_runtime_IModule_Interface__BASE__C
0020c0e0   xdc_runtime_Log_L_error__C
002099db   xdc_runtime_Main_Module_GateProxy_query__E
0020c0e4   xdc_runtime_Main_Module__diagsEnabled__C
0020c0e8   xdc_runtime_Main_Module__diagsIncluded__C
0020c0ec   xdc_runtime_Main_Module__diagsMask__C
0020c1b0   xdc_runtime_Main_Module__id__C
0020c1b4   xdc_runtime_Main_Module__loggerDefined__C
0020c0f0   xdc_runtime_Main_Module__loggerFxn4__C
0020c0f4   xdc_runtime_Main_Module__loggerObj__C
20009152   xdc_runtime_Main_Module__root__V
00209a1b   xdc_runtime_Memory_HeapProxy_alloc__E
00209a1f   xdc_runtime_Memory_HeapProxy_free__E
0020c1b8   xdc_runtime_Memory_Module__id__C
20009154   xdc_runtime_Memory_Module__state__V
00207831   xdc_runtime_Memory_alloc__E
00207831   xdc_runtime_Memory_alloc__F
00209911   xdc_runtime_Memory_calloc__E
00209911   xdc_runtime_Memory_calloc__F
0020c0f8   xdc_runtime_Memory_defaultHeapInstance__C
00209815   xdc_runtime_Memory_free__E
00209815   xdc_runtime_Memory_free__F
0020991d   xdc_runtime_Memory_getMaxDefaultTypeAlign__E
0020991d   xdc_runtime_Memory_getMaxDefaultTypeAlign__F
00209381   xdc_runtime_Memory_valloc__E
00209381   xdc_runtime_Memory_valloc__F
20009158   xdc_runtime_Registry_Module__state__V
002091e5   xdc_runtime_Registry_findById__E
002091e5   xdc_runtime_Registry_findById__F
20009160   xdc_runtime_Startup_Module__state__V
00000001   xdc_runtime_Startup__EXECFXN__C
00000001   xdc_runtime_Startup__RESETFXN__C
0020c0fc   xdc_runtime_Startup_execImpl__C
00207f61   xdc_runtime_Startup_exec__E
00207f61   xdc_runtime_Startup_exec__F
002096e3   xdc_runtime_Startup_exec__I
0020be4c   xdc_runtime_Startup_firstFxns__A
0020be8c   xdc_runtime_Startup_firstFxns__C
0020c100   xdc_runtime_Startup_lastFxns__A
0020be94   xdc_runtime_Startup_lastFxns__C
0020c104   xdc_runtime_Startup_maxPasses__C
00209a23   xdc_runtime_Startup_reset__I
0020be34   xdc_runtime_Startup_sfxnRts__A
0020c108   xdc_runtime_Startup_sfxnRts__C
0020bb5c   xdc_runtime_Startup_sfxnTab__A
0020c10c   xdc_runtime_Startup_sfxnTab__C
00205545   xdc_runtime_Startup_startMods__I
200022e8   xdc_runtime_SysMin_Module_State_0_outbuf__A
20009168   xdc_runtime_SysMin_Module__state__V
00209205   xdc_runtime_SysMin_Module_startup__E
00209205   xdc_runtime_SysMin_Module_startup__F
00208c71   xdc_runtime_SysMin_abort__E
00208c71   xdc_runtime_SysMin_abort__F
0020c110   xdc_runtime_SysMin_bufSize__C
0020939d   xdc_runtime_SysMin_exit__E
0020939d   xdc_runtime_SysMin_exit__F
0020c1bc   xdc_runtime_SysMin_flushAtExit__C
00208511   xdc_runtime_SysMin_flush__E
00208511   xdc_runtime_SysMin_flush__F
0020c114   xdc_runtime_SysMin_outputFunc__C
002090c1   xdc_runtime_SysMin_output__I
002088d9   xdc_runtime_SysMin_putch__E
002088d9   xdc_runtime_SysMin_putch__F
00209825   xdc_runtime_SysMin_ready__E
00209825   xdc_runtime_SysMin_ready__F
00209a27   xdc_runtime_System_Module_GateProxy_enter__E
00209a2b   xdc_runtime_System_Module_GateProxy_leave__E
002099db   xdc_runtime_System_Module_GateProxy_query__E
20009174   xdc_runtime_System_Module_State_0_atexitHandlers__A
0020c118   xdc_runtime_System_Module__gateObj__C
20009194   xdc_runtime_System_Module__state__V
002099bd   xdc_runtime_System_Module_startup__E
002099bd   xdc_runtime_System_Module_startup__F
00208c71   xdc_runtime_System_SupportProxy_abort__E
0020939d   xdc_runtime_System_SupportProxy_exit__E
00208511   xdc_runtime_System_SupportProxy_flush__E
002088d9   xdc_runtime_System_SupportProxy_putch__E
00209825   xdc_runtime_System_SupportProxy_ready__E
00209651   xdc_runtime_System_abort__E
00209651   xdc_runtime_System_abort__F
00209421   xdc_runtime_System_aprintf__E
00209a2f   xdc_runtime_System_aprintf_va__F
00208655   xdc_runtime_System_atexit__E
00208655   xdc_runtime_System_atexit__F
00209225   xdc_runtime_System_avprintf__F
002016f1   xdc_runtime_System_doPrint__I
00209929   xdc_runtime_System_exit__E
00209929   xdc_runtime_System_exit__F
0020c11c   xdc_runtime_System_extendFxn__C
00208511   xdc_runtime_System_flush__E
00208511   xdc_runtime_System_flush__F
00207fb1   xdc_runtime_System_formatNum__I
00209935   xdc_runtime_System_lastFxn__I
0020c120   xdc_runtime_System_maxAtexitHandlers__C
0020591f   xdc_runtime_System_printfExtend__I
0020943b   xdc_runtime_System_printf__E
00209a33   xdc_runtime_System_printf_va__F
00209245   xdc_runtime_System_putchar__I
00208e35   xdc_runtime_System_rtsExit__I
00209265   xdc_runtime_System_vprintf__F
00209a37   xdc_runtime_System_vsprintf__E
0020987d   xdc_runtime_System_vsprintf__F
200091a0   xdc_runtime_Text_Module__state__V
0020c1c0   xdc_runtime_Text_charCnt__C
00209a50   xdc_runtime_Text_charTab__A
0020c124   xdc_runtime_Text_charTab__C
00208e61   xdc_runtime_Text_cordText__E
00208e61   xdc_runtime_Text_cordText__F
0020c1c4   xdc_runtime_Text_isLoaded__C
0020c128   xdc_runtime_Text_nameEmpty__C
0020c12c   xdc_runtime_Text_nameStatic__C
0020c130   xdc_runtime_Text_nameUnknown__C
0020b7d0   xdc_runtime_Text_nodeTab__A
0020c134   xdc_runtime_Text_nodeTab__C
00208b1d   xdc_runtime_Text_printVisFxn__I
00207e15   xdc_runtime_Text_putLab__E
00207e15   xdc_runtime_Text_putLab__F
00206ff9   xdc_runtime_Text_putMod__E
00206ff9   xdc_runtime_Text_putMod__F
00206f65   xdc_runtime_Text_putSite__E
00206f65   xdc_runtime_Text_putSite__F
0020c1c8   xdc_runtime_Text_registryModsLastId__C
0020952d   xdc_runtime_Text_ropeText__E
0020952d   xdc_runtime_Text_ropeText__F
0020c1cc   xdc_runtime_Text_unnamedModsLastId__C
0020817d   xdc_runtime_Text_visitRope2__I
0020c138   xdc_runtime_Text_visitRopeFxn__C
00209835   xdc_runtime_Text_visitRope__I
00208ca1   xdc_runtime_Text_xprintf__I
00209a3b   xdc_runtime_TimestampNull_Module__startupDone__S
00209a3f   xdc_runtime_Timestamp_Module__startupDone__S
002098b1   xdc_runtime_Timestamp_SupportProxy_get32__E
00208eb5   xdc_runtime_Timestamp_SupportProxy_get64__E
00209775   xdc_runtime_Timestamp_SupportProxy_getFreq__E
002098b1   xdc_runtime_Timestamp_get32__E
002098b1   xdc_runtime_Timestamp_get32__F
00208eb5   xdc_runtime_Timestamp_get64__E
00208eb5   xdc_runtime_Timestamp_get64__F
00209775   xdc_runtime_Timestamp_getFreq__E
00209775   xdc_runtime_Timestamp_getFreq__F


GLOBAL SYMBOLS: SORTED BY Symbol Address 

address    name
--------   ----
00000000   __ASM__
00000001   __TI_args_main
00000001   xdc_runtime_Startup__EXECFXN__C
00000001   xdc_runtime_Startup__RESETFXN__C
00000062   __ISA__
00000074   __PLAT__
0000009b   __TARG__
000000c0   __TRDR__
00001000   __STACK_SIZE
00200031   _ti_catalog_arm_cortexm3_concertoInit_Boot_entry
00200040   ti_sysbios_family_arm_m3_Hwi_resetVectors
002001ed   SysCtlSRAMSizeGet
0020020b   SysCtlFlashSizeGet
00200217   SysCtlPeripheralPresent
00200279   SysCtlPeripheralReset
00200341   SysCtlPeripheralEnable
00200367   SysCtlPeripheralDisable
0020038d   SysCtlPeripheralIsEnabled
002003ab   SysCtlPeripheralSleepEnable
002003d1   SysCtlPeripheralSleepDisable
002003f7   SysCtlPeripheralDeepSleepEnable
00200421   SysCtlPeripheralDeepSleepDisable
0020044d   SysCtlPeripheralClockGating
00200475   SysCtlReset
00200489   SysCtlDeepSleep
002004a9   SysCtlResetCauseGet
002004b5   SysCtlResetCauseClear
002004d1   SysCtlXPllClockDividerSet
00200549   SysCtlClockDividersSet
0020064f   SysCtlPowerOffPLL
00200681   SysCtlClockPllConfig
002007ad   SysCtlClockConfigSet
002007e1   SysCtlClockConfigGet
00200831   SysCtlClockGet
002008ab   SysCtlC28Enable
002008c3   SysCtlC28Disable
002008db   SysCtlGPIOAHBEnable
002008f7   SysCtlGPIOAHBDisable
00200915   SysCtlUSBPLLEnable
00200949   SysCtlUSBPLLDisable
00200965   SysCtlUSBPLLConfigSet
002009fd   SysCtlUSBPLLConfigGet
00200a1b   SysCtlEnableAERRNMI
00200a35   SysCtlEnableVREGWarnNMI
00200a4d   SysCtlGetNmiConfig
00200a53   SysCtlGetNmiInterruptStatus
00200a61   SysCtlGetNmiFlagStatus
00200a69   SysCtlNmiIsSet
00200a81   SysCtlNmiFlgClr
00200a99   SysCtlNmiFlgClrAll
00200ab7   SysCtlHoldSubSystemInReset
00200add   SysCtlReleaseSubSystemFromReset
00200b05   SysCtlSubSystemReset
00200bff   GPIODirModeSet
00200c2f   GPIODirModeGet
00200c59   GPIOIntTypeSet
00200c9f   GPIOIntTypeGet
00200cd9   GPIOPadConfigSet
00200d33   GPIOPadConfigGet
00200d6f   GPIOPinIntEnable
00200d7b   GPIOPinIntDisable
00200d89   GPIOPinIntStatus
00200d97   GPIOPinIntClear
00200d9d   GPIOPortIntRegister
00200db5   GPIOPortIntUnregister
00200dc9   GPIOPinRead
00200dcf   GPIOPinWrite
00200dd5   GPIOPinTypeCAN
00200de9   GPIOPinTypeGPIOInput
00200dfd   GPIOPinTypeGPIOOutput
00200e19   GPIOPinTypeGPIOOutputOD
00200e2d   GPIOPinTypeI2C
00200e45   GPIOPinTypeSSI
00200e5d   GPIOPinTypeTimer
00200e71   GPIOPinTypeUART
00200e85   GPIOPinTypeUSBDigital
00200e99   GPIOPinTypeUSBAnalog
00200ead   GPIOPinTypeEPI
00200ec1   GPIOPinConfigure
00200f2b   GPIOPinConfigureCoreSelect
00200f4b   GPIOPinLockStatus
00200f55   GPIOPinLock
00200f7b   GPIOPinUnlock
00200fad   ti_sysbios_family_arm_m3_Hwi_excDumpRegs__I
00201385   write
00201433   unlink
00201457   rename
00201493   remove_device
002014bb   read
00201537   open
002015bf   lseek
002015ff   find_registered_device
00201615   close
00201663   add_device
002016f1   xdc_runtime_System_doPrint__I
00201ced   getenv
00201d2b   HOSTwrite
00201d79   HOSTunlink
00201db3   HOSTtime
00201def   HOSTrename
00201e4f   HOSTread
00201e9d   HOSTopen
00201eed   HOSTlseek
00201f49   HOSTclose
00201f8d   HOSTclock
00201fd9   UARTParityModeSet
00201fe5   UARTParityModeGet
00201fed   UARTFIFOLevelSet
00201ff3   UARTFIFOLevelGet
00202003   UARTConfigSetExpClk
0020204d   UARTConfigGetExpClk
00202075   UARTEnable
00202089   UARTDisable
002020a1   UARTFIFOEnable
002020ab   UARTFIFODisable
002020b5   UARTEnableSIR
002020cb   UARTDisableSIR
002020d5   UARTSmartCardEnable
002020eb   UARTSmartCardDisable
002020f5   UARTModemControlSet
00202101   UARTModemControlClear
00202111   UARTModemControlGet
00202119   UARTModemStatusGet
00202123   UARTFlowControlSet
0020212f   UARTFlowControlGet
00202137   UARTTxIntModeSet
00202143   UARTTxIntModeGet
0020214b   UARTCharsAvail
00202157   UARTSpaceAvail
00202163   UARTCharGetNonBlocking
00202173   UARTCharGet
0020217d   UARTCharPutNonBlocking
0020218d   UARTCharPut
00202197   UARTBreakCtl
002021ab   UARTBusy
002021b3   UARTIntRegister
002021ef   UARTIntUnregister
0020222b   UARTIntEnable
00202233   UARTIntDisable
0020223d   UARTIntStatus
00202247   UARTIntClear
0020224b   UARTDMAEnable
00202253   UARTDMADisable
0020225d   UARTRxErrorGet
00202265   UARTRxErrorClear
00202281   IntMasterEnable
0020228b   IntMasterDisable
00202295   IntFlashVTable
00202297   IntRAMVTable
00202299   IntRegister
0020229b   IntUnregister
0020229d   IntPriorityGroupingSet
002022ad   IntPriorityGroupingGet
002022cd   IntPrioritySet
002022f9   IntPriorityGet
00202311   IntEnable
00202385   IntDisable
002023fb   IntPendSet
00202463   IntPendClear
002024dd   ti_sysbios_heaps_HeapMem_free__E
0020272d   ti_sysbios_utils_Load_update__E
0020297d   ti_sysbios_heaps_HeapMem_alloc__E
00202bb5   ti_sysbios_knl_Task_Instance_finalize__F
00202de1   f_write
00202fc1   ti_sysbios_knl_Task_Instance_init__F
0020319d   ti_catalog_arm_cortexm3_concertoInit_Boot_initC28RAMs
00203249   ti_catalog_arm_cortexm3_concertoInit_Boot_defaultLimpAbortFunction
0020324b   ti_catalog_arm_cortexm3_concertoInit_Boot_configurePllDivs
00203339   ti_catalog_arm_cortexm3_concertoInit_Boot_bootC28
00203375   ti_sysbios_utils_Load_logLoads__I
00203549   ti_sysbios_knl_Semaphore_pend__E
00203715   ti_uia_runtime_LoggerStopMode_write8__E
002038c1   f_read
00203a65   GPIO_write
00203bf1   ti_sysbios_family_arm_m3_Hwi_excHandlerMax__I
00203d7d   f_lseek
00203f07   ti_sysbios_family_arm_lm3_Timer_setNextTick__E
00203f09   ti_uia_runtime_LoggerStopMode_writeMemoryRange__E
0020406d   UartTask
002041c1   f_open
00204313   ti_sysbios_gates_GateHwi_Instance_init__F
00204315   xdc_runtime_Core_createObject__I
00204465   ti_uia_runtime_LoggerStopMode_write4__E
002045b1   xdc_runtime_Error_raiseX__E
002045b1   xdc_runtime_Error_raiseX__F
002046ed   ti_sysbios_family_arm_m3_Hwi_dispatchC__I
00204815   ti_sysbios_knl_Clock_Instance_init__F
0020493d   ti_sysbios_knl_Clock_workFunc__E
00204a65   ti_sysbios_knl_Task_exit__E
00204b8d   f_rename
00204cdb   SSIConfigSetExpClk
00204d1f   SSIEnable
00204d29   SSIDisable
00204d33   SSIIntRegister
00204d4b   SSIIntUnregister
00204d5f   SSIIntEnable
00204d67   SSIIntDisable
00204d71   SSIIntStatus
00204d7b   SSIIntClear
00204d7f   SSIDataPut
00204d89   SSIDataPutNonBlocking
00204d99   SSIDataGet
00204da5   SSIDataGetNonBlocking
00204db7   SSIDMAEnable
00204dbf   SSIDMADisable
00204dc9   SSIBusy
00204dd5   ti_sysbios_family_arm_m3_Hwi_Module_startup__E
00204dd5   ti_sysbios_family_arm_m3_Hwi_Module_startup__F
00204ef5   ti_sysbios_knl_Swi_run__I
0020511d   main
0020522d   ti_sysbios_knl_Task_schedule__I
0020533d   ti_sysbios_family_arm_m3_Hwi_dispatch__I
002053ef   ti_sysbios_family_arm_m3_Hwi_pendSV__I
00205407   ti_sysbios_family_arm_m3_Hwi_return
00205421   ti_sysbios_family_arm_m3_Hwi_excHandlerAsm__I
00205441   uart1Isr
00205545   xdc_runtime_Startup_startMods__I
00205641   ti_sysbios_knl_Task_postInit__I
00205739   ti_sysbios_knl_Task_startup__E
0020591f   xdc_runtime_System_printfExtend__I
00205a0d   put_fat
00205af9   ti_sysbios_family_arm_lm3_Timer_enableTimers__I
00205bcd   ti_sysbios_family_arm_m3_Hwi_excUsageFault__I
00205c9d   get_fat
00205d6d   __cxa_atexit
00205d71   atexit
00205d7f   __cxa_finalize
00205dbd   __cxa_ia64_exit
00205dc3   __aeabi_atexit
00205ef9   ti_sysbios_family_arm_lm3_Timer_startup__E
00205ef9   ti_sysbios_hal_Timer_TimerProxy_startup__E
00205ef9   ti_sysbios_hal_Timer_startup__E
00205fb9   ti_sysbios_heaps_HeapMem_Instance_init__F
00206079   ti_sysbios_knl_Task_unblockI__E
00206139   f_sync
002061f7   f_unlink
002062b5   ti_sysbios_knl_Semaphore_post__E
00206371   ti_sysbios_family_arm_m3_Hwi_excBusFault__I
00206429   ti_sysbios_utils_Load_idleFxn__E
002064e1   ti_sysbios_family_arm_m3_Hwi_excHardFault__I
00206595   ti_sysbios_gates_GateMutex_enter__E
00206649   ti_sysbios_family_arm_m3_Hwi_excDebugMon__I
002066f9   WatchdogRunning
00206701   WatchdogEnable
0020670b   WatchdogResetEnable
00206715   WatchdogResetDisable
0020671f   WatchdogLock
00206727   WatchdogUnlock
0020672f   WatchdogLockState
0020673f   WatchdogReloadSet
00206743   WatchdogReloadGet
00206747   WatchdogValueGet
0020674b   WatchdogIntRegister
0020675b   WatchdogIntUnregister
0020676b   WatchdogIntEnable
00206775   WatchdogIntStatus
0020677f   WatchdogIntClear
00206785   WatchdogStallEnable
00206793   WatchdogStallDisable
002067a5   ffcio_open
00206851   ti_sysbios_knl_Clock_Instance_finalize__F
002068fd   ti_sysbios_knl_Swi_post__E
002069a9   ti_sysbios_knl_Task_checkStacks__E
00206a55   ti_sysbios_knl_Semaphore_Instance_init__F
00206afd   ti_sysbios_knl_Swi_schedule__I
00206ba5   ti_sysbios_utils_Load_addTask__E
00206c4d   ti_sysbios_family_arm_m3_Hwi_excMemFault__I
00206cf1   __TI_auto_init
00206d91   ti_sysbios_knl_Task_blockI__E
00206e31   __aeabi_memcpy
00206e31   __aeabi_memcpy4
00206e31   __aeabi_memcpy8
00206e31   memcpy
00206f65   xdc_runtime_Text_putSite__E
00206f65   xdc_runtime_Text_putSite__F
00206ff9   xdc_runtime_Text_putMod__E
00206ff9   xdc_runtime_Text_putMod__F
00207089   ti_sysbios_utils_Load_taskCreateHook__E
00207115   TMDXDOCKH52C1_initGeneral
0020721d   ti_sysbios_family_arm_lm3_Timer_Module_startup__E
0020721d   ti_sysbios_family_arm_lm3_Timer_Module_startup__F
0020729d   ti_sysbios_knl_Task_Module_startup__E
0020729d   ti_sysbios_knl_Task_Module_startup__F
0020731d   ti_uia_runtime_LoggerStopMode_getContents__E
0020739d   ti_uia_runtime_LoggerStopMode_setFilterLevel__E
0020741d   UART_init
0020750d   __aeabi_memclr
0020750d   __aeabi_memclr4
0020750d   __aeabi_memclr8
0020750f   __aeabi_memset
0020750f   __aeabi_memset4
0020750f   __aeabi_memset8
00207515   memset
00207585   ti_sysbios_utils_Load_taskDeleteHook__E
002075fd   ti_uia_runtime_LoggerStopMode_getFilterLevel__E
00207751   ti_sysbios_knl_Clock_start__E
002077c1   ti_sysbios_utils_Load_removeTask__E
00207831   xdc_runtime_Memory_alloc__E
00207831   xdc_runtime_Memory_alloc__F
0020790d   ti_uia_runtime_LoggerStopMode_writeBlockOfMemory__I
00207979   xdc_runtime_Error_print__E
00207979   xdc_runtime_Error_print__F
002079e5   ti_sysbios_knl_Task_Object__create__S
00207a4d   xdc_runtime_Core_deleteObject__I
00207b79   GPIO_init
00207bd9   writemsg
00207c03   C$$IO$$
00207c07   readmsg
00207c39   ti_sysbios_knl_Clock_logTick__E
00207c99   ti_sysbios_knl_Clock_startI__E
00207cf9   ti_uia_runtime_LoggerStopMode_Object__create__S
00207db7   ti_uia_runtime_LoggerStopMode_readBlockOfMemory__I
00207e15   xdc_runtime_Text_putLab__E
00207e15   xdc_runtime_Text_putLab__F
00207e6d   ti_sysbios_knl_Swi_restoreHwi__E
00207ec1   TMDXDOCKH52C1_initUART
00207f11   ti_sysbios_utils_Load_taskSwitchHook__E
00207f61   xdc_runtime_Startup_exec__E
00207f61   xdc_runtime_Startup_exec__F
00207fb1   xdc_runtime_System_formatNum__I
00208001   ti_sysbios_family_arm_m3_TaskSupport_buildTaskStack
0020804d   ti_sysbios_fatfs_startup
00208099   ti_sysbios_knl_Clock_getTicks__E
002080e5   ti_uia_runtime_LoggerStopMode_filterOutEvent__I
00208131   ti_uia_runtime_QueueDescriptor_removeFromList__E
0020817d   xdc_runtime_Text_visitRope2__I
002081c9   copy_in
00208211   ti_sysbios_family_arm_m3_Hwi_excReserved__I
00208259   ti_sysbios_heaps_HeapMem_getStats__E
002082a1   xdc_runtime_Assert_raise__I
002082e9   xdc_runtime_Core_assignParams__I
00208331   ti_uia_runtime_LoggerStopMode_Instance_init__F
00208379   _c_int00
00208401   C$$EXIT
00208405   abort
0020840d   exit
00208445   ti_sysbios_BIOS_errorRaiseHook__I
00208489   ti_uia_runtime_LoggerStopMode_reset__E
00208489   ti_uia_runtime_LoggerStopMode_reset__F
002084cd   ti_uia_runtime_QueueDescriptor_addToList__E
00208511   xdc_runtime_SysMin_flush__E
00208511   xdc_runtime_SysMin_flush__F
00208511   xdc_runtime_System_SupportProxy_flush__E
00208511   xdc_runtime_System_flush__E
00208511   xdc_runtime_System_flush__F
00208555   ti_sysbios_family_xxx_Hwi_switchToIsrStack
00208565   ti_sysbios_family_xxx_Hwi_switchToTaskStack
00208571   ti_sysbios_family_arm_m3_Hwi_getTaskSP__E
00208571   ti_sysbios_hal_Hwi_HwiProxy_getTaskSP__E
00208571   ti_sysbios_hal_Hwi_getTaskSP__E
00208577   ti_sysbios_family_arm_m3_Hwi_init__I
002085d5   ti_sysbios_knl_Idle_loop__E
00208615   ti_sysbios_knl_Swi_startup__E
00208655   xdc_runtime_System_atexit__E
00208655   xdc_runtime_System_atexit__F
00208695   ti_sysbios_family_arm_m3_Hwi_disableInterrupt__E
00208695   ti_sysbios_hal_Hwi_HwiProxy_disableInterrupt__E
00208695   ti_sysbios_hal_Hwi_disableInterrupt__E
002086d1   ti_sysbios_family_arm_m3_Hwi_enableInterrupt__E
002086d1   ti_sysbios_hal_Hwi_HwiProxy_enableInterrupt__E
002086d1   ti_sysbios_hal_Hwi_enableInterrupt__E
0020870d   ti_sysbios_family_arm_m3_Hwi_excSvCall__I
00208749   ti_sysbios_heaps_HeapMem_init__I
00208785   ti_sysbios_knl_Clock_Object__create__S
002087c1   ti_sysbios_family_arm_m3_Hwi_excNoIsr__I
002087f9   ti_sysbios_family_arm_m3_Hwi_initVTOR__I
00208831   ti_sysbios_family_arm_m3_TaskSupport_start__E
00208831   ti_sysbios_knl_Task_SupportProxy_start__E
00208869   ti_sysbios_knl_Semaphore_Object__create__S
002088a1   ti_sysbios_knl_Semaphore_pendTimeout__I
002088d9   xdc_runtime_SysMin_putch__E
002088d9   xdc_runtime_SysMin_putch__F
002088d9   xdc_runtime_System_SupportProxy_putch__E
00208911   CPUcpsid
0020891d   CPUprimask
00208927   CPUcpsie
00208933   CPUwfi
00208933   SysCtlSleep
00208937   CPUbasepriSet
00208937   IntPriorityMaskSet
0020893d   CPUbasepriGet
0020893d   IntPriorityMaskGet
00208949   TMDXDOCKH52C1_initGPIO
0020897d   ffcio_lseek
002089b1   ti_sysbios_family_arm_m3_Hwi_excNmi__I
002089e5   ti_sysbios_gates_GateHwi_Object__create__S
00208a19   ti_sysbios_gates_GateMutex_Object__create__S
00208a4d   ti_sysbios_heaps_HeapMem_Object__create__S
00208a81   ti_sysbios_knl_Queue_Object__create__S
00208ab5   ti_sysbios_knl_Task_restore__E
00208b1d   xdc_runtime_Text_printVisFxn__I
00208b4f   strncpy
00208b81   ti_sysbios_BIOS_exitFunc__I
00208bb1   ti_sysbios_family_arm_lm3_Timer_getExpiredCounts__E
00208be1   ti_sysbios_hal_Hwi_checkStack
00208c11   ti_sysbios_knl_Clock_Module_startup__E
00208c11   ti_sysbios_knl_Clock_Module_startup__F
00208c41   xdc_runtime_Core_assignLabel__I
00208c71   xdc_runtime_SysMin_abort__E
00208c71   xdc_runtime_SysMin_abort__F
00208c71   xdc_runtime_System_SupportProxy_abort__E
00208ca1   xdc_runtime_Text_xprintf__I
00208cd1   malloc
00208d2d   ti_sysbios_hal_Hwi_initStack
00208d59   ti_sysbios_knl_Clock_doTick__I
00208d85   ti_sysbios_knl_Task_allBlockedFunction__I
00208db1   ti_uia_runtime_LoggerStopMode_Module_startup__E
00208db1   ti_uia_runtime_LoggerStopMode_Module_startup__F
00208ddd   ti_uia_runtime_LoggerStopMode_disable__E
00208e09   ti_uia_runtime_LoggerStopMode_enable__E
00208e35   xdc_runtime_System_rtsExit__I
00208e61   xdc_runtime_Text_cordText__E
00208e61   xdc_runtime_Text_cordText__F
00208e8d   ti_sysbios_BIOS_startFunc__I
00208eb5   ti_sysbios_family_arm_f28m35x_TimestampProvider_get64__E
00208eb5   ti_uia_runtime_LogSync_CpuTimestampProxy_get64__E
00208eb5   xdc_runtime_Timestamp_SupportProxy_get64__E
00208eb5   xdc_runtime_Timestamp_get64__E
00208eb5   xdc_runtime_Timestamp_get64__F
00208edd   ti_sysbios_gates_GateMutex_Instance_init__F
00208f2d   ti_uia_runtime_LogSync_Module_startup__E
00208f2d   ti_uia_runtime_LogSync_Module_startup__F
00208f55   ti_uia_runtime_QueueDescriptor_initHeader__E
00208fa1   ffcio_close
00208fe9   ti_sysbios_BIOS_registerRTSLock__I
0020900d   ti_sysbios_family_arm_lm3_Timer_isrStub__E
00209031   ti_sysbios_family_arm_m3_Hwi_doTaskRestore__I
00209055   ti_sysbios_gates_GateMutex_Object__delete__S
00209079   ti_sysbios_knl_Swi_Module_startup__E
00209079   ti_sysbios_knl_Swi_Module_startup__F
0020909d   ti_uia_runtime_LoggerStopMode_Instance_finalize__F
002090c1   xdc_runtime_SysMin_output__I
002090e5   ffcio_read
00209105   ffcio_write
00209125   ti_sysbios_gates_GateHwi_Object__delete__S
00209145   ti_sysbios_heaps_HeapMem_Object__delete__S
00209165   ti_sysbios_knl_Clock_Object__destruct__S
00209185   ti_sysbios_knl_Semaphore_Object__destruct__S
002091a5   ti_sysbios_knl_Task_enter__I
002091c5   ti_uia_runtime_LoggerStopMode_Object__delete__S
002091e5   xdc_runtime_Registry_findById__E
002091e5   xdc_runtime_Registry_findById__F
00209205   xdc_runtime_SysMin_Module_startup__E
00209205   xdc_runtime_SysMin_Module_startup__F
00209225   xdc_runtime_System_avprintf__F
00209245   xdc_runtime_System_putchar__I
00209265   xdc_runtime_System_vprintf__F
00209285   disk_initialize
002092a1   disk_ioctl
002092bd   disk_read
002092d9   disk_status
002092f5   disk_write
00209311   free
00209349   ti_sysbios_knl_Queue_Object__destruct__S
00209365   xdc_runtime_Error_check__E
00209365   xdc_runtime_Error_check__F
00209381   xdc_runtime_Memory_valloc__E
00209381   xdc_runtime_Memory_valloc__F
0020939d   xdc_runtime_SysMin_exit__E
0020939d   xdc_runtime_SysMin_exit__F
0020939d   xdc_runtime_System_SupportProxy_exit__E
002093b9   ti_sysbios_gates_GateHwi_Handle__label__S
002093d3   ti_sysbios_gates_GateMutex_Handle__label__S
002093ed   ti_sysbios_heaps_HeapMem_Handle__label__S
00209407   ti_uia_runtime_LoggerStopMode_Handle__label__S
00209421   xdc_runtime_System_aprintf__E
0020943b   xdc_runtime_System_printf__E
00209455   clust2sect
0020946d   _register_unlock
00209473   _register_lock
00209479   _nop
00209485   _args_main
0020949d   strcmp
002094b5   ti_sysbios_family_arm_lm3_Timer_Module__startupDone__F
002094b5   ti_sysbios_family_arm_lm3_Timer_Module__startupDone__S
002094cd   ti_sysbios_family_arm_m3_Hwi_Module__startupDone__F
002094cd   ti_sysbios_family_arm_m3_Hwi_Module__startupDone__S
002094e5   ti_sysbios_gates_GateMutex_leave__E
002094fd   ti_sysbios_hal_Timer_Module__startupDone__F
002094fd   ti_sysbios_hal_Timer_Module__startupDone__S
0020952d   xdc_runtime_Text_ropeText__E
0020952d   xdc_runtime_Text_ropeText__F
00209545   strchr
00209571   ti_uia_runtime_LoggerStopMode_getFreeSize__E
00209587   ti_uia_runtime_LoggerStopMode_getUnreadSize__E
0020959d   strlen
002095b1   ti_sysbios_family_arm_m3_Hwi_switchFromBootStack__E
002095b1   ti_sysbios_hal_Hwi_HwiProxy_switchFromBootStack__E
002095b1   ti_sysbios_hal_Hwi_switchFromBootStack__E
002095c5   ti_sysbios_gates_GateHwi_enter__E
002095d9   ti_sysbios_heaps_HeapMem_Object__get__S
002095ed   ti_sysbios_knl_Swi_Object__get__S
00209601   ti_sysbios_knl_Task_Object__first__S
00209615   ti_sysbios_knl_Task_Object__get__S
00209629   ti_sysbios_knl_Task_Object__next__S
0020963d   ti_uia_runtime_LoggerStopMode_write2__E
00209651   xdc_runtime_System_abort__E
00209651   xdc_runtime_System_abort__F
00209665   __TI_zero_init
00209677   ffcio_rename
00209689   ffcio_unlink
0020969b   strcpy
002096ad   ti_sysbios_hal_Hwi_Module_startup__E
002096ad   ti_sysbios_hal_Hwi_Module_startup__F
002096bf   ti_sysbios_hal_Timer_Module_startup__E
002096bf   ti_sysbios_hal_Timer_Module_startup__F
002096d1   ti_uia_runtime_LoggerStopMode_write1__E
002096e3   xdc_runtime_Startup_exec__I
00209705   ti_sysbios_family_arm_m3_TaskSupport_glue
00209715   ti_sysbios_family_arm_m3_TaskSupport_swap__E
00209715   ti_sysbios_knl_Task_SupportProxy_swap__E
00209735   f_close
00209755   ti_sysbios_BIOS_setThreadType__E
00209765   ti_sysbios_BIOS_start__E
00209775   ti_sysbios_family_arm_f28m35x_TimestampProvider_getFreq__E
00209775   ti_uia_runtime_LogSync_CpuTimestampProxy_getFreq__E
00209775   xdc_runtime_Timestamp_SupportProxy_getFreq__E
00209775   xdc_runtime_Timestamp_getFreq__E
00209775   xdc_runtime_Timestamp_getFreq__F
00209785   ti_sysbios_family_arm_m3_Hwi_excHandler__I
00209795   ti_sysbios_gates_GateMutex_Instance_finalize__F
002097a5   ti_sysbios_knl_Semaphore_Instance_finalize__F
002097b5   ti_sysbios_knl_Swi_disable__E
002097c5   ti_sysbios_knl_Task_disable__E
002097d5   ti_uia_runtime_LoggerStopMode_Object__get__S
002097e5   ti_uia_runtime_LoggerStopMode_isEmpty__E
002097f5   ti_uia_runtime_LoggerStopMode_write0__E
00209805   xdc_runtime_Gate_leaveSystem__E
00209805   xdc_runtime_Gate_leaveSystem__F
00209815   xdc_runtime_Memory_free__E
00209815   xdc_runtime_Memory_free__F
00209825   xdc_runtime_SysMin_ready__E
00209825   xdc_runtime_SysMin_ready__F
00209825   xdc_runtime_System_SupportProxy_ready__E
00209835   xdc_runtime_Text_visitRope__I
00209845   __TI_decompress_none
00209861   ti_sysbios_family_arm_m3_TaskSupport_checkStack__E
00209861   ti_sysbios_knl_Task_SupportProxy_checkStack__E
0020986f   ti_sysbios_knl_Queue_empty__E
0020987d   xdc_runtime_System_vsprintf__F
0020988b   ti_catalog_arm_cortexm3_concertoInit_Boot_init
00209897   ti_catalog_arm_cortexm3_concertoInit_Boot_initStartup
002098b1   ti_sysbios_family_arm_f28m35x_TimestampProvider_get32__E
002098b1   ti_uia_runtime_LogSync_CpuTimestampProxy_get32__E
002098b1   xdc_runtime_Timestamp_SupportProxy_get32__E
002098b1   xdc_runtime_Timestamp_get32__E
002098b1   xdc_runtime_Timestamp_get32__F
002098bd   ti_sysbios_family_arm_m3_TaskSupport_getStackAlignment__E
002098bd   ti_sysbios_knl_Task_SupportProxy_getStackAlignment__E
002098c9   ti_sysbios_knl_Clock_Params__init__S
002098d5   ti_sysbios_knl_Queue_Object__get__S
002098e1   ti_sysbios_knl_Task_Params__init__S
002098ed   ti_sysbios_utils_Load_taskRegHook__E
002098f9   xdc_runtime_Error_init__E
002098f9   xdc_runtime_Error_init__F
00209905   xdc_runtime_Gate_enterSystem__E
00209905   xdc_runtime_Gate_enterSystem__F
00209911   xdc_runtime_Memory_calloc__E
00209911   xdc_runtime_Memory_calloc__F
0020991d   xdc_runtime_Memory_getMaxDefaultTypeAlign__E
0020991d   xdc_runtime_Memory_getMaxDefaultTypeAlign__F
00209929   xdc_runtime_System_exit__E
00209929   xdc_runtime_System_exit__F
00209935   xdc_runtime_System_lastFxn__I
00209941   ti_sysbios_family_arm_m3_IntrinsicsSupport_maxbit__E
00209941   ti_sysbios_knl_Intrinsics_SupportProxy_maxbit__E
00209941   ti_sysbios_knl_Intrinsics_maxbit__E
0020995f   ff_req_grant
00209967   ti_sysbios_family_arm_m3_Hwi_startup__E
00209967   ti_sysbios_hal_Hwi_HwiProxy_startup__E
00209967   ti_sysbios_hal_Hwi_startup__E
00209971   get_fattime
00209971   ti_sysbios_fatfs_getFatTime
00209979   ti_catalog_arm_cortexm3_concertoInit_Boot_stepDelay
00209981   SysCtlDelay
00209987   __xdc__init
0020998d   __TI_decompress_rle24
00209999   ti_sysbios_family_arm_m3_Hwi_doSwiRestore__I
0020999f   ti_sysbios_gates_GateHwi_leave__E
002099a5   ti_sysbios_heaps_HeapMem_isBlocking__E
002099ab   ti_sysbios_knl_Queue_Instance_init__F
002099b1   ti_uia_runtime_LoggerStopMode_getPriority__E
002099b7   ti_uia_runtime_LoggerStopMode_getTransferType__E
002099b7   ti_uia_runtime_LoggerStopMode_getTransferType__F
002099bd   xdc_runtime_System_Module_startup__E
002099bd   xdc_runtime_System_Module_startup__F
002099c3   ti_catalog_arm_cortexm3_concertoInit_Boot_limpAbort
002099c7   ff_rel_grant
002099cb   ti_sysbios_BIOS_RtsGateProxy_enter__E
002099cf   ti_sysbios_BIOS_RtsGateProxy_leave__E
002099d3   ti_sysbios_family_arm_lm3_Timer_getPeriod__E
002099d7   ti_sysbios_family_arm_m3_TaskSupport_Module__startupDone__S
002099db   ti_sysbios_gates_GateHwi_query__E
002099db   ti_sysbios_gates_GateHwi_query__F
002099db   xdc_runtime_Main_Module_GateProxy_query__E
002099db   xdc_runtime_System_Module_GateProxy_query__E
002099df   ti_sysbios_BIOS_RtsGateProxy_query__E
002099df   ti_sysbios_gates_GateMutex_query__E
002099df   ti_sysbios_gates_GateMutex_query__F
002099df   ti_sysbios_heaps_HeapMem_Module_GateProxy_query__E
002099e3   ti_sysbios_hal_Hwi_HwiProxy_Module__startupDone__S
002099e7   ti_sysbios_hal_Timer_TimerProxy_Module__startupDone__S
002099eb   ti_sysbios_hal_Timer_TimerProxy_getExpiredCounts__E
002099ef   ti_sysbios_hal_Timer_TimerProxy_getPeriod__E
002099f3   ti_sysbios_hal_Timer_TimerProxy_setNextTick__E
002099f7   ti_sysbios_heaps_HeapMem_Module_GateProxy_enter__E
002099fb   ti_sysbios_heaps_HeapMem_Module_GateProxy_leave__E
002099ff   ti_sysbios_knl_Task_SupportProxy_Module__startupDone__S
00209a03   ti_uia_runtime_LogSync_CpuTimestampProxy_Module__startupDone__S
00209a07   ti_uia_runtime_LogSync_GlobalTimestampProxy_Module__startupDone__S
00209a0b   ti_uia_runtime_LoggerStopMode_getInstanceId__E
00209a0f   ti_uia_runtime_LoggerStopMode_getMaxLength__E
00209a13   ti_uia_runtime_LoggerStopMode_setPriority__E
00209a17   xdc_runtime_Error_getSite__E
00209a17   xdc_runtime_Error_getSite__F
00209a1b   xdc_runtime_Memory_HeapProxy_alloc__E
00209a1f   xdc_runtime_Memory_HeapProxy_free__E
00209a23   xdc_runtime_Startup_reset__I
00209a27   xdc_runtime_System_Module_GateProxy_enter__E
00209a2b   xdc_runtime_System_Module_GateProxy_leave__E
00209a2f   xdc_runtime_System_aprintf_va__F
00209a33   xdc_runtime_System_printf_va__F
00209a37   xdc_runtime_System_vsprintf__E
00209a3b   xdc_runtime_TimestampNull_Module__startupDone__S
00209a3f   xdc_runtime_Timestamp_Module__startupDone__S
00209a50   xdc_runtime_Text_charTab__A
0020b7d0   xdc_runtime_Text_nodeTab__A
0020b8d0   GPIO_config
0020b8d8   uartHWAttrs
0020b8e0   UART_config
0020b8ec   emacHWAttrs
0020b8f4   EMAC_config
0020b900   SDSPI_config
0020b90c   USBMSCHFatFsHWAttrs
0020b910   USBMSCHFatFs_config
0020b91c   I2CHWAttrs
0020b92c   I2C_config
0020b938   ti_uia_runtime_LoggerStopMode_Module__FXNS__C
0020bac4   ti_sysbios_knl_Task_Object__PARAMS__C
0020bafc   ti_sysbios_knl_Task_hooks__A
0020bb2c   ti_uia_runtime_LoggerStopMode_Object__PARAMS__C
0020bb5c   xdc_runtime_Startup_sfxnTab__A
0020bb88   sdspiHWAttrs
0020bbb0   ti_sysbios_heaps_HeapMem_Module__FXNS__C
0020bbd8   gpioHWAttrs
0020bbfc   ti_sysbios_gates_GateHwi_Module__FXNS__C
0020bc20   ti_sysbios_gates_GateMutex_Module__FXNS__C
0020bc44   ti_sysbios_knl_Clock_Object__PARAMS__C
0020bc68   ti_sysbios_knl_Semaphore_Object__PARAMS__C
0020bccc   ti_sysbios_gates_GateHwi_Object__DESC__C
0020bcec   ti_sysbios_gates_GateMutex_Object__DESC__C
0020bd0c   ti_sysbios_heaps_HeapMem_Object__DESC__C
0020bd2c   ti_sysbios_heaps_HeapMem_Object__PARAMS__C
0020bd4c   ti_sysbios_knl_Clock_Object__DESC__C
0020bd6c   ti_sysbios_knl_Queue_Object__DESC__C
0020bd8c   ti_sysbios_knl_Semaphore_Object__DESC__C
0020bdac   ti_sysbios_knl_Task_Object__DESC__C
0020bdcc   ti_uia_runtime_LoggerStopMode_Object__DESC__C
0020bdec   ti_sysbios_gates_GateHwi_Object__PARAMS__C
0020be04   ti_sysbios_gates_GateMutex_Object__PARAMS__C
0020be1c   ti_sysbios_knl_Queue_Object__PARAMS__C
0020be34   xdc_runtime_Startup_sfxnRts__A
0020be4c   xdc_runtime_Startup_firstFxns__A
0020be74   ti_sysbios_knl_Idle_funcList__A
0020be7c   ti_sysbios_knl_Idle_funcList__C
0020be84   ti_sysbios_knl_Task_hooks__C
0020be8c   xdc_runtime_Startup_firstFxns__C
0020be94   xdc_runtime_Startup_lastFxns__C
0020be9c   ti_sysbios_BIOS_Module__diagsEnabled__C
0020bea0   ti_sysbios_BIOS_Module__diagsIncluded__C
0020bea4   ti_sysbios_BIOS_Module__diagsMask__C
0020bea8   ti_sysbios_BIOS_installedErrorHook__C
0020beac   ti_sysbios_family_arm_lm3_Timer_WRALLOW__C
0020beb0   ti_sysbios_family_arm_lm3_Timer_numTimerDevices__C
0020beb4   ti_sysbios_family_arm_lm3_Timer_startupNeeded__C
0020beb8   ti_sysbios_family_arm_m3_Hwi_E_NMI__C
0020bebc   ti_sysbios_family_arm_m3_Hwi_E_busFault__C
0020bec0   ti_sysbios_family_arm_m3_Hwi_E_debugMon__C
0020bec4   ti_sysbios_family_arm_m3_Hwi_E_hardFault__C
0020bec8   ti_sysbios_family_arm_m3_Hwi_E_memFault__C
0020becc   ti_sysbios_family_arm_m3_Hwi_E_noIsr__C
0020bed0   ti_sysbios_family_arm_m3_Hwi_E_reserved__C
0020bed4   ti_sysbios_family_arm_m3_Hwi_E_svCall__C
0020bed8   ti_sysbios_family_arm_m3_Hwi_E_usageFault__C
0020bedc   ti_sysbios_family_arm_m3_Hwi_LD_end__C
0020bee0   ti_sysbios_family_arm_m3_Hwi_LM_begin__C
0020bee4   ti_sysbios_family_arm_m3_Hwi_Module__diagsEnabled__C
0020bee8   ti_sysbios_family_arm_m3_Hwi_Module__diagsIncluded__C
0020beec   ti_sysbios_family_arm_m3_Hwi_Module__diagsMask__C
0020bef0   ti_sysbios_family_arm_m3_Hwi_Module__loggerFxn1__C
0020bef4   ti_sysbios_family_arm_m3_Hwi_Module__loggerFxn8__C
0020bef8   ti_sysbios_family_arm_m3_Hwi_Module__loggerObj__C
0020befc   ti_sysbios_family_arm_m3_Hwi_NUM_INTERRUPTS__C
0020bf00   ti_sysbios_family_arm_m3_Hwi_ccr__C
0020bf04   ti_sysbios_family_arm_m3_Hwi_disablePriority__C
0020bf08   ti_sysbios_family_arm_m3_Hwi_excHandlerFunc__C
0020bf0c   ti_sysbios_family_arm_m3_Hwi_excHookFunc__C
0020bf10   ti_sysbios_family_arm_m3_Hwi_priGroup__C
0020bf14   ti_sysbios_family_arm_m3_TaskSupport_stackAlignment__C
0020bf18   ti_sysbios_gates_GateMutex_A_badContext__C
0020bf1c   ti_sysbios_gates_GateMutex_Instance_State_sem__O
0020bf20   ti_sysbios_gates_GateMutex_Module__diagsEnabled__C
0020bf24   ti_sysbios_gates_GateMutex_Module__diagsIncluded__C
0020bf28   ti_sysbios_gates_GateMutex_Module__diagsMask__C
0020bf2c   ti_sysbios_hal_Hwi_E_stackOverflow__C
0020bf30   ti_sysbios_heaps_HeapMem_A_align__C
0020bf34   ti_sysbios_heaps_HeapMem_A_heapSize__C
0020bf38   ti_sysbios_heaps_HeapMem_A_invalidFree__C
0020bf3c   ti_sysbios_heaps_HeapMem_A_zeroBlock__C
0020bf40   ti_sysbios_heaps_HeapMem_E_memory__C
0020bf44   ti_sysbios_heaps_HeapMem_Module__diagsEnabled__C
0020bf48   ti_sysbios_heaps_HeapMem_Module__diagsIncluded__C
0020bf4c   ti_sysbios_heaps_HeapMem_Module__diagsMask__C
0020bf50   ti_sysbios_heaps_HeapMem_Module__gateObj__C
0020bf54   ti_sysbios_heaps_HeapMem_Object__count__C
0020bf58   ti_sysbios_heaps_HeapMem_reqAlignMask__C
0020bf5c   ti_sysbios_heaps_HeapMem_reqAlign__C
0020bf60   ti_sysbios_knl_Clock_A_badThreadType__C
0020bf64   ti_sysbios_knl_Clock_LM_begin__C
0020bf68   ti_sysbios_knl_Clock_LM_tick__C
0020bf6c   ti_sysbios_knl_Clock_LW_delayed__C
0020bf70   ti_sysbios_knl_Clock_Module_State_clockQ__O
0020bf74   ti_sysbios_knl_Clock_Module__diagsEnabled__C
0020bf78   ti_sysbios_knl_Clock_Module__diagsIncluded__C
0020bf7c   ti_sysbios_knl_Clock_Module__diagsMask__C
0020bf80   ti_sysbios_knl_Clock_Module__loggerFxn1__C
0020bf84   ti_sysbios_knl_Clock_Module__loggerFxn2__C
0020bf88   ti_sysbios_knl_Clock_Module__loggerObj__C
0020bf8c   ti_sysbios_knl_Semaphore_A_badContext__C
0020bf90   ti_sysbios_knl_Semaphore_A_noEvents__C
0020bf94   ti_sysbios_knl_Semaphore_Instance_State_pendQ__O
0020bf98   ti_sysbios_knl_Semaphore_LM_pend__C
0020bf9c   ti_sysbios_knl_Semaphore_LM_post__C
0020bfa0   ti_sysbios_knl_Semaphore_Module__diagsEnabled__C
0020bfa4   ti_sysbios_knl_Semaphore_Module__diagsIncluded__C
0020bfa8   ti_sysbios_knl_Semaphore_Module__diagsMask__C
0020bfac   ti_sysbios_knl_Semaphore_Module__loggerFxn2__C
0020bfb0   ti_sysbios_knl_Semaphore_Module__loggerFxn4__C
0020bfb4   ti_sysbios_knl_Semaphore_Module__loggerObj__C
0020bfb8   ti_sysbios_knl_Swi_LD_end__C
0020bfbc   ti_sysbios_knl_Swi_LM_begin__C
0020bfc0   ti_sysbios_knl_Swi_LM_post__C
0020bfc4   ti_sysbios_knl_Swi_Module__diagsEnabled__C
0020bfc8   ti_sysbios_knl_Swi_Module__diagsIncluded__C
0020bfcc   ti_sysbios_knl_Swi_Module__diagsMask__C
0020bfd0   ti_sysbios_knl_Swi_Module__loggerFxn1__C
0020bfd4   ti_sysbios_knl_Swi_Module__loggerFxn4__C
0020bfd8   ti_sysbios_knl_Swi_Module__loggerObj__C
0020bfdc   ti_sysbios_knl_Swi_Object__count__C
0020bfe0   ti_sysbios_knl_Task_A_badPriority__C
0020bfe4   ti_sysbios_knl_Task_A_badTaskState__C
0020bfe8   ti_sysbios_knl_Task_A_badThreadType__C
0020bfec   ti_sysbios_knl_Task_A_noPendElem__C
0020bff0   ti_sysbios_knl_Task_E_spOutOfBounds__C
0020bff4   ti_sysbios_knl_Task_E_stackOverflow__C
0020bff8   ti_sysbios_knl_Task_LD_block__C
0020bffc   ti_sysbios_knl_Task_LD_exit__C
0020c000   ti_sysbios_knl_Task_LD_ready__C
0020c004   ti_sysbios_knl_Task_LM_switch__C
0020c008   ti_sysbios_knl_Task_Module_State_inactiveQ__O
0020c00c   ti_sysbios_knl_Task_Module_State_terminatedQ__O
0020c010   ti_sysbios_knl_Task_Module__diagsEnabled__C
0020c014   ti_sysbios_knl_Task_Module__diagsIncluded__C
0020c018   ti_sysbios_knl_Task_Module__diagsMask__C
0020c01c   ti_sysbios_knl_Task_Module__loggerFxn2__C
0020c020   ti_sysbios_knl_Task_Module__loggerFxn4__C
0020c024   ti_sysbios_knl_Task_Module__loggerObj__C
0020c028   ti_sysbios_knl_Task_Object__count__C
0020c02c   ti_sysbios_knl_Task_Object__heap__C
0020c030   ti_sysbios_knl_Task_allBlockedFunc__C
0020c034   ti_sysbios_knl_Task_defaultStackHeap__C
0020c038   ti_sysbios_knl_Task_defaultStackSize__C
0020c03c   ti_sysbios_knl_Task_numConstructedTasks__C
0020c040   ti_sysbios_knl_Task_numPriorities__C
0020c044   ti_sysbios_utils_Load_LS_cpuLoad__C
0020c048   ti_sysbios_utils_Load_LS_hwiLoad__C
0020c04c   ti_sysbios_utils_Load_LS_swiLoad__C
0020c050   ti_sysbios_utils_Load_LS_taskLoad__C
0020c054   ti_sysbios_utils_Load_Module_State_gate__O
0020c058   ti_sysbios_utils_Load_Module_State_taskList__O
0020c05c   ti_sysbios_utils_Load_Module__diagsEnabled__C
0020c060   ti_sysbios_utils_Load_Module__diagsIncluded__C
0020c064   ti_sysbios_utils_Load_Module__diagsMask__C
0020c068   ti_sysbios_utils_Load_Module__loggerFxn1__C
0020c06c   ti_sysbios_utils_Load_Module__loggerFxn2__C
0020c070   ti_sysbios_utils_Load_Module__loggerFxn4__C
0020c074   ti_sysbios_utils_Load_Module__loggerObj__C
0020c078   ti_sysbios_utils_Load_postUpdate__C
0020c07c   ti_sysbios_utils_Load_windowInMs__C
0020c080   ti_uia_runtime_ILoggerSnapshot_Interface__BASE__C
0020c084   ti_uia_runtime_IUIATransfer_Interface__BASE__C
0020c088   ti_uia_runtime_LoggerStopMode_E_badLevel__C
0020c08c   ti_uia_runtime_LoggerStopMode_Object__count__C
0020c090   ti_uia_runtime_LoggerStopMode_overflowLogger__C
0020c094   ti_uia_runtime_LoggerStopMode_statusLogger__C
0020c098   xdc_runtime_Assert_E_assertFailed__C
0020c09c   xdc_runtime_Core_A_initializedParams__C
0020c0a0   xdc_runtime_Core_Module__diagsEnabled__C
0020c0a4   xdc_runtime_Core_Module__diagsIncluded__C
0020c0a8   xdc_runtime_Core_Module__diagsMask__C
0020c0ac   xdc_runtime_Error_E_generic__C
0020c0b0   xdc_runtime_Error_E_memory__C
0020c0b4   xdc_runtime_Error_Module__diagsEnabled__C
0020c0b8   xdc_runtime_Error_Module__diagsIncluded__C
0020c0bc   xdc_runtime_Error_Module__diagsMask__C
0020c0c0   xdc_runtime_Error_Module__loggerFxn8__C
0020c0c4   xdc_runtime_Error_Module__loggerObj__C
0020c0c8   xdc_runtime_Error_raiseHook__C
0020c0cc   xdc_runtime_IFilterLogger_Interface__BASE__C
0020c0d0   xdc_runtime_IGateProvider_Interface__BASE__C
0020c0d4   xdc_runtime_IHeap_Interface__BASE__C
0020c0d8   xdc_runtime_ILogger_Interface__BASE__C
0020c0dc   xdc_runtime_IModule_Interface__BASE__C
0020c0e0   xdc_runtime_Log_L_error__C
0020c0e4   xdc_runtime_Main_Module__diagsEnabled__C
0020c0e8   xdc_runtime_Main_Module__diagsIncluded__C
0020c0ec   xdc_runtime_Main_Module__diagsMask__C
0020c0f0   xdc_runtime_Main_Module__loggerFxn4__C
0020c0f4   xdc_runtime_Main_Module__loggerObj__C
0020c0f8   xdc_runtime_Memory_defaultHeapInstance__C
0020c0fc   xdc_runtime_Startup_execImpl__C
0020c100   xdc_runtime_Startup_lastFxns__A
0020c104   xdc_runtime_Startup_maxPasses__C
0020c108   xdc_runtime_Startup_sfxnRts__C
0020c10c   xdc_runtime_Startup_sfxnTab__C
0020c110   xdc_runtime_SysMin_bufSize__C
0020c114   xdc_runtime_SysMin_outputFunc__C
0020c118   xdc_runtime_System_Module__gateObj__C
0020c11c   xdc_runtime_System_extendFxn__C
0020c120   xdc_runtime_System_maxAtexitHandlers__C
0020c124   xdc_runtime_Text_charTab__C
0020c128   xdc_runtime_Text_nameEmpty__C
0020c12c   xdc_runtime_Text_nameStatic__C
0020c130   xdc_runtime_Text_nameUnknown__C
0020c134   xdc_runtime_Text_nodeTab__C
0020c138   xdc_runtime_Text_visitRopeFxn__C
0020c13c   ti_sysbios_BIOS_Module__id__C
0020c140   ti_sysbios_family_arm_m3_Hwi_Module__id__C
0020c144   ti_sysbios_family_arm_m3_Hwi_Module__loggerDefined__C
0020c148   ti_sysbios_gates_GateMutex_Module__id__C
0020c14c   ti_sysbios_hal_Hwi_Module__id__C
0020c150   ti_sysbios_heaps_HeapMem_Module__id__C
0020c154   ti_sysbios_knl_Clock_Module__id__C
0020c158   ti_sysbios_knl_Clock_Module__loggerDefined__C
0020c15c   ti_sysbios_knl_Semaphore_Module__id__C
0020c160   ti_sysbios_knl_Semaphore_Module__loggerDefined__C
0020c164   ti_sysbios_knl_Swi_Module__id__C
0020c168   ti_sysbios_knl_Swi_Module__loggerDefined__C
0020c16c   ti_sysbios_knl_Task_Module__id__C
0020c170   ti_sysbios_knl_Task_Module__loggerDefined__C
0020c174   ti_sysbios_knl_Task_deleteTerminatedTasks__C
0020c178   ti_sysbios_knl_Task_initStackFlag__C
0020c17c   ti_sysbios_utils_Load_Module__id__C
0020c180   ti_sysbios_utils_Load_Module__loggerDefined__C
0020c184   ti_sysbios_utils_Load_autoAddTasks__C
0020c188   ti_sysbios_utils_Load_hwiEnabled__C
0020c18c   ti_sysbios_utils_Load_swiEnabled__C
0020c190   ti_sysbios_utils_Load_taskEnabled__C
0020c194   ti_sysbios_utils_Load_updateInIdle__C
0020c198   ti_uia_runtime_LoggerStopMode_Module__id__C
0020c19c   ti_uia_runtime_LoggerStopMode_filterByLevel__C
0020c1a0   ti_uia_runtime_LoggerStopMode_isTimestampEnabled__C
0020c1a4   xdc_runtime_Core_Module__id__C
0020c1a8   xdc_runtime_Error_Module__loggerDefined__C
0020c1ac   xdc_runtime_Error_maxDepth__C
0020c1b0   xdc_runtime_Main_Module__id__C
0020c1b4   xdc_runtime_Main_Module__loggerDefined__C
0020c1b8   xdc_runtime_Memory_Module__id__C
0020c1bc   xdc_runtime_SysMin_flushAtExit__C
0020c1c0   xdc_runtime_Text_charCnt__C
0020c1c4   xdc_runtime_Text_isLoaded__C
0020c1c8   xdc_runtime_Text_registryModsLastId__C
0020c1cc   xdc_runtime_Text_unnamedModsLastId__C
0020c1d0   ti_sysbios_knl_Clock_tickMode__C
0020c1d4   ti_sysbios_knl_Clock_tickSource__C
0020c1d8   xdc_runtime_Error_policy__C
0020c6d0   __TI_Handler_Table_Base
0020c6dc   __TI_Handler_Table_Limit
0020c6f0   __TI_CINIT_Base
0020c708   __TI_CINIT_Limit
0020c708   __TI_static_base__
0020c708   __TI_table_binit
0020c708   __binit__
0020c708   binit
20000000   ti_sysbios_family_arm_m3_Hwi_ramVectors
200001ad   ti_catalog_arm_cortexm3_concertoInit_Boot_initFlash
200001e8   ti_sysbios_heaps_HeapMem_Instance_State_0_buf__A
200011e8   ti_sysbios_knl_Task_Instance_State_0_stack__A
200019e8   ti_uia_runtime_LoggerStopMode_Instance_State_1_bufferArray__A
20001e68   ti_uia_runtime_LoggerStopMode_Instance_State_2_bufferArray__A
200022e8   xdc_runtime_SysMin_Module_State_0_outbuf__A
200026e8   ti_uia_runtime_LoggerStopMode_Instance_State_0_bufferArray__A
20002968   __CIOBUF_
20002b50   I2CObjects
20002bc0   uartObjects
20002c0c   taskParams
20002c44   tMB_State
20002c48   Sem
20002c4c   echo
20002c50   TimerHd_Counter
20002c54   a
20002c64   pt
20002c65   n
20002c66   mb_tx_data
20002c67   input
20002c78   eb
20002cd0   emacObjects
20002cd4   sdspiObjects
20002ce0   USBMSCHFatFsObjects
20002ce8   ti_sysbios_knl_Task_Instance_State_0_hookEnv__A
20008000   __stack
20008100   __STACK_TOP
20009000   __STACK_END
20009000   ti_sysbios_BIOS_Module__state__V
2000901c   ti_sysbios_family_arm_f28m35x_TimestampProvider_Module__state__V
20009024   ti_sysbios_family_arm_lm3_Timer_Module__root__V
2000902c   ti_sysbios_family_arm_lm3_Timer_Module_State_0_device__A
2000904c   ti_sysbios_family_arm_lm3_Timer_Module_State_0_handles__A
2000905c   ti_sysbios_family_arm_lm3_Timer_Module__state__V
20009068   ti_sysbios_family_arm_m3_Hwi_Module__root__V
20009070   ti_sysbios_family_arm_m3_Hwi_Object__table__V
20009088   ti_sysbios_gates_GateHwi_Module__root__V
20009090   ti_sysbios_gates_GateHwi_Object__table__V
20009094   ti_sysbios_gates_GateMutex_Module__root__V
2000909c   ti_sysbios_hal_Hwi_Module__root__V
200090a4   ti_sysbios_hal_Timer_Module__root__V
200090ac   ti_sysbios_hal_Timer_Object__table__V
200090b4   ti_sysbios_heaps_HeapMem_Module__root__V
200090bc   ti_sysbios_heaps_HeapMem_Object__table__V
200090d0   ti_sysbios_knl_Clock_Module__root__V
200090d8   ti_sysbios_knl_Event_Module__root__V
200090e4   ti_sysbios_knl_Queue_Module__root__V
200090ec   ti_sysbios_knl_Semaphore_Module__root__V
200090f8   ti_sysbios_knl_Swi_Module__root__V
20009100   ti_sysbios_knl_Swi_Module__state__V
2000911c   ti_sysbios_knl_Task_Module__root__V
20009128   ti_sysbios_utils_Load_Module__root__V
2000912c   ti_uia_runtime_LogSync_Module__root__V
20009134   ti_uia_runtime_LogSync_Module__state__V
20009140   ti_uia_runtime_LoggerStopMode_Module__root__V
20009148   ti_uia_runtime_LoggerStopMode_Module__state__V
20009150   xdc_runtime_Error_Module__state__V
20009152   xdc_runtime_Main_Module__root__V
20009154   xdc_runtime_Memory_Module__state__V
20009158   xdc_runtime_Registry_Module__state__V
20009160   xdc_runtime_Startup_Module__state__V
20009168   xdc_runtime_SysMin_Module__state__V
20009174   xdc_runtime_System_Module_State_0_atexitHandlers__A
20009194   xdc_runtime_System_Module__state__V
200091a0   xdc_runtime_Text_Module__state__V
200091a8   __xdc__init__addr
200091ac   ti_sysbios_family_arm_m3_Hwi_Module_State_0_dispatchTable__A
20009358   ti_uia_runtime_LoggerStopMode_Object__table__V
20009460   ti_sysbios_utils_Load_Module__state__V
200094f8   ti_sysbios_knl_Swi_Module_State_0_readyQ__A
20009578   ti_sysbios_knl_Task_Module_State_0_readyQ__A
20009670   ti_sysbios_family_arm_m3_Hwi_Module_State_0_priorities__A
2000977c   ti_sysbios_family_arm_m3_Hwi_Module__state__V
200097cc   TSK_idle
200097cc   ti_sysbios_knl_Task_Object__table__V
20009814   ti_sysbios_gates_GateMutex_Object__table__V
2000984c   ti_sysbios_knl_Task_Module__state__V
20009880   ti_sysbios_family_arm_lm3_Timer_Object__table__V
200098b0   ti_sysbios_knl_Swi_Object__table__V
200098e0   ti_sysbios_knl_Clock_Module__state__V
20009920   _lock
20009924   _unlock
20009928   _cleanup_ptr
2000992c   _dtors_ptr
20009930   ti_uia_runtime_QueueDescriptor_gPtrToFirstDescriptor
20009934   ti_uia_runtime_QueueDescriptor_gUpdateCount
20009938   macAddress
20009948   main_func_sp
40000400   ti_sysbios_family_arm_ducati_CTM_ctm
e000e000   ti_sysbios_family_arm_m3_Hwi_nvic
ffffffff   __c_args__
UNDEFED    SHT$$INIT_ARRAY$$Base
UNDEFED    SHT$$INIT_ARRAY$$Limit

[978 symbols]
